:020000040800F2
:10000000384D0020E1010008516200081537000852
:1000100079610008D9030008397600080000000063
:10002000000000000000000000000000490100087E
:10003000F5040008000000008D010008AD6D000807
:10004000FB010008FB010008FB0100088D690008A6
:10005000FB010008FB010008FB010008FB01000890
:10006000FB010008FB010008FB010008FB01000880
:1000700049040008590400086904000879040008CC
:100080008904000899040008FB010008197600089B
:1000900029760008DD030008ED030008FB010008D5
:1000A000FB010008696E0008FB010008FB01000865
:1000B000796E0008896E0008FB010008FB0100084A
:1000C000FB010008FB010008FB010008FB01000820
:1000D000FB01000875750008857500089575000816
:1000E000FB010008FB010008FB010008FB01000800
:1000F000FB010008FB010008FB010008FB010008F0
:10010000FB010008FB010008FB010008FB010008DF
:10011000B96F000845700008FB010008FB010008EA
:10012000FB010008FB010008A9040008B90400084D
:10013000DFF810D000F0CAF8004800478DA400088E
:10014000AFF30080384D0020224B19680868B0E8F2
:10015000F00F80F30988BFF36F8F4FF0000080F33A
:1001600011884EF00D0E7047000000000648006830
:10017000006880F3088862B661B6BFF34F8FBFF3A3
:100180006F8F00DF00BF00BF08ED00E0EFF30980D4
:10019000BFF36F8F0F4B1A6820E9F00F106008B59E
:1001A0004FF0500080F31188BFF34F8FBFF36F8F74
:1001B0000CF0D2F84FF0000080F31188BDE8084041
:1001C00019680868B0E8F00F80F30988BFF36F8FF3
:1001D000704700BF90020020EFF3058070470000D9
:1001E0000648804706480047FEE7FEE7FEE7FEE7D1
:1001F000FEE7FEE7FEE7FEE7FEE7FEE7676E0008C4
:1002000031010008202A04DB203A21FA02F0002103
:10021000704721FA02F3D040C2F120029140084316
:100220001946704740EA01039B0703D009E008C95B
:10023000121F08C0042AFAD203E011F8013B00F8AB
:10024000013B521EF9D27047D2B201E000F8012BF7
:10025000491EFBD270470022F6E710B513460A4646
:1002600004461946FFF7F0FF204610BD30B505469D
:100270002A460B4612F8010B13F8014B08B1A042B5
:10028000F8D01CB1002802D06D1CF1E7284630BD23
:10029000421C10F8011B0029FBD1801A704730B5B1
:1002A0000B46014600202022012409E021FA02F534
:1002B0009D4205D303FA02F5491B04FA02F52844CE
:1002C000151EA2F10102F1DC30BD0000064C074D05
:1002D00006E0E06840F0010394E807009847103416
:1002E000AC42F6D3FFF728FFA4F60008C4F60008D6
:1002F00070B58C1810F8015B15F0070301D110F8E8
:10030000013B2A1106D110F8012B03E010F8016B14
:1003100001F8016B5B1EF9D12B0705D40023521E97
:100320000DD401F8013BFAE710F8013BCB1A921CFF
:1003300003E013F8015B01F8015B521EF9D5A142FD
:10034000D8D3002070BD2DE9F04104460D46164675
:1003500004F1B00800270AE04146284607F074FA85
:100360002146284600F04AF8A84610351037B74213
:10037000F2D31022414604F1B000FFF753FFBDE86D
:10038000F08170B504460E4615463146204604F00D
:100390002FFE1022294604F1B000FFF743FF70BD85
:1003A00070B504460B46002013E000210DE0250146
:1003B00005EB80050D44555D03EB8006765C7540CA
:1003C00003EB800675544D1CE9B20429EFDB451C94
:1003D000E8B20428E9DB70BD00BFFEE710B50248B3
:1003E00000F0D4F910BD0000301E002010B5024806
:1003F00000F0CCF910BD0000301E002070B505469D
:100400000E460024324629460020FFF7C9FF01248A
:1004100000BF284606F0B0FC284606F055FB0A2C23
:1004200000D10AE0284605F0A9FE324629462046BA
:10043000FFF7B6FF601CC4B2EBE700BF32462946A7
:100440000A20FFF7ADFF70BD10B5024800F01EFD99
:1004500010BD0000DC2A002010B5024800F016FD97
:1004600010BD0000982A002010B5024800F00EFDD3
:1004700010BD0000CC29002010B5024800F006FD98
:1004800010BD00008829002010B5024800F0FEFCD5
:1004900010BD0000102A002010B5024800F0F6FC44
:1004A00010BD0000542A002010B5024800F0EEFCF8
:1004B00010BD00000029002010B5024800F0E6FC45
:1004C00010BD00004429002030B590F840500124B0
:1004D000AC40C56B6C60046863604468102C04D148
:1004E0000468A2600468E16003E00468A160046835
:1004F000E26030BD7047000010B504464FF6FF7350
:1005000022460249024803F09BF810BDDC0F002090
:10051000BC28002072B600BFFEE700000021074A99
:10052000D1610749096941F00401054A1161114689
:10053000096941F04001116170470000283C00202A
:10054000002002400021074AD1610749096941F0B2
:100550000201054A116111464861096941F04001F3
:1005600011617047283C0020002002400022054B0A
:10057000DA61054A126942F00102034B1A610180F7
:1005800070470000283C00200020024000201E4947
:10059000C96801F0100139B11C49C96941F0020173
:1005A0001A4AD16140F010001749C96801F00401EE
:1005B00039B11649C96941F00101144AD16140F0CD
:1005C00004001149C96901F0010169B10F49C96904
:1005D00041F004010D4AD16100BF0B49C96921F006
:1005E0000101094AD16100BF00BF40F201118842F8
:1005F00006D10549C96921F00101034AD16101E031
:100600000149C86000BF704700200240283C00201C
:1006100070B5044601F038F9054609E0601C38B1B0
:1006200024B101F031F9401BA04201D9032070BD73
:100630001248C06800F001000028EFD10F48C068E0
:1006400000F0200020B100BF20200C49C86000BF8E
:100650000A48C06800F0100048B90848C06900F0B6
:10066000010020B90548C06800F0040018B1FFF788
:100670008DFF0120DBE70020D9E7000000200240C9
:10068000F0B504460A46216894F82050012D01D0A7
:10069000022D74D1D1F8000240F00100C1F800022F
:1006A000107D00F01F06012000FA06F3D1F81C02AD
:1006B0009843C1F81C02D069C8B9D1F80C0298431C
:1006C000C1F80C02908880B2968940EA064601F58E
:1006D0001070576940F83760108880B2168940EA78
:1006E000064601F51070576900EBC7004660D069F7
:1006F000012819D1D1F80C021843C1F80C029088D6
:1007000080B2168840EA064601F51070576940F835
:100710003760908980B2168940EA064601F510706C
:10072000576900EBC7004660906928B9D1F8040208
:100730009843C1F8040204E0D1F804021843C1F858
:100740000402106928B9D1F814029843C1F81402C0
:1007500004E0D1F814021843C1F81402106A012809
:1007600004D1D1F81C021843C1F81C02D1F80002D0
:1007700020F00100C1F800020020F0BDFFE7606A30
:1007800040F4802060620120F7E770472DE9F05FB8
:1007900004460025206846692068D0F80490206847
:1007A00087682068D0F80CA02068D0F810B02068C6
:1007B000D0F8188006F00100002855D007F001009D
:1007C000C0B101202168886007F0020018B12046FE
:1007D00000F057FA0EE007F0040010B145F4006590
:1007E00008E007F0080010B145F4805502E020460B
:1007F00000F046FA07F48070C8B14FF480702168A9
:10080000886007F4007018B1204600F03CFA0EE052
:1008100007F4806010B145F4005508E007F400606B
:1008200010B145F4804502E0204600F02BFA07F4B1
:100830008030C8B14FF480302168886007F4003000
:1008400018B1204600F021FA0EE007F4802010B124
:1008500045F4004508E007F4002010B145F4803568
:1008600002E0204600F010FA06F0080038B10AF065
:10087000100020B145F4007510202168C86006F012
:10088000040040B10AF0080028B108202168C860BF
:10089000204600F0C1F906F0020038B12068C068B7
:1008A00000F0030010B1204600F0B7F906F0400058
:1008B00038B10BF0100020B145F48065102021689C
:1008C000086106F0200040B10BF0080028B10820B4
:1008D00021680861204600F0A1F906F0100038B147
:1008E0002068006900F0030010B1204600F097F97D
:1008F00006F4003040B109F0100028B11020216842
:100900004860204600F08CF906F4803040B109F0D0
:10091000080028B1082021684860204600F0B6F998
:1009200006F4004088B309F0040078B306F4807040
:1009300020B108F0010008B145F0010506F400708F
:1009400020B108F0020008B145F0020506F480600D
:1009500020B108F0040008B145F0040506F4006079
:10096000A0B108F0700088B108F07000402817D0DE
:1009700006DC10280BD020280CD0302819D10CE030
:10098000502810D0602814D110E01DE019E045F087
:1009900008050FE045F010050CE045F0200509E0E2
:1009A00045F0400506E045F0800503E045F480751C
:1009B00000E000BF00BF2068806920F0700021685F
:1009C00088610420216848602DB1606A2843606214
:1009D0002046FFF7DAFEBDE8F09F70B504460CB97B
:1009E000012070BD94F8200010B9204600F0B0F846
:1009F0002068006840F001002168086000F044FFB2
:100A000005460DE000F040FF401B0A2808D9606A47
:100A100040F400306062052084F820000120E0E707
:100A20002068406800F001000028EBD020680068D2
:100A300020F002002168086000F026FF05460DE066
:100A400000F022FF401B0A2808D9606A40F40030F9
:100A50006062052084F820000120C2E72068406819
:100A600000F002000028EBD1207E012806D120688A
:100A7000006840F080002168086005E02068006898
:100A800020F0800021680860607E012806D120687F
:100A9000006840F040002168086005E020680068B8
:100AA00020F0400021680860A07E012806D120685F
:100AB000006840F020002168086005E020680068B8
:100AC00020F0200021680860E07E012806D120681F
:100AD000006820F010002168086005E020680068C8
:100AE00040F0100021680860207F012806D12068AE
:100AF000006840F008002168086005E02068006890
:100B000020F0080021680860607F012806D1206875
:100B1000006840F004002168086005E02068006873
:100B200020F0040021680860D4E90201084321692B
:100B30000843616908436168491E08432168C86128
:100B400000206062012084F82000002049E70000B6
:100B500010B586B0044600200290039004900590E2
:100B60002A49206888424ED100BF2948C06940F018
:100B700000702749C8610846C06900F00070019004
:100B800000BF00BF00BF0846806940F004008861D4
:100B90000846806900F00400019000BF00BFC8143F
:100BA000029000200390049002A91A4800F0B4FCBF
:100BB0004FF480500290022003900320059002A978
:100BC000144800F0A9FC00220521132000F012FFB8
:100BD000132000F0FFFE00220521142000F00AFF80
:100BE000142000F0F7FE00220521152000F002FF7E
:100BF000152000F0EFFE00220521162000F0FAFE7D
:100C0000162000F0E7FE06B010BD000000640040B2
:100C1000001002400008014070477047704770475D
:100C2000704770B5044694F82000012822D10220B4
:100C300084F820002068006820F001002168086026
:100C400000F022FE05460DE000F01EFE401B0A28C3
:100C500008D9606A40F400306062052084F8200002
:100C6000012070BD2068406800F001000028EBD131
:100C70006062F6E7606A40F4002060620120F0E7FD
:100C8000704770477047704770477047704701461C
:100C9000002291F82100022808D00420886300BFB8
:100CA000002081F8200000BF01207047086800681C
:100CB00020F00E000B6818600868006820F0010042
:100CC0000B68186091F8403001209840CB6B586059
:100CD000012081F8210000BF002081F8200000BF22
:100CE0001046E2E770B50446002594F8210002287A
:100CF00003D00420A0630125C1E02068006820F033
:100D00000E00216808602068006820F0010021685A
:100D100008605C492068884252D95A49783920686D
:100D2000884201D1012047E0564964392068884251
:100D300001D1102040E0534950392068884201D148
:100D4000801539E04F493C392068884201D1801430
:100D500032E04C4928392068884202D14FF4803073
:100D60002AE0484914392068884202D14FF48010A3
:100D700022E044492068884201D140041CE04249F5
:100D80002068884201D1012016E03F4914312068D3
:100D9000884201D110200FE03B4928312068884269
:100DA00001D1801508E038493C312068884201D1E2
:100DB000801401E04FF480303349091F086051E08E
:100DC000304978392068884201D1012047E02D4917
:100DD00064392068884201D1102040E02949503907
:100DE0002068884201D1801539E026493C392068C5
:100DF000884201D1801432E0224928392068884293
:100E000002D14FF480302AE01E491439206888420C
:100E100002D14FF4801022E01A492068884201D1A3
:100E200040041CE018492068884201D1012016E0E6
:100E3000154914312068884201D110200FE0124971
:100E400028312068884201D1801508E00E493C31E4
:100E50002068884201D1801401E04FF480300949B4
:100E600080394860012084F8210000BF002084F808
:100E7000200000BF606B10B12046616B8847284698
:100E800070BD0000800002400804024070B50446B6
:100E9000E06B05682068066894F8401004208840DC
:100EA0002840002875D006F004000028FAD02068F9
:100EB000006800F0200028B92068006820F00400D5
:100EC00021680860D5492068884254D9D3497839C7
:100ED0002068884201D1042049E0D0496439206863
:100EE000884201D1402042E0CC49503920688842F4
:100EF00001D100153BE0C9493C392068884202D144
:100F00004FF4804033E0C54928392068884202D137
:100F10004FF480202BE0C14914392068884202D167
:100F20004FF4800023E0BD492068884201D1C0040D
:100F30001DE0BB492068884201D1042017E0B84970
:100F400014312068884201D1402010E0B449283192
:100F50002068884201D1001509E0B1493C31206880
:100F6000884202D14FF4804001E04FF48020AC4928
:100F7000091F086054E0A94978392068884201D1E6
:100F800004204AE0A54964392068884202D1402003
:100F900043E04CE0A14950392068884201D1001556
:100FA0003BE09E493C392068884202D14FF48040A2
:100FB00033E09A4928392068884202D14FF48020D2
:100FC0002BE0964914392068884202D14FF4800002
:100FD00023E092492068884201D1C0041DE0904975
:100FE0002068884201D1042017E08D49143120681F
:100FF000884201D1402010E0894928312068884288
:1010000001D1001509E086493C312068884202D1AF
:101010004FF4804001E04FF48020804980394860DF
:10102000E06A002802D02046E16A8847F4E094F89C
:101030004010022088402840002871D006F00200AD
:101040000028FAD02068006800F0200040B920682D
:10105000006820F00A0021680860012084F821005F
:101060006E492068884254D96C4978392068884292
:1010700001D1022049E0694964392068884201D1E0
:10108000202042E0654950392068884201D140154E
:101090003BE062493C392068884202D14FF400505D
:1010A00033E05E4928392068884202D14FF400308D
:1010B0002BE05A4914392068884202D14FF40010BD
:1010C00023E056492068884201D180041DE054493C
:1010D0002068884201D1022017E05149143120686C
:1010E000884201D1202010E04D49283120688842F3
:1010F00001D1401509E04A493C312068884202D1BB
:101100004FF4005001E04FF400304549091F0860DA
:1011100054E0424978392068884202D102204AE0EE
:1011200057E03E4964392068884201D1202042E0DE
:101130003A4950392068884201D140153BE037498F
:101140003C392068884202D14FF4005033E03349E3
:1011500028392068884202D14FF400302BE02F4913
:1011600014392068884202D14FF4001023E02B4943
:101170002068884201D180041DE029492068884206
:1011800001D1022017E0264914312068884201D19C
:10119000202010E0224928312068884201D14015E2
:1011A00009E01F493C312068884202D14FF40050C9
:1011B00001E04FF4003019498039486000BF002039
:1011C00084F8200000BFA06A30B32046A16A884797
:1011D00022E094F84010082088402840E0B106F052
:1011E0000800C8B12068006820F00E00216808607F
:1011F00094F8401001208840E16B48600120A06312
:1012000084F8210000BF002084F8200000BF206B7C
:1012100010B12046216B884770BD0000800002405D
:10122000080402400146002209B9012070471E4B04
:10123000086898420BD21D4B0868C01A1423B0FBF3
:10124000F3F08000086419480838C8630AE0164BB8
:101250000868C01A1423B0FBF3F080000864124839
:101260000838C863022081F821000868026843F644
:10127000F0708243D1E901031843CB6818430B692E
:1012800018434B6918438B691843CB6918430243D1
:101290000868026000208863012081F82100002096
:1012A00081F8200000BFC1E70804024008000240A6
:1012B0002DE9F04104460D4616461F464FF0000842
:1012C00000BF94F82000012802D10220BDE8F0817F
:1012D000012084F8200000BF94F8210001282CD1BF
:1012E000022084F821000020A0632068006820F01C
:1012F0000100216808603B46324629462046FFF738
:10130000E3F8E06A30B12068006840F00E00216820
:1013100008600BE02068006820F004002168086085
:101320002068006840F00A002168086020680068B2
:1013300040F001002168086006E000BF002084F84A
:10134000200000BF4FF002084046BFE770B50446DA
:1013500000F09AFA06462546681C10B10448007849
:10136000054400BF00F090FA801BA842FAD370BD7C
:10137000880200202DE9F04104460E460127002591
:1013800000BF2648007E012802D10220BDE8F0817E
:1013900001202249087600BF2068022813D14CF2B0
:1013A0005030FFF735F990BB0120FFF7B7F84CF24A
:1013B0005030FFF72DF907461948006920F0040066
:1013C0001749086123E04CF25030FFF721F9F0B9DA
:1013D0004FF0FF303060A56812E02846FFF7B2F802
:1013E0004CF25030FFF714F907460D48006920F021
:1013F00002000B4908610FB1356007E005F5006593
:10140000D4E9021001EBC020A842E6D800BF00BF1B
:1014100000200249087600BF3846B7E7283C002084
:10142000002002400348006940F080000149086143
:1014300000207047002002402DE9FE4F05468B46F4
:1014400017469846012600240020029000BF244839
:10145000007E012802D10220BDE8FE8F0120204934
:10146000087600BF4CF25030FFF7D2F8064686BB34
:10147000012D02D10120029006E0022D02D10220AE
:10148000029001E00420029000241EE02201B946EF
:10149000C24648465146FEF7B5FE80B20190022092
:1014A00000FB04B000900199FFF760F84CF2503057
:1014B000FFF7AEF806460B48006920F00100094925
:1014C000086106B104E0601CC4B202988442DDDB0E
:1014D00000BF00BF00200249087600BF3046BBE7CE
:1014E000283C00200020024000200849096901F042
:1014F000800151B10649054A5160064951601146C3
:10150000096901F0800101B101207047002002400B
:1015100023016745AB89EFCD2DE9F847024600234B
:101520009C467BE14FF0010808FA03F4D1F80080F3
:1015300008EA0400A0427DD1DFF8F4A2D1F80480CB
:10154000A8EB0A09D0453AD014DCB8F1030F50D00B
:1015500009DCB8F1000F31D0B8F1010F1CD0B8F19F
:10156000020F49D120E0B8F1110F18D0B8F1120FD5
:1015700042D11EE0B9F5881F25D006DCB9F5803FC1
:1015800020D0B9F5801F37D11AE0B9F5001F18D067
:10159000B9F5041F30D117E0D1F80CC02DE0D1F817
:1015A0000C8008F1040C28E0D1F80C8008F1080C3C
:1015B00023E0D1F80C8008F10C0C1EE000BF00BF46
:1015C00000BF00BF00BF00BFD1F80880B8F1000F16
:1015D00002D14FF0040C0BE0D1F80880B8F1010FF4
:1015E00003D14FF0080C146102E04FF0080C546175
:1015F00003E04FF0000C00E000BF00BFFF2801D85F
:10160000904601E002F104084646FF2802D84FEA5E
:10161000830803E0A3F108084FEA88084746D6F894
:1016200000804FF00F0909FA07F928EA09080CFAB7
:1016300007F900E07AE048EA0908C6F80080D1F826
:10164000048008F08058B8F1805F6FD100BFDFF8E8
:10165000E481D8F8188048F00108DFF8D891C9F87B
:101660001880C846D8F8188008F00108CDF8008026
:1016700000BF00BF4FEAB9384FEA930958F8295024
:101680004FEA83784FEA18794FF00F0808FA09F803
:1016900025EA0805DFF8A081424502D14FF0000895
:1016A00024E0DFF89881424502D14FF001081DE0A7
:1016B000DFF88C81424502D14FF0020816E0DFF8D6
:1016C0008481424502D14FF003080FE0DFF87881B2
:1016D000424502D14FF0040808E0DFF8708142452E
:1016E00002D14FF0050801E04FF006084FEA837978
:1016F0004FEA197908FA09F848EA0505DFF8508138
:101700004FEA930948F82950D1F8048008F480384A
:10171000B8F5803F0BD1DFF83C81D8F8008048EA6B
:101720000008DFF83091C9F800800AE075E0DFF8C2
:101730002481D8F8008028EA0008DFF81891C9F859
:101740000080D1F8048008F40038B8F5003F0ED1CD
:10175000DFF8008108F10408D8F8008048EA0008A2
:10176000DFF8F09009F10409C9F800800DE0DFF816
:10177000E48008F10408D8F8008028EA0008DFF8BF
:10178000D49009F10409C9F80080D1F8048008F464
:101790008018B8F5801F0ED1DFF8B88008F108086E
:1017A000D8F8008048EA0008DFF8A89009F1080995
:1017B000C9F800800DE0DFF89C8008F10808D8F82F
:1017C000008028EA0008DFF88C9009F10809C9F8C0
:1017D0000080D1F8048008F40018B8F5001F0ED17D
:1017E000DFF8708008F10C08D8F8008048EA00089B
:1017F000DFF8609009F10C09C9F800800DE0DFF80E
:10180000548008F10C08D8F8008028EA0008DFF8B6
:10181000449009F10C09C9F800805B1CD1F80080E4
:1018200028FA03F8B8F1000F7FF47CAEBDE8F88722
:10183000000011100010024000080140000C01409F
:10184000001001400014014000180140001C01403C
:101850000800014000040140024693680B400BB1B0
:10186000012000E00020704710B5C26821EA0203A1
:1018700002EA010443EA0443036110BD0AB10161B5
:1018800001E00B04036170470148006870470000E5
:101890008002002003480068034909780844014990
:1018A00008607047800200208802002010B50848B8
:1018B000006840F0100006490860032000F0D8F8E6
:1018C0000F2000F007F800F055F8002010BD0000D0
:1018D00000200240F0B587B004460026002700250E
:1018E00000BF1F48806940F400601D4988610846B8
:1018F000806900F40060009000BF00BF01A902A849
:1019000000F0C8FA00F0FEFA06461648B6FBF0F002
:10191000471E15481549086040F2E7311348C16079
:101920004760002101618160816101F075F8054621
:1019300095B90E4801F0E0F805466DB9192000F0A0
:1019400049F8102C07D200222146192000F052F845
:101950000748046000E00125284607B0F0BD0000FC
:101960000010024040420F00002C0140E02B0020FC
:101970008402002008B500BF1448806940F00100CF
:10198000124988610846806900F00100009000BF9C
:1019900000BF00BF0846C06940F08050C8610846DB
:1019A000C06900F08050009000BF00BF00220F21EE
:1019B000901E00F01FF800BF0549486820F0E06065
:1019C00040F00070486000BF08BD000000100240F9
:1019D0000000014001460846002809DB00F01F0313
:1019E00001229A4043099B0003F1E023C3F8002140
:1019F00000BF70472DE9F05F80460D461646002770
:101A000005F040FF074639462A46334601F00700F5
:101A1000C0F1070ABAF1040F02D94FF0040A01E03D
:101A2000C0F1070AD14600F1040ABAF1070F02D249
:101A30004FF0000A01E0A0F1030AD4464FF0010A7A
:101A40000AFA09FAAAF1010A0AEA020A0AFA0CFADF
:101A50004FF0010B0BFA0CFBABF1010B0BEA030B84
:101A60004AEA0B042146404605F014FFBDE8F09F0A
:101A700000BF00F00702064B19684FF6FF0319403C
:101A8000044B0B4343EA0221014B196000BF70472E
:101A90000CED00E00000FA050120014908627047E2
:101AA00000000E422DE9F04385B0064642A30FCB5D
:101AB00001AC0FC444A0006800904FF0000800255E
:101AC00000270024A146042E36D004DC012E3BD092
:101AD000022E6BD15FE0082E32D0102E66D13B482B
:101AE0004468006800F0807000B301A8C4F383412B
:101AF000475C04F4803070B134484068C0F3404023
:101B00001DF8008004F4803040B13148B0FBF8F09B
:101B100000FB07F502E02F4807FB00F52B48406863
:101B200000F48000B0F5800F01D1A94603E0680001
:101B30000321B0FBF1F93AE000F0F4F9814636E018
:101B400000F0F0F9814632E02048046A04F4407065
:101B5000B0F5807F05D104F0020010B14FF40049C8
:101B600018E004F44070B0F5007F07D11748406AD0
:101B700000F0020010B149F640490BE004F4407057
:101B8000B0F5407F06D11148006800F4003008B17C
:101B90004FF224490BE000F0B5F90C494968C1F354
:101BA0008131491C4900B0FBF1F900E000BF00BFE2
:101BB000484605B0BDE8F08302030405060708099E
:101BC0000A0B0C0D0E0F1010010200000010024055
:101BD00000127A0000093D00F8B5044600260025F1
:101BE000207800F0010000286BD000274348C0692E
:101BF00000F0805070B900BF4048C06940F080508C
:101C00003E49C8610846C06900F08050009000BF9E
:101C100000BF01273A48006800F48070B0B9384826
:101C2000006840F4807036490860FFF72DFE0646D4
:101C300006E0FFF729FE801B642801D90320F8BDC8
:101C40002F48006800F480700028F2D02B48006A0A
:101C500000F440752DB3A08800F44070A84220D055
:101C60002648006A20F440750120264908600020BB
:101C700008602248056205F0010090B1FFF704FEFC
:101C8000064608E0FFF700FE801B41F288318842DB
:101C900001D90320D3E71948006A00F002000028A8
:101CA000F0D01648006A20F4407061680843134978
:101CB0000862012F04D10846C06920F08050C86135
:101CC00000BF207800F00200022807D10B484068CE
:101CD00020F44040A168084308494860207800F09B
:101CE0001000102807D10548406820F48000616981
:101CF0000843024948600020A1E7000000100240AC
:101D0000007000404004424270B504460D460CB9D4
:101D1000012070BD5A48006800F00700A8420ED2AA
:101D20005748006820F007002843554908600846D6
:101D3000006800F00700A84201D00120E9E7207800
:101D400000F0020002281DD1207800F004000428D1
:101D500005D14C48406840F4E0604A49486020782A
:101D600000F00800082805D14648406840F460505B
:101D7000444948604348406820F0F000A1680843A7
:101D800040494860207800F0010078B3606801287D
:101D900006D13C48006800F4003090B90120B8E753
:101DA0006068022806D13748006800F0007040B92A
:101DB0000120AEE73348006800F0020008B90120B6
:101DC000A7E73048406820F00300616808432D49C8
:101DD0004860FFF759FD064609E0FFF755FD801BF7
:101DE00041F28831884202D9032092E707E0254872
:101DF000406800F00C006168B0EB810FEDD1204825
:101E0000006800F00700A8420ED91D48006820F0C5
:101E1000070028431A4908600846006800F00700D8
:101E2000A84201D0012074E7207800F004000428C3
:101E300007D11448406820F4E060E1680843114984
:101E40004860207800F00800082808D10D48406854
:101E500020F46050216940EAC1000A49486000F05E
:101E600061F808494968C1F30311074A515CC84049
:101E70000649086006480068FFF72CFD002048E787
:101E800000200240001002405BF600088C02002097
:101E9000840200200F2202600D4A526802F0030201
:101EA00042600B4A526802F0F0028260084A5268AF
:101EB00002F4E062C260064A526802F46052D2083C
:101EC0000261044A126802F007020A6070470000CB
:101ED00000100240002002400148006870470000E6
:101EE0008C02002000B5FFF7F7FF04494968C1F3F1
:101EF0000221034A515CC84000BD000000100240AE
:101F00006BF6000800B5FFF7E7FF04494968C1F325
:101F1000C221034A515CC84000BD000000100240CD
:101F20006BF60008F0B585B00FF26C0C9CE8E01081
:101F300001A8A0E8E0101CA52D6800950021002252
:101F4000002300240020194D696801F00C05F5B14B
:101F5000042D02D0082D19D101E0154819E001AD7A
:101F6000C1F38346AC5D01F4803555B10F4D6D680A
:101F7000C5F340451DF805200D4D6543B5FBF2F353
:101F800002E00C4D04FB05F3184602E000BF0848D0
:101F900000BF00BF05B0F0BD020304050607080935
:101FA0000A0B0C0D0E0F1010010200000010024071
:101FB00000127A0000093D00F8B504460CB9012072
:101FC000F8BD207800F00100002878D0F84840687B
:101FD00000F00C0004280CD0F548406800F00C001C
:101FE000082811D1F248406800F48030B0F5803FF5
:101FF0000AD1EF48006800F4003000285FD0606824
:1020000000285CD10120DBE700BF6068B0F5803FAD
:1020100006D1E748006840F48030E549086028E0D0
:10202000606858B9E248006820F48030E0490860F0
:102030000846006820F4802008601AE06068B0F567
:10204000A02F0BD1DA48006840F48020D8490860FE
:102050000846006840F4803008600AE0D448006810
:1020600020F48030D24908600846006820F48020BF
:10207000086000BF606888B1FFF706FC054606E00F
:10208000FFF702FC401B642801D9032098E7C848E9
:10209000006800F400300028F2D010E0FFF7F4FBF5
:1020A000054606E0FFF7F0FB401B642801D903203A
:1020B00086E7BF48006800F400300028F2D120789D
:1020C00000F00200022857D1B948406800F00C0027
:1020D00050B1B748406800F00C00082818D1B44847
:1020E000406800F4803098B9B148006800F0020000
:1020F00020B12069012801D0012061E7AC480068C7
:1021000020F0F800616940EAC100A949086033E0A5
:102110002069E8B10120A7490860FFF7B5FB054633
:1021200006E0FFF7B1FB401B022801D9032047E777
:102130009F48006800F002000028F2D09C48006828
:1021400020F0F800616940EAC1009949086013E095
:10215000002098490860FFF797FB054606E0FFF767
:1021600093FB401B022801D9032029E7904800680F
:1021700000F002000028F2D1207800F008000828C2
:102180002DD1A069B8B101208B490860FFF77CFB15
:10219000054606E0FFF778FB401B022801D9032023
:1021A0000EE78348406A00F002000028F2D00120C8
:1021B00004F092FB13E000207F490860FFF764FB06
:1021C000054606E0FFF760FB401B022801D903200B
:1021D000F6E67748406A00F002000028F2D1207845
:1021E00000F00400042873D100277148C06900F092
:1021F000805070B900BF6E48C06940F080506C4993
:10220000C8610846C06900F08050009000BF00BF60
:1022100001276A48006800F48070B0B96748006818
:1022200040F4807065490860FFF72EFB054606E024
:10223000FFF72AFB401B642801D90320C0E65F4852
:10224000006800F480700028F2D000BFE068012828
:1022500006D15748006A40F001005549086227E05E
:10226000E06858B95248006A20F0010050490862FD
:102270000846006A20F00400086219E0E0680528BA
:102280000BD14B48006A40F00400494908620846F7
:10229000006A40F0010008620AE04548006A20F048
:1022A0000100434908620846006A20F00400086201
:1022B00000BFE068A0B1FFF7E7FA054609E0FFF7C5
:1022C000E3FA401B41F28831884202D9032077E6C5
:1022D00022E03748006A00F002000028EFD012E048
:1022E000FFF7D2FA054608E0FFF7CEFA401B41F2AD
:1022F0008831884201D9032062E62D48006A00F047
:1023000002000028F0D1012F05D12948C06920F032
:1023100080502749C86100BFE069C8B324484068BD
:1023200000F00C00082860D0E069022848D10020A5
:1023300020490866FFF7A8FA054606E0FFF7A4FA69
:10234000401B022801D903203AE61948006800F032
:1023500000700028F2D1206AB0F5803F07D1144800
:10236000406820F40030A168084311494860D4E96E
:10237000080108430E49496821F4741108430C49C7
:10238000486001200B490866FFF77EFA054607E022
:102390003DE0FFF779FA401B022801D903200FE640
:1023A0000348006800F000700028F2D02FE0000021
:1023B000001002400000424280044242007000408F
:1023C000002014490866FFF75FFA054606E0FFF7AC
:1023D0005BFA401B022801D90320F1E50E48006892
:1023E00000F000700028F2D111E0E069012800D16E
:1023F000E6E50948466806F48031206A814204D146
:1024000006F47011606A814201D00120D8E50020F5
:10241000D6E50000000042420010024010B503461D
:1024200000220020024A02EB81021468A0B210BD13
:10243000006C004010B503460020034800EB81000B
:1024400094B2046010BD0000006C004070477047FB
:1024500010B504462068006800F00100F0B1206863
:10246000406800F00100C8B120684068C0F38000F7
:1024700048B12046FFF7EBFF6FF004002168486089
:102480000420607404E02046FFF7E0FF0120607440
:102490002068406820F001002168486010BD0000FD
:1024A00070B5044600250CB9012070BD607C20B9D0
:1024B00000202074204600F05BF802206074204663
:1024C00000F068F918B1042060740120EDE720469F
:1024D00004F021FA18B1042060740120E5E72068B7
:1024E000406820F0070021684860A06828B11F48B4
:1024F000006820F001001D4908601C48001F0068AA
:1025000020F46070A16808431849091F08606068DA
:10251000401C08B1656809E00120FFF7C3FA0546D1
:102520001DB9042060740120BFE76D1E206880681B
:1025300020F00F0040EA1540216888602068C068DC
:1025400065F30F002168C860204604F001FA18B155
:10255000042060740120A8E70021E1730121617368
:10256000A1730120607400209FE70000306C0040E0
:1025700038B504460F49206888421AD1FFF78CFA13
:1025800000BF0D48C06940F000600B49C8610846B3
:10259000C06900F00060009000BF00BF0120074943
:1025A0000860002205210320FFF724FA0320FFF72B
:1025B00011FA38BD00280040001002403C0442429D
:1025C0002DE9F04704460D46904600260027B14607
:1025D00004B115B90120BDE8F08700BF207C0128B7
:1025E00001D10220F7E70120207400BF02206074AF
:1025F000B8F1000F06D1E978E17369786173A978C1
:10260000A1730BE0E87804F07BF9E073687804F0DC
:1026100077F96073A87804F073F9A073A27B617BEB
:10262000E07B04F0E1F92073207B2870204604F061
:10263000C1F906464FF46160B6FBF0F9B9F1180F25
:102640002FD91820B9FBF0F000EB4000C000C0EB20
:102650004011C1EB0020A6EB00163146204604F0E5
:102660001CFA38B10420607400BF0020207400BF41
:102670000120B0E7204604F091F90746781C80B1AC
:10268000B7420ED20B4807443946204604F0EEF913
:1026900038B10420607400BF0020207400BF012006
:1026A00099E70120607400BF0020207400BF00BFC4
:1026B00091E70000805101002DE9F04704460D46E6
:1026C00090460026002704B115B90120BDE8F08727
:1026D00000BF207C012801D10220F7E701202074EF
:1026E00000BF02206074B8F1000F0BD128784FF4BE
:1026F000616148436978C1EB011100EB8100A97861
:10270000461812E0287804F0FBF84FF4616100FBF2
:1027100001F9687804F0F4F8C0EB001009EB8009C7
:10272000A87804F0EDF809EB00063146204604F0E5
:10273000B4F938B10420607400BF0020207400BFD9
:102740000120C3E72068406820F005002168486048
:10275000204604F023F90746781C80B1B7420ED218
:102760000B4807443946204604F080F938B104206C
:10277000607400BF0020207400BF0120A6E7012084
:10278000607400BF0020207400BF00BF9EE70000FF
:102790008051010070B5044600250CB9012070BDC0
:1027A0002068406820F0080021684860FFF76CF856
:1027B000054607E0FFF768F8401BB0F57A7F01D9BE
:1027C0000320ECE72068406800F008000028F1D002
:1027D0000020E4E710B504460CB9012010BD606A82
:1027E00038B96068B0F5827F00D105E00021E16171
:1027F00002E00021216161610021A16294F8510091
:1028000028B9002084F85000204600F043F8022048
:1028100084F851002068006820F0400021680860BA
:10282000A08800F48270218901F404410843A18941
:1028300001F400610843217C01F002010843217D7D
:1028400001F001010843218B01F400710843217F4D
:1028500001F0380108432021095D01F0800108439F
:10286000218D01F400510843216808600421A0690A
:1028700001EA1040216848602068C06920F40060C7
:102880002168C86100206065012084F851000020A3
:10289000A4E7000010B586B0044600200290039023
:1028A000049005902F492068884225D100BF2E480A
:1028B000806940F480502C4988610846806900F4A2
:1028C0008050019000BF00BF00BF0846806940F003
:1028D000040088610846806900F00400019000BF90
:1028E00000BFA0200290022003900320059002A9BF
:1028F0001E48FEF711FE33E01D49206888422FD1A3
:1029000000BF1948C06940F480401749C8610846B3
:10291000C06900F48040019000BF00BF00BF0846BE
:10292000806940F0080088610846806900F008006E
:10293000019000BF00BF4FF420400290022003909E
:102940000320059002A90B48FEF7E6FD4FF48040F6
:10295000029000200390049002A90648FEF7DCFDD7
:1029600006B010BD003001400010024000080140D8
:1029700000380040000C01407047704730B50246F7
:102980000B4600BF92F83C00012801D1022030BD67
:10299000012082F83C0000BF022082F83D00106850
:1029A00044681068816824F0700418680443106853
:1029B0004460144D1068A84213D0134D1068A8420B
:1029C0000FD01068B0F1804F0BD0104D1068A842A6
:1029D00007D00F4D1068A84203D00E4D1068A842D2
:1029E00005D121F080015868014310688160012001
:1029F00082F83D0000BF002082F83C0000BF00BF0D
:102A0000C5E70000002C01400034014000040040F4
:102A100000080040000C004010B504460CB901202D
:102A200010BD94F83D0028B9002084F83C002046F1
:102A300000F026F8022084F83D00211D206804F0F3
:102A400031FA012084F8460000BF84F83E000121DD
:102A50003F200155402001554120015500BF00BFD6
:102A6000012084F8420043200155442001554520AF
:102A7000015500BF012084F83D000020D0E7000090
:102A800038B504462068B0F1804F16D100BF184811
:102A9000C06940F001001649C8610846C06900F0ED
:102AA0000100009000BF00BF002205211C20FEF79E
:102AB000A1FF1C20FEF78EFF19E00E492068884216
:102AC00015D100BF0A48C06940F002000849C8613A
:102AD0000846C06900F00200009000BF00BF00225D
:102AE00005211D20FEF786FF1D20FEF773FF38BD70
:102AF0000010024000040040014691F83D0001280A
:102B000001D001207047022081F83D000868C068AC
:102B100040F001000B68D860164B0868984213D04B
:102B2000154B086898420FD00868B0F1804F0BD061
:102B3000124B0868984207D0114B0868984203D09E
:102B4000104B086898420CD10868806800F00702B2
:102B5000062A0CD00868006840F001000B68186075
:102B600005E00868006840F001000B68186000206C
:102B7000C8E70000002C0140003401400004004080
:102B800000080040000C00402DE9F04104460D46CD
:102B900000BF94F83C00012802D10220BDE8F0817A
:102BA000012084F83C0000BF022084F83D0020682A
:102BB000866826F0770626F47F46206886602868B7
:102BC000502833D00CDC202850D004DC00284BD017
:102BD000102851D149E0302849D040284CD139E063
:102BE00060282DD0702807D0B0F5805F03D0B0F5F5
:102BF000005F41D10DE040E0D5E902136A6820682A
:102C000004F09EF92068866846F0770620688660A2
:102C100033E0D5E902136A68206804F091F920686E
:102C2000806840F480402168886026E0EA6869682E
:102C3000206804F099F95021206804F08CF91CE018
:102C4000EA686968206804F0A2F96021206804F04D
:102C500082F912E0EA686968206804F085F9402189
:102C6000206804F078F908E000BF00BF00BF2968C1
:102C7000206804F070F900E000BF00BF012084F874
:102C80003D0000BF002084F83C0000BF00BF85E786
:102C9000704710B5044620680069C0F34000D8B101
:102CA0002068C068C0F34000B0B16FF00200216836
:102CB0000861012020772068806900F0030018B1C6
:102CC0002046FFF7E5FF05E0204600F0ADF820467E
:102CD00000F0ABF80020207720680069C0F3800086
:102CE000D8B12068C068C0F38000B0B16FF00400B4
:102CF00021680861022020772068806900F4407014
:102D000018B12046FFF7C4FF05E0204600F08CF81C
:102D1000204600F08AF80020207720680069C0F380
:102D2000C000D8B12068C068C0F3C000B0B16FF077
:102D3000080021680861042020772068C06900F03D
:102D4000030018B12046FFF7A3FF05E0204600F07E
:102D50006BF8204600F069F80020207720680069B1
:102D6000C0F30010D8B12068C068C0F30010B0B143
:102D70006FF0100021680861082020772068C06982
:102D800000F4407018B12046FFF782FF05E02046AE
:102D900000F04AF8204600F048F80020207720682C
:102DA000006900F0010058B12068C06800F001001F
:102DB00030B16FF0010021680861204600F036F85C
:102DC00020680069C0F3C01058B12068C068C0F323
:102DD000C01030B16FF08000216808612046FFF715
:102DE000CBFD20680069C0F3801058B12068C0682E
:102DF000C0F3801030B16FF04000216808612046B8
:102E000000F02EF820680069C0F3401058B1206827
:102E1000C068C0F3401030B16FF020002168086135
:102E20002046FFF7AAFD10BD7047704710B5044655
:102E300008492068884201D1FEF72CFD00BF0648F2
:102E40000068B0F1804F03D101210448FEF70CFD6A
:102E500000BF10BD002C01401C1F002000100140CD
:102E60007047704770B50446002520684069C0F37C
:102E7000C01594F83D0021280ED16DB1206840693D
:102E800020F0800021684861606B10B1606BFDF735
:102E9000FEFE204604F0C1F920684069C0F38015A9
:102EA00094F83E0022280ED16DB12068406920F0D0
:102EB000400021684861A06B10B1A06BFDF7E7FEF0
:102EC000204604F07FF9002070BD70472DE9F84FCF
:102ED0000446206805682068C668206847694FF086
:102EE0000009CA4605F00F09B9F1000F0AD105F033
:102EF000200038B106F0200020B1204604F097F9F8
:102F0000BDE8F88FB9F1000F71D007F0010018B9D2
:102F100006F4907000286AD005F0010030B106F484
:102F2000807018B1206C40F00100206405F00400AE
:102F300030B107F0010018B1206C40F002002064AD
:102F400005F0020030B107F0010018B1206C40F02C
:102F50000400206405F0080048B106F0200010B914
:102F600007F0010018B1206C40F008002064206CCC
:102F700068B305F0200028B106F0200010B120460B
:102F800004F055F920684069C0F3801A206C00F005
:102F9000080010B9BAF1000F22D0204604F012F94F
:102FA0002068406900F04000B0B12068406920F01E
:102FB000400021684861A06B50B15648A16B48633E
:102FC000A06BFDF78FFE10B1A06B416B88470CE042
:102FD0002046FFF77AFF08E02046FFF776FF04E07F
:102FE0002046FFF772FF0020206489E7FFE7206B8F
:102FF000012878D105F01000002874D006F01000E8
:10300000002870D000BF0020009020680068009069
:1030100020684068009000BF00BF2068406900F051
:103020004000C0B3A06B006840681FFA80F8B8F198
:10303000000F2FD0A08D40452CDDA4F82E80A06B72
:10304000806920281FD02068C06820F48070216823
:10305000C8602068406920F001002168486120684C
:10306000406920F0400021684861202084F83E003B
:10307000002020632068C06820F010002168C8602C
:10308000A06BFDF704FEA08DE28D801A81B2204670
:10309000FFF7E7FE34E7FFE7A08DE18D401A1FFA46
:1030A00080F8E08DE8B1B8F1000F1AD02068C06850
:1030B00020F490702168C8602068406920F0010009
:1030C00021684861202084F83E00002020632068A9
:1030D000C06820F010002168C86041462046FFF714
:1030E000C0FE0DE7FFE705F0800030B106F080007C
:1030F00018B1204604F0D8F902E705F0400030B1DD
:1031000006F0400018B1204604F077F8F8E600BF5A
:10311000F6E60000D970000810B504460CB901208D
:1031200010BDA06900B100E000BF94F83D0028B9CF
:10313000002084F83C00204600F028F8242084F881
:103140003D002068C06820F400502168C860204617
:1031500004F0E0F82068006920F4904021680861DC
:103160002068406920F02A00216848612068C06812
:1031700040F400502168C86000202064202084F8BA
:103180003D0084F83E000020CAE7000010B586B07C
:10319000044600200290039004900590FE492068A8
:1031A00088426AD100BFFD48C06940F40020FB4955
:1031B000C8610846C06900F40020019000BF00BF4C
:1031C00000BF0846806940F01000886108468069A9
:1031D00000F01000019000BF00BF0815029002200F
:1031E00003900320059002A9ED48FEF795F94FF4EE
:1031F0000060029000200390049002A9E848FEF7C6
:103200008BF9E848E8490860002048600021E6485A
:1032100081608021C1600021016141618161C161E2
:10322000FEF700F808B1FDF775F900BFDE48A063AE
:10323000446200BFDB482830DC4908601020486049
:103240000021DA4881608021C16000210161416173
:103250008161C161FDF7E6FF08B1FDF75BF900BFD1
:10326000D2486063446200BF002205213420FEF78B
:10327000C1FB3420FEF7AEFBBDE1CD49206888429A
:1032800043D100BFC548C06940F48010C349C8613C
:103290000846C06900F48010019000BF00BF00BF65
:1032A0000846806940F0100088610846806900F097
:1032B0001000019000BF00BF00BF0846806940F0C9
:1032C000200088610846806900F02000019000BF5E
:1032D00000BF88140290022003900320059002A9E9
:1032E000AF48FEF719F904200290002003900490E3
:1032F00002A9B048FEF710F9002205213520FEF79B
:1033000079FB3520FEF766FB75E1AB492068884202
:103310006AD100BFA148806940F480409F4988611C
:103320000846806900F48040019000BF00BF00BFE4
:103330000846806940F0040088610846806900F012
:103340000400019000BF00BF4815029002200390C6
:103350000320059002A99948FEF7DEF84FF480603B
:10336000029000200390049002A99448FEF7D4F83C
:10337000934894490860002048600021914881608A
:103380008021C1600021016141618161C161FDF75E
:1033900049FF08B1FDF7BEF800BF8A48A063446248
:1033A00000BF874814388849086010204860002111
:1033B000854881608021C160002101614161816196
:1033C000C161FDF72FFF08B1FDF7A4F800BF7E48EB
:1033D0006063446200BF002205212520FEF70AFB3E
:1033E0002520FEF7F7FA06E17849206888426AD17D
:1033F00000BF6A48C06940F400306849C8610846A7
:10340000C06900F40030019000BF00BF00BF084653
:10341000806940F0040088610846806900F004007B
:10342000019000BF00BF04200290022003900320FF
:10343000059002A96148FEF76FF80820029000206D
:103440000390049002A95D48FEF766F85C481430CA
:103450005F4908600020486000215D48816080214C
:10346000C1600021016141618161C161FDF7DAFE46
:1034700008B1FDF74FF800BF5548A063446200BF94
:103480004F482830534908601020486000215148B7
:1034900081608021C1600021016141618161C16160
:1034A000FDF7C0FE08B1FDF735F800BF494860637D
:1034B000446200BF002205212620FEF79BFA262049
:1034C000FEF788FA97E04449206888428BD100BF14
:1034D0003248C06940F480203049C8610846C0695C
:1034E00000F48020019000BF00BF00BF0846806943
:1034F00040F0080088610846806900F008000190EB
:1035000000BF00BF08150290022003900320059021
:1035100002A93248FEF700F84FF400600290002044
:103520000390049002A92D48FDF7F6FF244828389F
:103530002B490860002048600021294881608021D3
:10354000C1600021016141618161C161FDF76AFED5
:1035500008B1FCF7DFFF00BF2148A063446200BF51
:1035600017483C381F4908601020486000211D485A
:1035700081608021C1600021016141618161C1617F
:10358000FDF750FE08B1FCF7C5FF00BF15486063AA
:10359000446200BF002227E0004C004000100240BF
:1035A000001001403004024000290020442900207E
:1035B0000050004000140140003801400008014064
:1035C0005800024088290020CC29002000440040F7
:1035D000102A0020542A002000480040000C01401E
:1035E000982A0020DC2A002005212720FEF702FA75
:1035F0002720FEF7EFF906B010BD70B504460D4662
:10360000164694F83E00202816D105B10EB90120C7
:1036100070BD00BF94F83C00012801D10220F7E7FB
:10362000012084F83C0000BF002020633246294678
:10363000204603F0EDFEEBE70220E9E77047704714
:103640002DE9F84F04460E46174699464FF0000AFA
:1036500094F83D0020285AD106B117B90120BDE8E1
:10366000F88F00BF94F83C00012801D10220F6E752
:10367000012084F83C0000BF00202064212084F851
:103680003D00FEF701F98246A784E784A068B0F503
:10369000805F04D1206910B90025B04602E03546AC
:1036A0004FF0000800BF002084F83C0000BF1BE082
:1036B0005346002280212046CDF8009003F024FFDD
:1036C00008B10320CBE745B9B8F80000C0F3080003
:1036D0002168486008F1020803E028782168486002
:1036E0006D1CE08C401EE084E08C0028E0D1534645
:1036F000002240212046CDF8009003F005FF08B1DC
:103700000320ACE7202084F83D000020A7E702203A
:10371000A5E7704700BFFEE70FB400B58FB04F4874
:10372000007820B102F096FD00204C4908709DF809
:103730004000052851D006DC052819D2DFE800F04A
:103740000C19283D4C00062848D0072847D0A1284E
:1037500061D0BB287DD16DE041480078009041499F
:103760000B7841490A7841490978119804F062FAC6
:103770006FE0FEF789F83E490968401A42F210717D
:10378000884202D301203B49087006F001FF60E047
:10379000FEF77AF836490968401A42F210718842F9
:1037A00002D30120334908709DF8410010B904F09C
:1037B00071F94EE001F0AEFC4BE0FEF765F82C49E4
:1037C0000968401A42F21071884202D30120294947
:1037D000087008F05DFB3CE000BF00BF00BFFEF7D3
:1037E00053F823490968401A44F62061884208D3F7
:1037F00001231A4620A122A008F0B0FA01201D4999
:1038000008703C2214A96846FCF70CFD10A80FC8EC
:1038100008F0E8FD1DE0FEF737F815490968401A81
:1038200042F21071884202D301201249087002F05E
:10383000FDFA0EE0FEF728F80D490968401A42F239
:103840001071884202D301200A49087003F0F6FE85
:1038500000BF00BF0FB05DF814FB0000F5000020B2
:10386000F9000020F8000020F7000020F6000020FA
:1038700000020020FA0000204552524F5200000082
:1038800041542B444953434F4E4E3D300D0A0000E6
:1038900010B508217148FDF7DFFF7149087008462F
:1038A000007870490978884208D06D4800786D49E1
:1038B0000870FDF7E9FF6C490860CCE0FDF7E4FF14
:1038C00069490968401A1E28F7D965480078002818
:1038D00072D16648007800286FD1FDF7D5FF6449A2
:1038E00008606448007807286CD007DC07281FD2DE
:1038F000DFE800F0131F2C47656667000B286FD0C8
:1039000006DC08287DD009287CD00A2810D17AE06E
:103910000D287AD0A128F9D178E000BF00205549C0
:10392000087048708870C87001205349087000BF43
:1039300087E000BF01204F49087048700020887060
:103940000120C8704C49087000BF7AE049484078AF
:10395000042809D047484078401C4649487008462A
:103960008078401E887008E042484078042804D1DE
:103970000020404948700420887001203E490870AA
:103980005FE03C484078032809D03A484078401C22
:103990003849487008468078401E887008E03548ED
:1039A0004078032804D100203249487003208870F1
:1039B00001203149087044E049E046E002E000BFE0
:1039C00000BF00BF2B48407801280DD0294840781F
:1039D000401C2849487008468078401E88700CE0DA
:1039E00012E00EE00EE010E022484078012804D1F9
:1039F0000020204948700120887001201E4908706D
:103A00001FE000BF00BF00BF00BF00BF19484078E3
:103A10000F2809D017484078401C164948700846BE
:103A20008078401E887008E0124840780F2804D142
:103A30000020104948700F20887001200E4908703E
:103A400000BF00BF012009490870012010BD0020FF
:103A500006490870FAE70020F8E70000000C014072
:103A6000040200200502002008020020DC010020E2
:103A700000020020F4020020F500002010B5102103
:103A80006E48FDF7E9FE6E490870084600786D49FA
:103A90000978884208D06A4800786A490870FDF7BA
:103AA000F3FE69490860C7E0FDF7EEFE6649096864
:103AB000401A1E28F7D962480078002870D1634860
:103AC000007800286DD1FDF7DFFE6149086061488C
:103AD0000078072869D007DC07281FD2DFE800F04C
:103AE000131F2C46626364000B287FD006DC082875
:103AF00079D0092878D00A2810D176E00D2876D020
:103B0000A128F9D174E000BF002052490870487024
:103B10008870C87001205049087000BF82E000BF63
:103B200001204C4908700020487001208870C8703E
:103B30004949087000BF75E046488078042809D0DC
:103B400044484078401E4349487008468078401CED
:103B5000887007E03F488078042803D13D494870C9
:103B60000020887001203C4908705BE0394880786B
:103B7000032809D037484078401E36494870084627
:103B80008078401C887007E032488078032803D191
:103B9000304948700020887001202F49087041E0AA
:103BA00046E043E000BF00BF00BF2A4880780128FC
:103BB00009D028484078401E264948700846807839
:103BC000401C887007E023488078012803D12149F0
:103BD00048700020887001201F49087022E005E02D
:103BE00001E001E003E000BF00BF00BF00BF00BF75
:103BF000184880780F2809D016484078401E15498B
:103C0000487008468078401C887007E0114880782A
:103C10000F2803D10F4948700020887001200E49F9
:103C2000087000BF00BF012008490870012010BDC6
:103C3000002006490870FAE70020F8E7000C014070
:103C40000C0200200D02002010020020DD010020E7
:103C500000020020F4020020F500002010B5202111
:103C6000FA48FDF7F9FDFA49087008460078F94965
:103C70000978884209D0F6480078F6490870FDF7BF
:103C800003FEF549086001F0ACB8FDF7FDFDF2490F
:103C90000968401A1E28F6D9ED480078002841F03E
:103CA0009C80EE480078002841F09580FDF7ECFDFF
:103CB000EB490860EB48007807287DD00BDC07282B
:103CC00081F08580DFE810F0170025004900D90059
:103CD0004D014E014F010B286FD007DC08286DD035
:103CE00009286CD00A2841F0728043E10D2867D082
:103CF000A128F8D141E100BF0120DA4908704870DD
:103D0000002088700120C870D749087000BF01F0FA
:103D10005EB8D448407801280FD107F049FA00BFB7
:103D20000220D049087004204870002088700220CA
:103D3000C8700120CC4908700EE007F039FA00BFC6
:103D40000320C84908704870002088700220C8709D
:103D50000120C549087000BFD9E7C2484078002853
:103D600078D1C04948618860C86048628861C8618C
:103D700048638862C86248648863C86308610862EF
:103D800008630864B94803F031FF0A20FDF7DEFA42
:103D9000B74803F02BFF0A20FDF7D8FAB54803F027
:103DA00025FF0A20FDF7D2FAB34803F01FFF0A20CF
:103DB000FDF7CCFAB14804E0D6E0DCE0D8E0D8E08A
:103DC000DAE003F013FF0A20FDF7C0FAAC4803F075
:103DD0000DFF0A20FDF7BAFAAA4803F007FF0A20F0
:103DE000FDF7B4FAA84803F001FF0A20FDF7AEFA88
:103DF000A64803F0FBFE0A20FDF7A8FAA44803F04A
:103E0000F5FE0A20FDF7A2FAA24803F0EFFE0A2011
:103E1000FDF79CFAA04803F0E9FE0A20FDF796FAA8
:103E200000209E4908709E4908709E4908709E496E
:103E300008704FF480308B49486000BF0120087043
:103E40004870002088700120C8708749087000BF42
:103E50005DE7FFE783488078824981F8480000BF2A
:103E6000A12008700F204870002088700320C870BF
:103E700001207D49087000BF49E77A48407803284F
:103E800018D1784AD168032390681A4607F066FF74
:103E90006420FDF75BFA00BF04207249087001201E
:103EA0004870002088700320C87001206E49087097
:103EB00000BF2CE76B484078022818D1694AD169C5
:103EC000032390691A4607F049FF6420FDF73EFA84
:103ED00000BF0520634908700120487000208870E9
:103EE0000320C87001206049087000BF0FE75D48DB
:103EF0004078012818D15B4AD16A0323906A1A4698
:103F000007F02CFF6420FDF721FA00BF0620554979
:103F1000087001204870002088700320C8700120BC
:103F20005149087000BFF2E64E484078C0B94D4A8A
:103F3000D16B0323906B1A4607F010FF6420FDF746
:103F400005FA00BF0720474908700120487000208B
:103F500088700320C87001204349087000BFD6E66E
:103F600000BF00BF00BF00BF04203E49C870CEE6BE
:103F700000BF00BF00BF00BF00BF3A4890F8480034
:103F8000002860D13748807850B948A0354988600A
:103F90004CA0C86052A008610121384803F024FCFD
:103FA0003048807801280AD153A02E49886058A053
:103FB000C8605EA008610221304803F015FC294862
:103FC000807802280AD15FA02649886063A0C86073
:103FD00069A008610321294803F006FC2148807884
:103FE00003280AD16AA01F4988606FA0C86075A025
:103FF00008610421214803F0F7FB1A48807804285F
:104000000AD176A0174988607AA0C86080A00861AC
:1040100005211A4803F0E8FB1248807805280AD1E8
:1040200081A01049886086A0C8608CA00861062124
:10403000124803F0D9FB0B488078062804D18DA0E4
:104040000849886022E1B3E128E10000000C01404A
:10405000140200201502002018020020DE010020BA
:1040600000020020F4020020F500002000000708F4
:104070000010070800200708003007080060070844
:104080000068070800770708007807080038070865
:10409000004007080048070800500708F600002005
:1040A000F7000020F8000020F900002041542B43C5
:1040B0004F4E4E3D31303130303030303030303195
:1040C0000D0A00002B434F4E4E45435445443A30B1
:1040D0002C31303130303030303030303100000071
:1040E0002B444953434F4E4E3A302C31303130300F
:1040F000303030303030310041542B434F4E4E3D44
:104100003130313030303030303030320D0A000054
:104110002B434F4E4E45435445443A302C313031B9
:104120003030303030303030320000002B444953D2
:10413000434F4E4E3A302C31303130303030303009
:104140003030320041542B434F4E4E3D31303130F0
:1041500030303030303030330D0A00002B434F4EBA
:104160004E45435445443A302C31303130303030B4
:1041700030303030330000002B444953434F4E4E13
:104180003A302C3130313030303030303030330054
:1041900041542B434F4E4E3D313031303030303072
:1041A000303030340D0A00002B434F4E4E454354FF
:1041B00045443A302C3130313030303030303030CE
:1041C000340000002B444953434F4E4E3A302C31BB
:1041D00030313030303030303030340041542B43C7
:1041E0004F4E4E3D31303130303030303030303560
:1041F0000D0A00002B434F4E4E45435445443A3080
:104200002C3130313030303030303030350000003B
:104210002B444953434F4E4E3A302C3130313030DD
:10422000303030303030350041542B434F4E4E3D0E
:104230003130313030303030303030360D0A00001F
:104240002B434F4E4E45435445443A302C31303188
:104250003030303030303030360000002B4449539D
:10426000434F4E4E3A302C313031303030303030D8
:104270003030360041542B434F4E4E3D31303130BB
:1042800030303030303030370D0A00008BA0C8603D
:1042900091A008610721964803F0A6FA9548807816
:1042A00007280AD194A09349886099A0C8609FA06C
:1042B000086108218E4803F097FA8E488078082814
:1042C0000AD1A0A08B498860A4A0C860AAA00861F8
:1042D0000921874803F088FA8648807809280AD19E
:1042E000ABA084498860B0A0C860B6A008610A216C
:1042F0007F4803F079FA7F4880780A280AD1B7A06E
:104300007C498860BBA0C860C1A008610B217848C7
:1043100003F06AFA774880780B280AD1C2A0754961
:104320008860C7A0C860CDA008610C21704803F068
:104330005BFA704880780C280AD1CEA06D4988605D
:10434000D2A0C860D8A008610D21694803F04CFADA
:10435000684880780D280AD1D9A066498860DEA017
:10436000C860E4A008610E21614803F03DFA61488D
:1043700080780E280AD1E5A05E498860E9A0C8606F
:10438000EFA008610F215A4803F02EFA59488078AF
:104390000F280AD1F0A057498860F5A0C860FBA09B
:1043A00008611021524803F01FFA0120FD490870EE
:1043B000504890F8480001287ED14E48807868B96E
:1043C000AFF218304B498861AFF20830C861AFF2E4
:1043D000F02008620121F44803F006FA454880788D
:1043E00001280DD1AFF2F02042498861AFF2E02000
:1043F000C861AFF2C82008620221EB4803F0F4F96B
:104400003C48807802280DD1AFF2C8203949886134
:10441000AFF2B820C861AFF2A02008620321E248E1
:1044200003F0E2F93348807803280DD1AFF2A020E1
:1044300030498861AFF29020C861AFF278200862FD
:104440000421D94803F0D0F92A48807804280DD1F6
:10445000AFF2782027498861AFF26820C861AFF2D7
:10446000502008620521D04803F0BEF92148807829
:1044700005280DD1AFF250201E498861AFF24020CF
:10448000C861AFF2282008620621C74803F0ACF9E2
:104490001848807806280BD1AFF22820154988618A
:1044A00006A0C8610CA008620721BF4803F09CF970
:1044B00010488078072879E11AE200002B434F4E1C
:1044C0004E45435445443A302C3130313030303051
:1044D00030303030370000002B444953434F4E4EAC
:1044E0003A302C31303130303030303030303700ED
:1044F00000600708F402002041542B434F4E4E3D0C
:104500003130313030303030303030380D0A00004A
:104510002B434F4E4E45435445443A302C313031B5
:104520003030303030303030380000002B444953C8
:10453000434F4E4E3A302C31303130303030303005
:104540003030380041542B434F4E4E3D31303130E6
:1045500030303030303030390D0A00002B434F4EB0
:104560004E45435445443A302C31303130303030B0
:1045700030303030390000002B444953434F4E4E09
:104580003A302C313031303030303030303039004A
:1045900041542B434F4E4E3D31303130303030306E
:1045A000303030410D0A00002B434F4E4E454354EE
:1045B00045443A302C3130313030303030303030CA
:1045C000410000002B444953434F4E4E3A302C31AA
:1045D00030313030303030303030410041542B43B6
:1045E0004F4E4E3D3130313030303030303030424F
:1045F0000D0A00002B434F4E4E45435445443A307C
:104600002C3130313030303030303030420000002A
:104610002B444953434F4E4E3A302C3130313030D9
:10462000303030303030420041542B434F4E4E3DFD
:104630003130313030303030303030430D0A00000E
:104640002B434F4E4E45435445443A302C31303184
:104650003030303030303030430000002B4449538C
:10466000434F4E4E3A302C313031303030303030D4
:104670003030430041542B434F4E4E3D31303130AA
:1046800030303030303030440D0A00002B434F4E74
:104690004E45435445443A302C313031303030307F
:1046A00030303030440000002B444953434F4E4ECD
:1046B0003A302C313031303030303030303044000E
:1046C00041542B434F4E4E3D31303130303030303D
:1046D000303030450D0A00002B434F4E4E454354B9
:1046E00045443A302C313031303030303030303099
:1046F000450000002B444953434F4E4E3A302C3175
:1047000030313030303030303030450041542B4380
:104710004F4E4E3D31303130303030303030304619
:104720000D0A00002B434F4E4E45435445443A304A
:104730002C313031303030303030303046000000F5
:104740002B444953434F4E4E3A302C3130313030A8
:10475000303030303030460041542B434F4E4E3DC8
:104760003130313030303030303031300D0A0000EF
:104770002B434F4E4E45435445443A302C31303153
:104780003030303030303031300000002B4449536D
:10479000434F4E4E3A302C313031303030303030A3
:1047A00030313000F6000020006807080DD1AFF26C
:1047B000B820FE498861AFF2A820C861AFF294200A
:1047C00008620821FA4803F00FF8F84880780828B2
:1047D0000DD1AFF29020F5498861AFF28020C86119
:1047E000AFF26C2008620921F14802F0FDFFEF48AA
:1047F000807809280DD1AFF26820EC498861AFF2CA
:104800005820C861AFF2442008620A21E84802F04B
:10481000EBFFE64880780A280DD1AFF24020E3494B
:104820008861AFF23020C861AFF21C2008620B2112
:10483000DF4802F0D9FFDD4880780B280DD1AFF2B8
:104840001820DA498861AFF20820C861AFF2F4108D
:1048500008620C21D64802F0C7FFD44880780C28A3
:104860000DD1AFF2F010D1498861AFF2E010C8610C
:10487000AFF2CC1008620D21CD4802F0B5FFCB4855
:1048800080780D280DD1AFF2C810C8498861AFF209
:10489000B810C861AFF2A41008620E21C44802F03B
:1048A000A3FFC24880780E280DD1AFF2A010BF49F7
:1048B0008861AFF29010C861AFF27C1008620F21DE
:1048C000BB4802F091FFB94880780F280DD1AFF2B4
:1048D0007810B6498861AFF26810C861AFF2541021
:1048E00008621021B24802F07FFF0120B149087030
:1048F000AE4890F8480002287ED1AC48807868B96C
:10490000AFF65800A9498862AFF64800C862AFF612
:10491000300008630121A84802F066FFA3488078B0
:1049200001280DD1AFF63000A0498862AFF6200013
:10493000C862AFF60800086302219F4802F054FFE6
:104940009A48807802280DD1AFF60800974988620E
:10495000AFF2F870C862AFF2E070086303219648C6
:1049600002F042FF9148807803280DD1AFF2E07049
:104970008E498862AFF2D070C862AFF2B870086337
:1049800004218D4802F030FF8848807804280DD13A
:10499000AFF2B87085498862AFF2A870C862AFF212
:1049A000907008630521844802F01EFF7F488078DC
:1049B00005280DD1AFF290707C498862AFF280700B
:1049C000C862AFF26870086306217B4802F00CFFF2
:1049D0007648807806280DD1AFF2687073498862F6
:1049E000AFF22850C862AFF2105008630721724836
:1049F00002F0FAFE6D4800E0A3E0807807280DD1B0
:104A0000AFF20C5069498862AFF2FC40C862AFF265
:104A1000E44008630821684802F0E6FE63488078B5
:104A200008280DD1AFF2E44060498862AFF2D4406B
:104A3000C862AFF2BC40086309215F4802F0D4FEAF
:104A40005A48807809280DD1AFF2BC405749886296
:104A5000AFF2AC40C862AFF2944008630A215648F6
:104A600002F0C2FE514880780A280DD1AFF294407E
:104A70004E498862AFF28440C862AFF26C4008636E
:104A80000B214D4802F0B0FE484880780B280DD12C
:104A9000AFF26C4045498862AFF25C40C862AFF249
:104AA000444008630C21444802F09EFE3F48807851
:104AB0000C280DD1AFF244403C498862AFF234403B
:104AC000C862AFF21C4008630D213B4802F08CFE27
:104AD000364880780D280DD1AFF21C4033498862EA
:104AE000AFF20C40C862AFF2F43008630E213248D6
:104AF00002F07AFE2D4880780E280DD1AFF2F43006
:104B00002A498862AFF2E430C862AFF2CC30086361
:104B10000F21294802F068FE244880780F280DD123
:104B2000AFF2CC3021498862AFF2BC30C862AFF23C
:104B3000A43008631021204802F056FE01201F49CE
:104B400008701A4890F8480003287DD117488078EB
:104B500068B9AFF6A82015498863AFF69820C863F6
:104B6000AFF6842008640121154802F03DFE0F488D
:104B7000807801280DD1AFF680200C498863AFF60C
:104B80007020C863AFF65C20086402210C4802F074
:104B90002BFE0648807802281BD1AFF65820034927
:104BA0008863AFF64820C8630CE00000F4020020E0
:104BB00000680708F700002000770708F8000020C9
:104BC00000780708AFF6502008640321864802F0F9
:104BD0000BFE8648807803280DD1AFF64C20834920
:104BE0008863AFF63C20C863AFF628200864042130
:104BF0007D4802F0F9FD7D48807804280DD1AFF69C
:104C000024207A498863AFF61420C863AFF60020E9
:104C100008640521744802F0E7FD7448807805288F
:104C20000DD1AFF6FC1071498863AFF6EC10C86384
:104C3000AFF6D810086406216B4802F0D5FD6B482A
:104C4000807806280FD100E0B2E0AFF6D8106749AF
:104C50008863AFF29870C863AFF28470086407216C
:104C6000614802F0C1FD6148807807280DD1AFF29C
:104C700078705E498863AFF26870C863AFF25470B1
:104C800008640821584802F0AFFD58488078082889
:104C90000DD1AFF2507055498863AFF24070C863D0
:104CA000AFF22C70086409214F4802F09DFD4F4877
:104CB000807809280DD1AFF228704C498863AFF293
:104CC0001870C863AFF2047008640A21464802F005
:104CD0008BFD464880780A280DD1AFF20070434919
:104CE0008863AFF2F060C863AFF2DC6008640B2148
:104CF0003D4802F079FD3D4880780B280DD1AFF298
:104D0000D8603A498863AFF2C860C863AFF2B46054
:104D100008640C21344802F067FD344880780C2880
:104D20000DD1AFF2B06031498863AFF2A060C863C3
:104D3000AFF28C6008640D212B4802F055FD2B4822
:104D400080780D280DD1AFF2886028498863AFF2D2
:104D50007860C863AFF2646008640E21224802F0F4
:104D600043FD224880780E280DD1AFF260601F49C4
:104D70008863AFF25060C863AFF23C6008640F21F3
:104D8000194802F031FD194880780F280DD1AFF293
:104D9000386016498863AFF22860C863AFF21460C8
:104DA00008641021104802F01FFD0120104908700E
:104DB00000BF02200D490870042048700020887050
:104DC0000220C87001200B49087000BF00BF00BF5F
:104DD000012009490870012010BD00200649087013
:104DE000FAE70020F8E7000000780708F402002046
:104DF000F9000020F5000020DE01002010B5402160
:104E00006548FCF729FD6549087008460078644943
:104E10000978884208D06148007861490870FCF739
:104E200033FD60490860B4E0FCF72EFD5D49096878
:104E3000401A1E28F7D959480078002873D1FCF78A
:104E400023FD594908605948007800286CD158481A
:104E50000078072839D007DC072822D2DFE800F0E5
:104E600013142223323334000B2861D006DC0828C7
:104E70005BD009285AD00A2813D158E00D2858D001
:104E8000A1287CD156E000BF06F092F900BF0020B7
:104E90004749087048708870C870012045490870FB
:104EA00000BF6CE000BF06F083F900BF012040495D
:104EB00008704870002088700120C8703D49087053
:104EC00000BF5CE000BF00BF00BF01231A463AA14B
:104ED0003BA006F043FF4FF49670FCF737FA3C48CE
:104EE00006F060F93B4908803B4806F05BF93B4916
:104EF00008803B4806F056F93A4908803A4806F0DF
:104F000051F93A49088006F053F900BF03202849B7
:104F100008704870002088700220C8700120254960
:104F2000087000BF2BE030E02DE000BF00BF00BFE5
:104F300000BF24E0264806F035F9264908802648B7
:104F400006F030F925490880254806F02BF9254957
:104F50000880254806F026F92449088006F028F93B
:104F600000BF02201249087003204870002088709A
:104F70000220C87001200F49087000BF00BF00BFA9
:104F800001200A490870012010BD0020074908705F
:104F9000FAE70020F8E70000000C01401C020020A6
:104FA0001D0200202002002000020020DF0100205E
:104FB000F4020020F50000204552524F520000003C
:104FC00041542B444953434F4E4E3D300D0A00008F
:104FD00000000708F601002000100708F801002073
:104FE00000200708FA01002000300708FC0100201B
:104FF00078B502460C46002020E0002505EB800530
:10500000655D002606EB80069555012505EB8005BC
:10501000655D012606EB80069555022505EB8005AA
:10502000655D022606EB80069555032505EB800598
:10503000655D032606EB80069555401C0428DCD3ED
:1050400004205FE0451EA900555C8DF800504D1C02
:10505000555D8DF801508D1C555D8DF80250CD1CAD
:10506000555D8DF8035000F003056DBB9DF80050B1
:105070009DF801608DF800609DF802608DF8016078
:105080009DF803608DF802608DF803509DF8005084
:105090001E4E755D8DF800509DF80150755D8DF8C0
:1050A00001509DF80250755D8DF802509DF8035037
:1050B000755D8DF803509DF80050154E06EB900677
:1050C000367875408DF800508300051FA900555CA7
:1050D0009DF800607540D5544D1C555D9DF80160EC
:1050E00075405E1C95558D1C555D9DF802607540A0
:1050F0009E1C9555CD1C555D9DF803607540DE1CCA
:105100009555401C2C289DD378BD000050F4000814
:1051100050F6000808B50120102350A2022100908B
:10512000142001F072FB01200E23102202210090B6
:10513000372001F057FA01200E231122022100909E
:105140004B2001F04FFA0120102345A211210090BD
:10515000142001F05AFB01200E231022112100908F
:10516000372001F03FFA01200E2311221146009052
:105170004B2001F037FA012010233AA220210090A1
:10518000142001F042FB01200E2310222021009068
:10519000372001F027FA01200E2311222021009050
:1051A0004B2001F01FFA012010232FA22F21009085
:1051B000142001F02AFB01200E2310222F21009041
:1051C000372001F00FFA01200E2311222F21009029
:1051D0004B2001F007FA2548407804280BD12348DA
:1051E000807840B90020102321A202210090642081
:1051F00001F00BFB31E01D48407803280CD11B481F
:105200008078012808D10020102319A211210090D4
:10521000642001F0FAFA20E01448407802280CD10A
:1052200012488078022808D10020102310A22021E3
:105230000090642001F0E9FA0FE00C484078012862
:105240000BD10A488078032807D10020102308A238
:105250002F210090642001F0D8FA08BD4C203100C5
:105260004C2032004C2033004C203400F40200204B
:105270003C2D2D0010B50C480078401C0A490870E0
:105280000AA002F0EFFA00224FF400410A48FCF7AE
:10529000F5FA4FF47A60FCF759F8012007490870D5
:1052A0000749087010BD00002402002042742072DB
:1052B000657365740D0A0000000801402802002093
:1052C0002C02002010B5494849490861FF200876A2
:1052D0004848017848A002F0C5FA01F059FC0123C2
:1052E0001A464BA14CA006F039FD10B14EA002F0B9
:1052F000B9FA51480078052870D2DFE800F00304BD
:105300001F3A55006AE001231A464CA14EA006F050
:1053100025FD78B101231A464EA14FA006F01EFDCF
:1053200058B151A002F09EFA43480078401C42490F
:10533000087002E0FFF79EFF50E000BF01231A460D
:105340004EA151A006F00AFD78B101231A4641A1F1
:1053500050A006F003FD58B152A002F083FA36487F
:105360000078401C3449087002E0FFF783FF35E005
:1053700000BF01231A4650A152A006F0EFFC78B1FD
:1053800001231A4633A152A006F0E8FC58B154A0FC
:1053900002F068FA28480078401C2749087002E0AB
:1053A000FFF768FF1AE000BF01231A4651A154A07D
:1053B00006F0D4FC78B101231A4626A154A006F0C9
:1053C000CDFC58B156A002F04DFA1B480078401CA5
:1053D0001949087002E0FFF74DFF00BF00BF002031
:1053E0005549087001205549087010BD3175746425
:1053F000C007002024020020092323233031094262
:10540000545F696E697425642E2E2E0D0A0000000B
:105410004552524F5200000041542B444953434FD0
:105420004E4E3D300D0A000023D2D1CEDEC9E8B188
:10543000B8C1ACBDD30A0000280200202B55554945
:1054400044533A464646300041542B55554944533F
:105450003F0D0A004F4B000041542B555549445312
:105460003D303030320D0A00233031C9E8D6C3D682
:10547000F7B7FECEF1B3C9B9A60A00002B555549BE
:10548000444E3A464646310041542B555549444E08
:105490003F0D0A0041542B555549444E3D46463078
:1054A000340D0A00233032C9E8D6C3B6C1B7FECEE8
:1054B000F1B3C9B9A60A00002B55554944573A46DD
:1054C0004646320041542B55554944573F0D0A007A
:1054D00041542B55554944573D464646350D0A0023
:1054E000233033C9E8D6C3D0B4B7FECEF1B3C9B9BF
:1054F000A60A00002B5458504F5745523A3000002E
:1055000041542B5458504F5745523F0D0A0000004C
:1055100041542B5458504F5745523D31300D0A00DD
:10552000233034C9E8D6C3B7A2C9E4B9A6C2CAB306
:10553000C9B9A60A00000000F4020020F50000200E
:1055400010B501200C4908700C480078401C0B492C
:1055500008700BA002F086F9002202210D48FCF72A
:105560008DF941F28830FBF7F1FE01220221094852
:10557000FCF784F910BD00007C02002079020020B5
:105580003447204D6F64756C655F52657365740AAE
:10559000000000000008014008B53248017832A040
:1055A00002F060F936A13948FAF760FE002856D0BB
:1055B00037A002F057F90F213448FAF74CFE642067
:1055C000FBF7C4FE01231A4634A135A006F08CFB7C
:1055D00028B901203449087034A002F043F9324858
:1055E000007818B135A002F03DF93AE001231A46DF
:1055F00037A13BA006F078FB58B13CA002F032F98D
:1056000000200C2340A2322100902A2001F0FDF856
:1056100027E0C820FBF79AFE01231A463DA130A0DF
:1056200006F062FB58B13FA002F01CF900200C23E9
:1056300041A22D210090232001F0E7F811E0012381
:105640001A4640A141A006F04FFB01231A463DA196
:1056500041A006F049FB43A002F004F901E0FFF786
:105660006FFF08BD7902002009232323303209345B
:10567000475F696E697425642E2E2E0D0A000000A6
:105680002B4D41545245414459000000283400201C
:10569000233447C4A3BFE9C9CFB5E7004F4B00008F
:1056A00041540D0A000000007B0200203447C4A3CF
:1056B000D7E9D2ECB3A3A3A10D0A0000233447C459
:1056C000A3BFE9B3F5CABCBBAF4661696C0000007B
:1056D0002B434D45204552524F523A203130000065
:1056E00041542B4350494E3F0D0A00000945525288
:1056F0004F52212D2D3ECEB4BCECB2E2B5BD534984
:105700004DBFA80D0A000000204E4F5F53494D20A9
:10571000000000002B434D45204552524F523A2085
:1057200031330000094552524F52212D2D3E53492D
:105730004DCAA7B0DC0D0A002053494D5F46616990
:105740006C2000004552524F5200000041542B4340
:1057500053510D0A0000000041542B434552454768
:105760003F0D0A00696E69745F73756363657373D7
:105770000D0A000000B58BB019481A4908600420D2
:105780004860002117488160C1604FF4A021016189
:105790004FF4801141610021017641768176C17616
:1057A00001774177FBF719F908B1FAF7B3FE00204A
:1057B000069007900120089000200190029003902D
:1057C00004900590012009900E200A9001A9054837
:1057D000FAF756FF0348FBF724FA0BB000BD0000B0
:1057E00000640040301E002008B500BF2D4840690D
:1057F00040F001002B4948610846406900F0010073
:10580000009000BF00BF00BF0846406940F00200A2
:1058100048610846406900F00200009000BF00BFE8
:10582000002205210C20FCF7E5F80C20FCF7D2F84B
:10583000002205210D20FCF7DDF80D20FCF7CAF849
:10584000002205210E20FCF7D5F80E20FCF7C2F847
:10585000002205210F20FCF7CDF80F20FCF7BAF845
:10586000002205211020FCF7C5F81020FCF7B2F843
:10587000002205211120FCF7BDF81120FCF7AAF841
:10588000002205213A20FCF7B5F83A20FCF7A2F8EF
:10589000002205213B20FCF7ADF83B20FCF79AF8ED
:1058A00008BD00000010024000B59DB01C22184940
:1058B00016A8FAF7B7FC002116A805F0B2F81549AA
:1058C00008601C2212491C310FA8FAF7ABFC00211A
:1058D0000FA805F0A6F8104908601C220C493831C1
:1058E00008A8FAF79FFC002108A805F09AF80B49D0
:1058F00008601C220649543101A8FAF793FC0021E4
:1059000001A805F08EF8064908601DB000BD000032
:10591000E0F300086002002064020020680200201A
:105920006C02002000B585B0002001900290039029
:10593000049000BF3D48806940F010003B498861F9
:105940000846806900F01000009000BF00BF00BF53
:105950000846806940F0200088610846806900F0B0
:105960002000009000BF00BF00BF0846806940F0E3
:10597000040088610846806900F00400009000BFC0
:1059800000BF00BF0846806940F0080088610846F3
:10599000806900F00800009000BF00BF002240F2C4
:1059A00011212348FBF76AFF012248F21201214826
:1059B000FBF764FF002240211E48FBF75FFF012236
:1059C00080211B48FBF75AFF40F2912001900120F3
:1059D0000290002003900220049001A91448FBF7D4
:1059E0009BFD48F2420001900120029000200390AC
:1059F0000220049001A90F48FBF78EFD10200190B2
:105A000001200290002003900320049001A909487E
:105A1000FBF782FD78200190002002900120039086
:105A200001A90548FBF778FD05B000BD0010024054
:105A30000010014000080140000C01401FB500208B
:105A40000290019000BF5648C06940F00060544980
:105A5000C8610846C06900F00060009000BF00BF48
:105A600000BF0846C06940F08050C8610846C06960
:105A700000F08050009000BF00BF4A484A490860CB
:105A80004FF0FF304860002147488160FCF708FD77
:105A900008B1FAF73FFD01214348FCF7BFFC45F28E
:105AA000510188424CD013208DF8080000208DF859
:105AB00009008DF80A00012202A93B48FCF7FCFD11
:105AC00008B1FAF727FD04208DF8040001208DF8B5
:105AD000050018208DF8060023208DF8070001220C
:105AE00001A93148FCF76CFD08B1FAF713FD2E4807
:105AF0000068006840F001002B49096808600198BF
:105B0000039045F2510201212748FCF793FC9DF8D0
:105B10000F2002212448FCF78DFC9DF80D20032165
:105B20002148FCF787FC9DF80E2004211E48FCF755
:105B300081FC9DF80C2005211B48FCF77BFC2DE027
:105B400002211948FCF76AFCC0B28DF80F0003214E
:105B50001548FCF763FCC0B28DF80D000421124813
:105B6000FCF75CFCC0B28DF80E0005210E48FCF776
:105B700055FCC0B28DF80C0003980190002201A9D9
:105B80000948FCF71DFD08B1FAF7C4FC0648006897
:105B9000006840F001000449096808601FBD00006A
:105BA0000010024000280040581E002010B50F4889
:105BB0000F4908604FF4827048604FF400410C4870
:105BC00081600021C160016141614FF40071816118
:105BD0000821C16100210162416281620A21C16222
:105BE000FCF7F8FD08B1FAF795FC10BD0030014054
:105BF0006C1E002010B50E480E4908604FF48270EC
:105C0000486000210B488160C160016141614FF42F
:105C1000007181610021C1610162416281620A21DA
:105C2000C162FCF7D7FD08B1FAF774FC10BD0000A3
:105C300000380040C41E002000B587B0002003904B
:105C4000049005900690019002904FF08040144916
:105C500008600920486000211148816041F63F71C9
:105C6000C160002101618161FCF7D6FE08B1FAF73D
:105C700051FC4FF48050039003A90948FCF784FFBE
:105C800008B1FAF747FC00200190029001A90448EE
:105C9000FCF774FE08B1FAF73DFC07B000BD000048
:105CA0001C1F002000B587B00020039004900590D1
:105CB00006900190029015481549086041F287301E
:105CC000486000211248816041F63F71C1600021A7
:105CD00001618161FCF7A0FE08B1FAF71BFC4FF4EB
:105CE0008050039003A90A48FCF74EFF08B1FAF769
:105CF00011FC00200190029001A90548FCF73EFE2E
:105D000008B1FAF707FC07B000BD0000000400402E
:105D1000641F002010B50B480B4908604FF4E130B8
:105D20004860002108488160C16001610C21416127
:105D300000218161C161FDF7EFF908B1FAF7EAFBD3
:105D400010BD0000004C0040AC27002010B50B48EF
:105D50000B4908604FF4E130486000210848816039
:105D6000C16001610C21416100218161C161FDF7C8
:105D7000D3F908B1FAF7CEFB10BD00000050004087
:105D8000F027002010B50B480B4908604FF4E130B4
:105D90004860002108488160C16001610C214161B7
:105DA00000218161C161FDF7B7F908B1FAF7B2FBD3
:105DB00010BD0000003801403428002010B50B4809
:105DC0000B4908604FF4E1304860002108488160C9
:105DD000C16001610C21416100218161C161FDF758
:105DE0009BF908B1FAF796FB10BD00000044004093
:105DF0007828002010B50B480B4908604FF4E130BB
:105E00004860002108488160C16001610C21416146
:105E100000218161C161FDF77FF908B1FAF77AFBD2
:105E200010BD000000480040BC28002008B501203B
:105E30001023BEA200210090084600F0E6FC0120DD
:105E40001023BAA20F210090002000F0DEFC0120F8
:105E50001023B6A21E210090002000F0D6FC0120E5
:105E60001023B2A22D210090002000F0CEFCB148FA
:105E7000807803284FDC01201023AF4A00210090D6
:105E8000202000F0C2FC01201023AC4A0F2100901A
:105E9000202000F0BAFC01201023A94A1E21009006
:105EA000202000F0B2FC01201023A64A2D210090F2
:105EB000202000F0AAFC9F48807838B900201023E9
:105EC0009D4A01460090202000F09FFC9948807870
:105ED000012807D100201023984A0F21009020208C
:105EE00000F093FC93488078022807D1002010230B
:105EF000934A1E210090202000F087FC8D48807876
:105F0000032807D1002010238E4A2D210090202045
:105F100000F07BFC09E187488078032854DD854840
:105F20008078072850DC01201023874A0021009048
:105F3000202000F06AFC01201023844A0F210090E9
:105F4000202000F062FC01201023814A1E210090D5
:105F5000202000F05AFC012010237E4A2D210090C1
:105F6000202000F052FC73488078042807D10020DC
:105F70001023754A01460090202000F046FC6D4831
:105F80008078052807D100201023704A0F21009047
:105F9000202000F03AFC67488078062807D10020CE
:105FA00010236B4A1E210090202000F02EFC614837
:105FB00080780728AED100201023664A2D2100905A
:105FC000202000F022FCB0E05A488078072854DDF9
:105FD000584880780B2850DC012010235E4A0021AD
:105FE0000090202000F011FC012010235B4A0F21BB
:105FF0000090202000F009FC01201023584A1E21A7
:106000000090202000F001FC01201023554A2D2192
:106010000090202000F0F9FB46488078082807D13E
:10602000002010234C4A01460090202000F0EDFB98
:1060300040488078092807D100201023474A0F21C3
:106040000090202000F0E1FB3A4880780A2807D130
:1060500000201023424A1E210090202000F0D5FB92
:10606000344880780B2860D1002010233D4A2D2130
:106070000090202000F0C9FB57E02E4880780B28C4
:1060800053DD2C4880780F284FDC01201023364A3E
:1060900000210090202000F0B8FB01201023334A9B
:1060A0000F210090202000F0B0FB01201023304A87
:1060B0001E210090202000F0A8FB012010232D4A73
:1060C0002D210090202000F0A0FB1A4880780C2899
:1060D00007D100201023244A01460090202000F020
:1060E00094FB144880780D2807D1002010231F4A04
:1060F0000F210090202000F088FB0E4880780E28A9
:1061000007D1002010231A4A1E210090202000F001
:106110007CFB084880780F2807D100201023154AFF
:106120002D210090202000F070FB08BD4D41433A26
:1061300000000000F4020020FB0000200801002005
:1061400015010020220100202F0100203C01002029
:106150004901002056010020630100207001002049
:106160007D0100208A01002097010020A401002069
:10617000B1010020BE01002000BFFEE72DE9F04183
:106180000546002460E015F8248015F8240005EB8E
:1061900084014978484005EB84018978484005EB43
:1061A0008401C97880EA010615F8240005EB840112
:1061B000497880EA0107384606F046FC074615F89C
:1061C000240087EA0601484005F8240005EB840016
:1061D000407805EB8401897880EA0107384606F0AB
:1061E00033FC074605EB8400407887EA0601484007
:1061F00005EB8401487005EB8400807805EB840191
:10620000C97880EA0107384606F01EFC074605EB10
:106210008400807887EA0601484005EB8401887095
:1062200005EB8400C07880EA0807384606F00CFCCD
:10623000074605EB8400C07887EA0601484005EB75
:106240008401C870601CC4B2042C9CDBBDE8F081E2
:1062500000BFFEE770B500240CE0002506E000203A
:10626000074901EBC5010855681CC5B2802DF6DB56
:10627000601CC4B2082CF0DB00F0F0F870BD000028
:106280004003002010B504461CB90021A62000F0F0
:10629000E1FA012C03D10021A72000F0DBFA10BDA8
:1062A00010B504463CB90021C82000F0D3FA002103
:1062B000A12000F0CFFA012C07D10021C02000F06E
:1062C000C9FA0021A02000F0C5FA10BDF0B51446AF
:1062D0000B46CF1701EB5777C7F3C702CF1701EB78
:1062E0005777FF10A1EBC707FEB20123B340DDB221
:1062F0004CB1134B03EBC0039B5C2B43104F07EBDC
:10630000C007BB541AE00E4B03EBC0039B5CDB439E
:106310000B4F07EBC007BB54094B03EBC0039B5C5F
:106320002B43074F07EBC007BB54054B03EBC003E0
:106330009B5CDB43024F07EBC007BB54F0BD000082
:10634000400300201FB5A020009001200190039081
:1063500069464048FBF7E0F80122A0213D48FBF7E1
:106360008DFA002210213C48FBF788FAC820FAF782
:10637000EDFF012210213848FBF780FA0021AE2002
:1063800000F068FA0021022000F064FA00211020D9
:1063900000F060FA0021402000F05CFA0021B020FB
:1063A00000F058FA0021812000F054FA0021CF209B
:1063B00000F050FA0021A12000F04CFA0021A620A4
:1063C00000F048FA0021A82000F044FA00213F2004
:1063D00000F040FA0021AD2000F03CFA00218B20B3
:1063E00000F038FA0021332000F034FA0021C820F0
:1063F00000F030FA0021D32000F02CFA00210846EA
:1064000000F028FA0021D52000F024FA0021802095
:1064100000F020FA0021D92000F01CFA00211F20F2
:1064200000F018FA0021DA2000F014FA00211220FE
:1064300000F010FA0021DB2000F00CFA00214020CF
:1064400000F008FAFFF706FF0021AF2000F002FA83
:106450001FBD0000000801400010014070B500247D
:106460001CE004F1B001C8B2002100F0F3F90021F2
:10647000022000F0EFF90021102000F0EBF90025D8
:1064800008E0084901EBC501085D012100F0E2F9CF
:10649000681CC5B2802DF4DB601CC4B2082CE0DBA4
:1064A00070BD0000400300202DE9FE4F07468846DE
:1064B00092461C460197CDF80080082C02D14FF07F
:1064C00006091FE02046E31704EB5373DB10214657
:1064D0004FEAE47C04EB5C7C4FEAEC0CA4EBCC0CC4
:1064E000BCF1000F02D04FF0010C01E04FF0000CA6
:1064F0006344224604EBD27C4FEA6C0C03FB0CF3A2
:1065000003F0FF09AAF12000C6B200255EE0082CC6
:1065100007D106EB46002F4901EB400010F805B00B
:106520001DE00C2C07D106EB46002B4901EB800047
:1065300010F805B013E0102C05D1284800EB061028
:1065400010F805B00BE0182C07D106EBC600244963
:1065500001EB800010F805B001E0BDE8FE8F0020DF
:1065600002901CE00BF0010028B1414638460C9A1D
:10657000FFF7ACFE09E00C9808B9012000E000200C
:10658000024641463846FFF7A1FE4FEA6B0B08F181
:10659000010000F0FF080298401CC0B2029002986F
:1065A0000828DFDB781CC7B2082C0BD004EBD471B1
:1065B0004A100199791A8A4204D1019F0098083043
:1065C000C0B20090DDF80080681CC5B24D459EDB6E
:1065D00000BFC2E75CCA000884CC0008F8D00008FD
:1065E000E8D600082DE9FC4F0746884616461C46AB
:1065F000BB46CDF804802046E21704EB5272D2105D
:106600002146E31704EB5373DB10A4EBC3030BB178
:10661000012300E000231A44624392B20092002555
:1066200075E0102C05D13C4800EB461010F80590A1
:106630003BE0182C07D106EBC600384901EBC0003F
:1066400010F8059031E0202C05D1354800EBC6103C
:1066500010F8059029E0402C05D1324800EB462087
:1066600010F8059021E00C2C07D106EB46002E49CE
:1066700001EBC00010F8059017E00E2C07D1C6EB17
:10668000C6002A4901EB800010F805900DE0122C9D
:1066900009D106EBC60000EB4000254901EB4000A4
:1066A00010F8059001E0BDE8FC8F4FF0000A1CE0F7
:1066B00009F0010028B1414638460B9AFFF706FE63
:1066C00009E00B9808B9012000E00020024641468D
:1066D0003846FFF7FBFD4FEA690908F1010000F0B9
:1066E000FF080AF1010000F0FF0ABAF1080FDFDB32
:1066F000781CC7B2A7EB0B00A04204D15F460198FB
:106700000830C0B20190DDF80480681C85B20098A2
:10671000854286DB00BFC6E744E4000864E9000860
:10672000ACE900082CEA00082CEC000884EE000814
:10673000ECF000082DE9FF4F05460E4617461C46B3
:10674000DDF838904FF0000A0095B3462046E21776
:1067500004EB5272D2102146E31704EB5373DB10A3
:10676000A4EBC3030BB1012300E000231A44D4B20D
:106770004FF0000845E0002003903BE00D9810F832
:106780000A0002900AF101001FFA80FA002001902D
:106790001DE0029800F0010028B14A463146284623
:1067A000FFF794FD0AE0B9F1000F01D1012000E0EC
:1067B0000020024631462846FFF788FD0298401027
:1067C0000290701CC6B20198401CC0B201900198A2
:1067D0000828DEDB681CC5B20098281AB84204D12C
:1067E000009D0BF1080000F0FF0B5E460398401C73
:1067F000C0B203900398B842C0DB08F1010000F07A
:10680000FF08A045B7DBBDE8FF8F2DE9F84106463C
:106810000F4614461D46DDF81C8013E0CDF80080BD
:1068200022782B4639463046FFF73EFE082D02D12E
:10683000B01DC6B205E0284605EBD07106EB61013C
:10684000CEB2641C2078202802DB20787E28E5DD8B
:10685000BDE8F88170B504460E462EB101224021F4
:106860001C48FBF70BF804E0002240211948FBF715
:1068700005F8002210211748FBF700F800251BE05F
:10688000002220211348FAF7F9FF04F0800028B114
:10689000012280210F48FAF7F1FF04E00022802155
:1068A0000C48FAF7EBFF012220210A48FAF7E6FF2D
:1068B0006006040E681CC5B2082DE1DB0122102120
:1068C0000448FAF7DBFF012240210248FAF7D6FF1D
:1068D00070BD00000008014008B508490968C908F2
:1068E0004FF47A72B1FBF2F14143009100BF00BF57
:1068F00000994A1E00920029F9D108BD8C0200209F
:10690000014600BF080900EB8000420001F00F00C3
:106910001044C0B2704770B504460025FAF7B4FFC2
:10692000054607E0FAF7B0FF401BB0F57A7F01D9C2
:10693000032070BD2068406800F020000028F1D0DE
:106940002068406840F01000216848600020F0E7AF
:1069500070B5044600252068406820F010002168CA
:106960004860FAF791FF054607E0FAF78DFF401BF4
:10697000B0F57A7F01D9032070BD2068406800F02F
:1069800020000028F1D00020F6E7000010B50248F2
:10699000FBF75EFD10BD0000581E002001460022DE
:1069A00000230868006A82B20868406A83B243EA3A
:1069B0000240704730B50146002200230024002029
:1069C0000D68AD69AAB20D68ED69ACB20D68AD692C
:1069D000ABB29A4205D00D68ED6963F31F452846B6
:1069E00001E044EA024030BDF0B504460B46002108
:1069F000002504F5FA61032B1BD2C3EBC30000EBA7
:106A000003100926B0FBF6F01044001D4618481E7E
:106A100006EB90066427B0FBF7F0361A481EBF005D
:106A2000B0FBF7F030440726B0FBF6F706FB17057E
:106A30001AE0C3EBC30000EB03100926B0FBF6F02D
:106A40001044001D084400EB91006426B1FBF6F6EB
:106A5000801B4FF4C876B1FBF6F63044801E072643
:106A6000B0FBF6F706FB1705E8B2F0BD70B50446BB
:106A70000D4600262046FFF74EFF08B101260AE02A
:106A8000280C21680862A8B2216848622046FFF7F6
:106A90005FFF00B10126304670BD70B504460D465B
:106AA00000262046FFF737FF08B101260AE0280C30
:106AB00021688861A8B22168C8612046FFF748FFB5
:106AC00000B10126304670BD417842794270437A68
:106AD0004371437B437241738178827A8270817201
:106AE0008179837B83718173C178C27BC270C37AE1
:106AF000C373C379C372C171704700BF012003F033
:106B00007FFFFBE790B000BF012003F079FF05F0A5
:106B10008FFA03F0ADFD3C2207496846F9F782FB86
:106B2000054810380FC8FCF7F7FDFFF797FC03F096
:106B3000C5FD05F0D7FCE7E70403002000BF0120F6
:106B400003F05EFF0E48007840B100200C49087049
:106B50004FF4E160FAF7FAFBFEF71EFD09480078F2
:106B60000028ECD000200749087000BF06490870D3
:106B700048708870C870012004490870DFE7000081
:106B80007C020020FA000020F4020020F500002022
:106B900010B5364804F006FB3549088008460088E1
:106BA0004FF6FF71884213D101231A4631A132A05A
:106BB00005F0D4F8002857D04AF6AA212B4800F057
:106BC00013FE31A000F04EFE0120344908704BE066
:106BD000274800884AF6AA21884245D130A000F013
:106BE00041FE3220FAF7B2FB01231A4632A135A04A
:106BF00005F0B4F830B936A137A000F033FE01201B
:106C00002649087001231A4636A139A005F0A6F8D6
:106C100030B93AA130A000F025FE02201F490870CB
:106C200001231A4637A13AA005F098F830B93BA1E4
:106C300029A000F017FE03201849087001231A4606
:106C400038A13BA005F08AF838B93DA122A000F098
:106C500009FE04201149087006E03BA13FA000F0A6
:106C600001FE00200D49087010BD0000005007080B
:106C7000260200204F4B000041542B5245534554EF
:106C80003D310D0A00000000232323B8B4CEBBC958
:106C9000E8B1B8B3C9B9A60D0A0000002802002067
:106CA000232323C0B6D1C0C4A3BFE9B7C7CAD7B492
:106CB000CEC6F4B6AF0D0A002B55554944533A30B1
:106CC0003030320041542B55554944533F0D0A0092
:106CD00055554944530000002573B2BBB7FBBACFEA
:106CE0000A0000002B555549444E3A4646303400C0
:106CF00041542B555549444E3F0D0A0055554944C2
:106D00004E0000002B55554944573A46464635003B
:106D100041542B55554944573F0D0A005555494498
:106D2000570000002B5458504F5745523A3130000D
:106D300041542B5458504F5745523F0D0A00000004
:106D40005458504F5745520055554944CFEEBCB0AA
:106D5000B7A2C9E4B9A6C2CA00000000232573B7D0
:106D6000FBBACFC9E8D6C3CFEE0A000000BF4FF48C
:106D70007A7003F045FEFAE710B5024600200FE0F6
:106D8000002109E002EB81031B5C074CE35C02EB92
:106D9000810423544B1CD9B20429F3DB431CD8B221
:106DA0000428EDDB10BD000050F4000810B500BF52
:106DB000502080F31188BFF34F8FBFF36F8F00BF58
:106DC00005F010FD18B14FF080500449086000BF75
:106DD000002080F3118800BF10BD000004ED00E02A
:106DE00000B595B028210BA8F9F735FA142106A8AB
:106DF000F9F731FA18216846F9F72DFA09200B90B6
:106E00004FF480300C9000200D9001200F901190D5
:106E100002201290C10313914FF4E01114910BA8BA
:106E2000FBF7CAF808B1F9F775FB0F2006900220AE
:106E30000790002008904FF48060099000200A908D
:106E4000022106A8FAF760FF08B1F9F763FB0120F9
:106E50000090400201906846FAF7BEFE08B1F9F7CB
:106E600059FB15B000BD704710B50248FBF711FF84
:106E700010BD0000E02B002010B50248FBF709FF11
:106E800010BD00001C1F002010B54FF40071034816
:106E9000FAF7EAFC0248FBF7FCFE10BD00100140C7
:106EA000641F002010B50268204B98420ED0204B82
:106EB00098420BD0B0F1804F08D01E4B984205D0BD
:106EC0001D4B984202D01D4B984203D122F0700214
:106ED0004B681A43154B98420ED0154B98420BD075
:106EE000B0F1804F08D0134B984205D0124B984216
:106EF00002D0124B984203D122F44072CB681A435D
:106F000022F080034C6943EA040202608B68C3628A
:106F10000B688362054B984202D0054B984201D121
:106F20000B6903630123436110BD0000002C014085
:106F3000003401400004004000080040000C004004
:106F400030B50C46816821F47F4142EA0325254390
:106F50002943816030BD0A46816821F0700142F00A
:106F6000070319438160704730B50B461446026A27
:106F7000056A25F001050562816921F0F00141EA09
:106F8000041122F00A021A438161026230BD30B559
:106F90000B461446056A25F0100505628169026AF0
:106FA00021F4704141EA043122F0A00242EA0312C6
:106FB0008161026230BD000038B500251A480068C2
:106FC0000068C0F3001555B300BF002000901648BC
:106FD000006800680090144800684068009000BF96
:106FE00000BF1148FBF73EFF10480068446860424C
:106FF000801E0F49087001200E4908700C48007867
:107000000D4908700A4802780C490D48F9F70AF949
:107010004FF400620949891E0348FCF7EEFA024862
:10702000FBF754FF38BD0000AC27002000290020EA
:10703000700200207A02002078020020AE1F00209B
:107040002834002010B51F480068002808DD1E48BD
:1070500000680068C0F3001010B1002019490860F2
:10706000194800680068C0F3401030B31648006843
:107070004068C4B21548134909684454114800686F
:1070800040F2FF71884204D20E480068401C0D494E
:1070900008600C4800880E4908800A4801680D48BD
:1070A000F9F7D9F8002004E00849095C094A1154AD
:1070B000401C044909688842F6DB0348FBF706FFD9
:1070C00010BD000074020020F0270020DC07002023
:1070D0002A020020DC0F002070B505466C6A0020F3
:1070E000E085E0842046FBF7F0FE70BD70B50646F3
:1070F0000025746A20684069C0F3C01594F83D000B
:10710000212805D125B10020E084204600F085F833
:1071100020684069C0F3801594F83E00222805D10C
:1071200025B10020E085204600F04CF8206C40F0AE
:10713000100020642046FBF7C8FE70BD70B5054600
:107140006C6A2868006800F02000F8B90020E0852B
:107150002068C06820F480702168C8602068406999
:1071600020F00100216848612068406920F040005B
:1071700021684861202084F83E00206B012805D159
:107180002068C06820F010002168C860206B0128CA
:1071900004D1A18D2046FBF764FE02E02046FCF7F7
:1071A0004DFA70BD70B505466C6A206B012805D19B
:1071B000A08D41082046FBF754FE02E02046FCF774
:1071C0003EFA70BD0168C96821F490710268D1600F
:1071D0000168496921F0010102685161016B0129CF
:1071E00005D10168C96821F010010268D160202131
:1071F00080F83E1000210163704710B504462068F6
:10720000C06820F040002168C860202084F83D005C
:107210002046FCF77EFA002010BD0168C96821F005
:10722000C0010268D160202180F83D107047F8B598
:10723000044694F83E00222869D1A068B0F5805F2A
:107240000CD1206950B90025A66A20684068C0F3B7
:1072500008003080A06A801CA06215E0A56A0026A4
:10726000A068B0F5805F03D0A06828B9206918B97C
:1072700020684068287004E02068406800F07F00C3
:107280002870A06A401CA062E08D401E80B2E0859C
:10729000A8BB2068C06820F020002168C860206872
:1072A000C06820F480702168C8602068406920F0C0
:1072B000010021684861202084F83E00206B0128ED
:1072C0001ED1002020632068C06820F010002168D3
:1072D000C8602068006800F0100010280AD100BFC4
:1072E00000200090206800680090206840680090AE
:1072F00000BF00BFA18D2046FBF7B3FD03E004E013
:107300002046FCF79BF90020F8BD0020FCE7022096
:10731000FAE7000070B504462168096921F440517C
:10732000E2681143226811612269A1681143626910
:1073300041EA02052168C96841F20C629143294380
:107340002268D1602168496921F44071A269114322
:10735000226851612D4A2168914202D1FAF7D2FD8B
:1073600001E0FAF7BFFD00EBC00101EB001162681C
:107370009200B1FBF2F100EBC00202EB0012636875
:107380009B00B2FBF3F26423B2FBF3F202EBC20305
:1073900003EB0212A1EB8201322202EB0111642203
:1073A000B1FBF2F101F0F00100EBC00202EB0012C0
:1073B00063689B00B2FBF3F26423B2FBF3F201EBD0
:1073C000021200EBC00101EB001163689B00B1FBEE
:1073D000F3F100EBC00303EB00136668B600B3FBE8
:1073E000F6F36426B3FBF6F303EBC30606EB0313D5
:1073F000A1EB8301322303EB01116423B1FBF3F111
:1074000001F00F0111442268916070BD0038014005
:1074100077B581B0044615460298A062A585002084
:107420002064222084F83E001C48A16B88621C481E
:10743000A16BC8621B48A16B08630020A16B486365
:1074400002AE32682368191D2B46A06BF9F730FF96
:1074500000BF00200090206800680090206840680D
:10746000009000BF00BF00BF002084F83C0000BFB8
:107470002068C06840F480702168C8602068406956
:1074800040F00100216848612068406940F04000F8
:1074900021684861002004B070BD00003D71000803
:1074A000A5710008ED700008014691F83D00212803
:1074B00028D18868B0F5805F0BD1086948B90A6A9D
:1074C0001088C0F308000B685860086A801C0862C6
:1074D00005E00B6A581C086218780B685860C88C65
:1074E000401E80B2C88458B90868C06820F0800087
:1074F0000B68D8600868C06840F040000B68D8602E
:10750000002070470220FCE72DE9F04104460D46BB
:1075100017469846069E21E0701CF8B12EB1FAF786
:10752000B3F9A0EB0800B04218D92068C06820F475
:10753000D0702168C8602068406920F0010021688F
:107540004861202084F83D0084F83E0000BF002000
:1075500084F83C0000BF0320BDE8F081206800688B
:107560002840A84201D1012000E00020B842D3D039
:107570000020F1E710B50248FBF7A8FC10BD0000A1
:107580003428002010B50248FBF7A0FC10BD000015
:107590007828002010B50248FBF798FC10BD0000C9
:1075A000BC28002070B505460E461446A2B24FF620
:1075B000FF7331462846FCF743F8A2B24FF6FF733B
:1075C00031460248FCF73CF870BD0000BC280020A2
:1075D00070B505460C460DA000F044F92046F8F7BA
:1075E00057FE86B24FF6FF73324621462846FCF717
:1075F00027F82046F8F74CFE86B24FF6FF73324666
:1076000021460448FCF71CF870BD00000D0A434DEC
:10761000443A0900BC28002010B50248F9F7B6F832
:1076200010BD0000301E002010B50248F9F7AEF87A
:1076300010BD0000301E002000BFFEE708B5664800
:107640000078062875D2DFE800F0C306920403052F
:1076500000BF00BF00BF00201023604A0146009019
:107660001D20FFF7D2F8012010235D4A2021009051
:107670000D20FFF7CAF8012010235A4A202100905C
:107680006420FFF7C2F854480078042818D101207C
:1076900010232022114600902620FEF7A3FF012090
:1076A00010232122202100903A20FEF79BFF012089
:1076B00010232222202100904E20FEF793FF55E058
:1076C00045480078032818D1012010231E222021CC
:1076D00000902620FEF786FF012010231F22202184
:1076E00000903A20FEF77EFF012010230022202187
:1076F00000904E20FEF776FF38E0374800780128EA
:1077000018D110231622202100902620FEF76AFFB0
:10771000012010231722202100903A20FEF762FF5B
:10772000012010230022202100904E20FEF75AFF56
:107730001CE04DE028480078052817D101201023CF
:107740002322202100902620FEF74CFF0120102349
:107750002422202100903A20FEF744FF012010232C
:107760002522202100904E20FEF73CFF31E0012031
:107770000C231B4A342100901420FFF746F8012007
:107780000C231122342100902620FEF72BFF01202C
:107790000C231222342100903320FEF723FF012016
:1077A0000C231322342100904020FEF71BFF012000
:1077B0000C231422342100904D20FEF713FF0120EA
:1077C0000C23084A342100905C20FFF71EF800E0EB
:1077D00000BF00BF08BD0000CB010020CC0100208D
:1077E000D9010020D601002070B504460D46204680
:1077F00000F0FCF9F9F778FE0F48844208D00F48F2
:10780000844205D00E48844202D00E48844207D1FB
:107810002A46002321460220F9F70EFE064607E01D
:107820002A46002321460120F9F706FE064600BF3E
:10783000F9F7F8FD70BD00000038070800400708A0
:10784000004807080050070810B50246002005E070
:10785000135C0C5C63401354431CD8B21028F7DB54
:1078600010BD00000FB4054B10B503A9044A0298DF
:1078700000F034F810BC5DF814FB0000197C00081F
:10788000F002002002480068C0F3022070470000A8
:107890000CED00E010B5002804DB0A07130E054AC2
:1078A000135406E00A07140E034A00F00F031B1FCF
:1078B000D45410BD00E400E018ED00E002E008C878
:1078C000121F08C1002AFAD170477047002001E05A
:1078D00001C1121F002AFBD1704700002DE9FF4FA4
:1078E0008BB09A460F460546002606E025280BD0A9
:1078F00052460D9990476D1C761C28780028F5D1CA
:107900000FB03046BDE8F08F0024A0460122604948
:1079100000E0044315F8013F203B02FA03F008425F
:10792000F7D128782E2817D115F8010F44F0040458
:107930002A280ED06FF02F022878A0F130010929F3
:107940000AD808EB880102EB410100EB01086D1C2D
:10795000F2E757F8048B6D1C287869283ED006DCC6
:107960000028CDD063280BD0642804D136E07328DA
:1079700010D075284BD052460D999047761C85E063
:1079800017F8040B8DF8000000208DF80100E9467F
:10799000012003E057F8049B4FF0FF3061074FF0E0
:1079A000000401D40AE0641C44450DDA8442FADB89
:1079B00019F804100029F6D106E0641C8442FCDBAF
:1079C00019F804100029F8D1264404E019F8010B35
:1079D00052460D999047641EF8D257E001CF4FF000
:1079E0000A0B002802DA40422D2102E0210504D5CD
:1079F0002B218DF82410012103E0E10705D020217F
:107A0000F7E70DF1200908910CE00021F9E701CF1B
:107A10004FF00A0BF9E75946F8F741FC01F1300243
:107A200009F8012D0028F6D1ADEB090000F1200B7B
:107A3000600701D44FF00108D84502DDA8EB0B0028
:107A400000E000208046002406E009A85246005DC0
:107A50000D999047641C761C08988442F5DB04E07D
:107A6000302052460D999047761CB8F10001A8F1DC
:107A70000108F5DC05E019F8010B52460D99904715
:107A8000761CBBF10001ABF1010BF4DC6D1C34E79B
:107A90000928010008B50120102323221921009094
:107AA0000A20FEF79FFD01201023242219210090B7
:107AB0001E20FEF797FD012010232522192100909A
:107AC0003220FEF78FFD012010232622192100907D
:107AD0004620FEF787FD0120102327221921009060
:107AE0005A20FEF77FFD0120102328221921009043
:107AF0006E20FEF777FD08BD0FB470B586B028A0E4
:107B00000068059027A30FCB01AC0FC4294800786B
:107B1000042800D10A9C27480078052800D10B9C36
:107B200024480078062800D10C9C224800780728B9
:107B300000D10D9C200E8DF80600200C8DF807005A
:107B4000200A8DF80800E0B28DF809000E9E300E74
:107B50008DF80A00300C8DF80B00300A8DF80C00FF
:107B6000F0B28DF80D000F9D280E8DF80E00280C38
:107B70008DF80F00280A8DF81000E8B28DF811007A
:107B800001200E2301AA0221009005A804F024F987
:107B90001420F8F7B1FC06B070BC5DF814FB0000CF
:107BA00066010000030B0000000000000000000060
:107BB00000000000F402002070B502460B464FF6AC
:107BC000FF7000210FE0555C6840002508E000F0E0
:107BD0000104401014B14AF20106704080B26D1CDD
:107BE000082DF4D3491C9942EDD370BD30B585B052
:107BF000044600200190039401200490002000908E
:107C0000F9F772FC694601A8F9F7B4FB0546F9F7E4
:107C100009FC05B030BD000013B50C464FF6FF73EC
:107C2000012269460248FBF70BFD00981CBD0000CD
:107C3000BC2800200FB583B0FE48406958B1012030
:107C40000090FC4840690C2302461D210290082048
:107C5000FEF7DBFD07E001200C23F7A21D210090B9
:107C60000E20FEF7D2FDF348406A58B10120009083
:107C7000F048406A0C2302461D2102902620FEF7A0
:107C8000C4FD07E001200C23ECA21D2100902C2054
:107C9000FEF7BBFDE748406B58B101200090E54876
:107CA000406B0C2302461D2102904420FEF7ADFDDF
:107CB00007E001200C23E2A21D2100904A20FEF7DC
:107CC000A4FDDC48406C58B101200090D948406CBC
:107CD0000C2302461D2102906220FEF796FD07E06C
:107CE00001200C23D7A21D2100906820FEF78DFDF6
:107CF00041F2F0120398811A904201F09A847ADCE2
:107D000040F61172A0EB0201904275D038DCB0F55C
:107D1000887F72D018DCF02870D009DC01286ED082
:107D20000F286DD010286CD0112842F08483B6E162
:107D3000FF2867D0B0F5807F7DD0A0F20110002829
:107D40007AD00E28F1D15AE240F2FF12811A904205
:107D500073D00ADCA0F2111000286FD00E286ED06C
:107D6000DF286DD0E028E0D1CAE3A1F60151002957
:107D700067D0012966D00F2965D01029D5D1FEE240
:107D8000B1F5877F6FD015DCEF296DD008DC0E29A7
:107D90006BD0DF296AD0E02969D0EE29C5D1B4E3E0
:107DA000F02972D0FE2971D0FF2970D0B1F5807F03
:107DB000BBD1F7E3B1F5F87F01F03B820BDCA1F218
:107DC000DF11002977D0012976D00F2975D010292D
:107DD000ABD101F073B9B1F5FF7F01F02B82A1F2B5
:107DE000FF11002901F02484012901F01F860F29C9
:107DF0009BD101F01CBE06E084E3BDE2F8E0A8E000
:107E0000A8E0F4E04CE14DF60F72881A914276D06A
:107E10005DDC40F60162A1EB0200914201F00C86AC
:107E200036DC40F61F52A1EB0200914201F00482C1
:107E30001EDC012908E097E1DFE162E35EE35EE337
:107E40009CE292E1DCE1D9E101F0F2850F2901F039
:107E5000F085B1F5516F01F03381A1F61151002980
:107E60008CD101F0E8B9FDE3FDE34CE385E24BE39F
:107E7000012801F0DF83022801F0DC85102801F0E1
:107E8000DA85E1288AD101F0D6BBEDE3EDE3EDE33D
:107E90004DF21F02811A90427DD00FDC0E2801F0B6
:107EA000CC85A0F550400F38002875D0012874D03B
:107EB0000F288DD1F5E3F5E3F5E3F5E301296DD066
:107EC0000F296CD0E0296BD0E12991D1EDE340F688
:107ED0000162811A904201F0F2801FDC122801F049
:107EE000AD850DDC012801F0EC80022801F0A581B0
:107EF000102801F0A3811128B2D101F09DBBFDE350
:107F0000202801F09C85F12801F09783F22801F0E8
:107F10009785B0F5807FA3D101F093BD1F2901F0B3
:107F200092850CDC012901F08A810F2901F08881FA
:107F3000102901F08383112992D101F083BDF0292A
:107F400001F07D83F12901F07F85FF2988D101F0BF
:107F50007CBD00BF01200C233B4A0821009008464D
:107F6000FEF753FC01200C23374A082100902620FD
:107F7000FEF74BFC01200C23334A082100904420DB
:107F8000FEF743FC089880B30398012818D12F49C5
:107F900014231A4605E0FDE3FDE3FDE3FDE3FDE305
:107FA000FDE3CDE9001006216420FEF7C3FB0120AC
:107FB00010230B222E2100906620FEF713FB14E005
:107FC00003980F2811D10120214914231A46CDE925
:107FD000001006216420FEF7ADFB012010230C22C7
:107FE0002E2100906620FEF7FDFA02F045BA00BF90
:107FF00001200C23144A082100900846FEF705FCD6
:1080000001200C23104A082100902620FEF7FDFBDA
:1080100001200C230C4A082100906220FEF7F5FB9A
:10802000069828B30398102823D101200749142368
:108030001A460FE0F40200204C3100004C320000E0
:108040004C3300004C340000F00000200000002001
:108050003C000020CDE9001006214620FEF76AFB17
:10806000012010230B222E2100904820FEF7BAFA9F
:1080700014E00398F02811D10120FE4914231A4678
:10808000CDE9001006214620FEF754FB0120102305
:108090000C222E2100904820FEF7A4FAA5E700BF8D
:1080A00001200C23F44A082100900846FEF7ADFB9E
:1080B00001200C23F04A082100902620FEF7A5FBA2
:1080C000069840B3089830B30398112824D10120B2
:1080D000EA4914231A46CDE9001006214620FEF78E
:1080E00029FB012010230B222E2100904820FEF7AF
:1080F00079FA0120E14914231A46CDE9001006213E
:108100006420FEF717FB012010230B222E21009084
:108110006620FEF767FA26E00398FF2823D10120A6
:10812000D44914231A46CDE9001006214620FEF753
:1081300001FB012010230C222E2100904820FEF785
:1081400051FA0120CB4914231A46CDE9001006212B
:108150006420FEF7EFFA012010230C222E2100905C
:108160006620FEF73FFA40E700BF01200C23C24A19
:10817000082100900846FEF748FB01200C23BE4A68
:10818000082100904420FEF740FB01200C23BA4A4E
:10819000082100906220FEF738FB059860B3039831
:1081A000B0F5807F12D10120B44914231A46CDE9DD
:1081B000001006212820FEF7BDFA012010230B2213
:1081C0002E2100902A20FEF70DFA15E00398B0F555
:1081D000706F11D10120A74914231A46CDE9001070
:1081E00006212820FEF7A6FA012010230C222E21BA
:1081F00000902A20FEF7F6F9F7E600BF00BF00BFA7
:1082000001200C239C4A082100900846FEF7FDFA45
:1082100001200C23984A082100904420FEF7F5FA2B
:10822000059850B3089840B340F201110398884272
:1082300024D10120914914231A46CDE900100621CA
:108240002820FEF777FA012010230B222E21009020
:108250002A20FEF7C7F90120884914231A46CDE9E0
:10826000001006216420FEF765FA012010230B227E
:108270002E2100906620FEF7B5F97CE040F60F71E4
:108280000398884224D101207A4914231A46CDE963
:10829000001006212820FEF74DFA012010230C22A1
:1082A0002E2100902A20FEF79DF901207149142308
:1082B0001A46CDE9001006216420FEF73BFA0120A2
:1082C00010230C222E2100906620FEF78BF952E03D
:1082D00040F20F110398884224D1012067491423EA
:1082E0001A46CDE9001006212820FEF723FA0120C6
:1082F00010230B222E2100902A20FEF773F9012073
:108300005C4914231A46CDE9001006216420FEF7CB
:1083100011FA012010230C222E2100906620FEF776
:1083200061F928E040F601710398884223D10120C9
:10833000504914231A46CDE9001006212820FEF7E3
:10834000F9F9012010230C222E2100902A20FEF79B
:1083500049F90120494914231A46CDE900100621A4
:108360006420FEF7E7F9012010230B222E21009054
:108370006620FEF737F938E600BF00BF00BF0120D6
:108380000C233D4A082100900846FEF73EFA0120E2
:108390000C23394A082100906220FEF736FA05982E
:1083A00048B3069838B30398B0F5887F24D10120EC
:1083B000324914231A46CDE9001006212820FEF781
:1083C000B9F9012010230B222E2100902A20FEF75C
:1083D00009F90120294914231A46CDE90010062184
:1083E0004620FEF7A7F9012010230B222E21009032
:1083F0004820FEF7F7F880E00398B0F57F6F24D1AE
:1084000001201C4914231A46CDE90010062128201A
:10841000FEF790F9012010230C222E2100902A2033
:10842000FEF7E0F80120134914231A46CDE90010A5
:1084300006214620FEF77EF9012010230C222E2172
:1084400000904820FEF7CEF857E00398B0F5F87F8B
:108450002BD10120094914231A46CDE90010062129
:108460002820FEF767F9012010230B222E2100900F
:108470002A2005E03C000020F00000200000002041
:10848000FEF7B0F80120FE4914231A46CDE900108A
:1084900006214620FEF74EF9012010230C222E2142
:1084A00000904820FEF79EF827E00398B0F5716F22
:1084B00023D10120F24914231A46CDE900100621E8
:1084C0002820FEF737F9012010230C222E210090DE
:1084D0002A20FEF787F80120EA4914231A46CDE93D
:1084E000001006214620FEF725F9012010230B225B
:1084F0002E2100904820FEF775F876E500BF00BFFA
:1085000000BF00BF00BF00BF00BF01200C23DE4A38
:10851000082100900846FEF778F90598002840D019
:1085200006980028FBD008980028F8D040F21111D6
:108530000398884237D10120D24914231A46CDE945
:10854000001006212820FEF7F5F8012010230B2249
:108550002E2100902A20FEF745F80120C949142356
:108560001A46CDE9001006214620FEF7E3F8012067
:1085700010230B222E2100904820FEF733F8012013
:10858000C04914231A46CDE9001006216420FEF7E5
:10859000D1F8012010230B222E2100906620FEF737
:1085A00021F8BEE18CE340F21F110398884236D1D6
:1085B0000120B44914231A46CDE9001006212820D1
:1085C000FEF7B8F8012010230B222E2100902A205C
:1085D000FEF708F80120AB4914231A46CDE9001034
:1085E00006214620FEF7A6F8012010230B222E219B
:1085F00000904820FDF7F6FF0120A14914231A46F8
:10860000CDE9001006216420FEF794F80120102324
:108610000C222E2100906620FDF7E4FF81E140F25C
:10862000F1110398884241D10120964914231A463A
:10863000CDE9001006212820FEF77CF80120102348
:108640000B222E2100902A20FDF7CCFF01208C491F
:1086500014231A46CDE9001006214620FEF76AF8D9
:10866000012004E02DE35DE1A5E1A6E162E2102333
:108670000C222E2100904820FDF7B4FF01208149F3
:1086800014231A46CDE9001006216420FEF752F8A3
:10869000012010230B222E2100906620FDF7A2FF5F
:1086A0003FE189E148E20DE30DE30FE340F2FF1102
:1086B0000398884238D10120724914231A46CDE923
:1086C000001006212820FEF735F8012010230B2288
:1086D0002E2100902A20FDF785FF012068491423F0
:1086E0001A46CDE9001006214620FEF723F80120A6
:1086F00010230C222E210090482000E0E7E2FDF735
:1087000071FF01205E4914231A46CDE900100621AD
:108710006420FEF70FF8012010230C222E21009078
:108720006620FDF75FFFFCE040F611710398884278
:108730003DD10120524914231A46CDE900100621EB
:108740002820FDF7F7FF012010230C222E21009096
:108750002A20FDF747FF01204A4914231A46CDE994
:10876000001006214620FDF7E5FF012010230B2213
:108770002E2100904820FDF735FF012041491423A8
:108780001A46CDE9001006216420FDF7D3FF012031
:10879000102305E0D1E1C6E010E195E295E2CAE1DF
:1087A0000B222E2100906620FDF71CFFB9E040F659
:1087B0001F710398884236D10120314914231A468B
:1087C000CDE9001006212820FDF7B4FF0120102379
:1087D0000C222E2100902A20FDF704FF01202949B8
:1087E00014231A46CDE9001006214620FDF7A2FF0A
:1087F000012010230B222E2100904820FDF7F2FECD
:1088000001201F4914231A46CDE9001006216420D7
:10881000FDF790FF012010230C222E2100906620EE
:10882000FDF7E0FE7DE040F6F171039888423DD10E
:108830000120134914231A46CDE9001006212820EF
:10884000FDF778FF012010230C222E2100902A2012
:10885000FDF7C8FE01200A4914231A46CDE900108D
:1088600006214620FDF766FF012010230C222E2151
:1088700000904820FDF7B6FE01200249142305E0D0
:108880003C00002000000020F00000201A46CDE946
:10889000001006216420FDF74DFF012010230B225C
:1088A0002E2100906620FDF79DFE3AE040F6FF7114
:1088B0000398884235D10120FE4914231A46CDE998
:1088C000001006212820FDF735FF012010230C227F
:1088D0002E2100902A20FDF785FE0120F549142362
:1088E0001A46CDE9001006214620FDF723FF01209E
:1088F00010230C222E2100904820FDF773FE01204A
:10890000EC4914231A46CDE9001006216420FDF736
:1089100011FF012010230C222E2100906620FDF76C
:1089200061FE20E400BF01200C23E34A08210090EF
:108930002620FDF76AFF01200C23DF4A0821009062
:108940004420FDF762FF01200C23DB4A0821009040
:108950006220FDF75AFF049860B30398B0F5805F7A
:1089600012D10120D54914231A46CDE90010062161
:108970000A20FDF7DFFE012010230B222E2100909C
:108980000C20FDF72FFE15E00398B0F5704F11D1C4
:108990000120C84914231A46CDE9001006210A20F7
:1089A000FDF7C8FE012010230C222E210090104656
:1089B000FDF718FE20E400BF00BF00BF01200C231C
:1089C000BD4A082100902620FDF71FFF01200C233F
:1089D000B94A082100904420FDF717FF049850B3CE
:1089E000089840B341F201010398884224D1012044
:1089F000B24914231A46CDE9001006210A20FDF7DA
:108A000099FE012010230B222E2100900C20FDF74F
:108A1000E9FD0120A94914231A46CDE900100621D9
:108A20006420FDF787FE012010230B222E210090E9
:108A30006620FDF7D7FD7CE04FF20F0103988842D6
:108A400024D101209B4914231A46CDE900100621A8
:108A50000A20FDF76FFE012010230C222E2100902A
:108A60001046FDF7BFFD0120924914231A46CDE9B7
:108A7000001006216420FDF75DFE012010230C226A
:108A80002E2100906620FDF7ADFD52E041F20F016E
:108A90000398884224D10120884914231A46CDE93D
:108AA000001006210A20FDF745FE012010230B22AD
:108AB0002E2100900C20FDF795FD01207D49142307
:108AC0001A46CDE9001006216420FDF733FE01208F
:108AD00010230C222E2100906620FDF783FD28E054
:108AE0004FF201010398884223D1012071491423D8
:108AF0001A46CDE9001006210A20FDF71BFE0120D1
:108B000010230C222E2100901046FDF76BFD012052
:108B10006A4914231A46CDE9001006216420FDF7A6
:108B200009FE012010230B222E2100906620FDF764
:108B300059FD20E400BF00BF00BF01200C235E4AA6
:108B4000082100902620FDF760FE01200C235A4AE0
:108B5000082100906220FDF758FE049850B3069853
:108B600040B341F210010398884224D101205349B7
:108B700014231A46CDE9001006210A20FDF7DAFD7C
:108B8000012010230B222E2100900C20FDF72AFD3E
:108B900001204A4914231A46CDE900100621462037
:108BA000FDF7C8FD012010230B222E210090482044
:108BB000FDF718FD7CE04FF2F0010398884224D1C4
:108BC00001203C4914231A46CDE9001006210A2051
:108BD000FDF7B0FD012010230C222E21009010463D
:108BE000FDF700FD0120334914231A46CDE900109A
:108BF00006214620FDF79EFD012010230C222E2188
:108C000000904820FDF7EEFC52E041F2F00103989D
:108C1000884224D10120294914231A46CDE90010A5
:108C200006210A20FDF786FD012010230B222E21AC
:108C300000900C20FDF7D6FC01201E4914231A4693
:108C4000CDE9001006214620FDF774FD0120102318
:108C50000C222E2100904820FDF7C4FC28E04FF2A2
:108C600010010398884223D10120124914231A4687
:108C7000CDE9001006210A20FDF75CFD012010233C
:108C80000C222E2100901046FDF7ACFC01200B4970
:108C900014231A46CDE9001006214620FDF74AFDAF
:108CA000012010230B222E2100904820FDF79AFC72
:108CB00023E400003C000020F00000200000002021
:108CC00000BF00BF00BF00BF00BF00BF00BF01204A
:108CD0000C23F74A082100902620FDF796FD049802
:108CE000002840D006980028FBD008980028F8D02B
:108CF00041F211010398884236D10120ED49142335
:108D00001A46CDE9001006210A20FDF713FD0120C7
:108D100010230B222E2100900C20FDF763FC012074
:108D2000E44914231A46CDE9001006214620FDF738
:108D300001FD012010230B222E2100904820FDF779
:108D400051FC0120DB4914231A46CDE9001006210D
:108D50006420FDF7EFFC012010230B222E21009050
:108D60006620FDF73FFCA2E141F21F010398884213
:108D700036D10120CF4914231A46CDE9001006212F
:108D80000A20FDF7D7FC012010230B222E21009092
:108D90000C20FDF727FC0120C64914231A46CDE913
:108DA000001006214620FDF7C5FC012010230B22F0
:108DB0002E2100904820FDF715FC0120BE49142308
:108DC0001A46CDE9001006216420FDF7B3FC01200E
:108DD00010230C222E2100906620FDF703FC66E193
:108DE00041F2F1010398884236D10120B1491423A0
:108DF0001A46CDE9001006210A20FDF79BFC012050
:108E000010230B222E2100900C20FDF7EBFB0120FC
:108E1000A94914231A46CDE9001006214620FDF782
:108E200089FC012010230C222E2100904820FDF700
:108E3000D9FB01209F4914231A46CDE900100621D1
:108E40006420FDF777FC012010230B222E210090D7
:108E50006620FDF7C7FB2AE141F2FF010398884233
:108E600036D10120934914231A46CDE9001006217A
:108E70000A20FDF75FFC012010230B222E21009019
:108E80000C20FDF7AFFB01208B4914231A46CDE9D6
:108E9000001006214620FDF74DFC012010230C2276
:108EA0002E2100904820FDF79DFB012082491423CC
:108EB0001A46CDE9001006216420FDF73BFC012095
:108EC00010230C222E2100906620FDF78BFBEEE094
:108ED0004FF211010398884236D1012076491423BC
:108EE0001A46CDE9001006210A20FDF723FC0120D7
:108EF00010230C222E2100901046FDF773FB012059
:108F00006C4914231A46CDE9001006214620FDF7CE
:108F100011FC012010230B222E2100904820FDF788
:108F200061FB0120634914231A46CDE90010062194
:108F30006420FDF7FFFB012010230B222E2100905F
:108F40006620FDF74FFBB2E04FF21F010398884205
:108F500036D10120584914231A46CDE900100621C4
:108F60000A20FDF7E7FB012010230C222E210090A0
:108F70001046FDF737FB01204E4914231A46CDE970
:108F8000001006214620FDF7D5FB012010230B22FF
:108F90002E2100904820FDF725FB0120464914238F
:108FA0001A46CDE9001006216420FDF7C3FB01201D
:108FB00010230C222E2100906620FDF713FB76E093
:108FC0004FF2F1010398884236D101203A49142327
:108FD0001A46CDE9001006210A20FDF7ABFB01205F
:108FE00010230C222E2100901046FDF7FBFA0120E1
:108FF000314914231A46CDE9001006214620FDF719
:1090000099FB012010230C222E2100904820FDF70F
:10901000E9FA0120274914231A46CDE90010062158
:109020006420FDF787FB012010230B222E210090E6
:109030006620FDF7D7FA3AE04FF2FF010398884225
:1090400035D101201C4914231A46CDE90010062110
:109050000A20FDF76FFB012010230C222E21009027
:109060001046FDF7BFFA0120134914231A46CDE933
:10907000001006214620FDF75DFB012010230C2285
:109080002E2100904820FDF7ADFA01200A49142353
:109090001A46CDE9001006216420FDF74BFB0120A4
:1090A00010230C222E2100906620FDF79BFA38E455
:1090B000F0000020000000203C00002000BF00BFA6
:1090C00000BF01200C23FD4A082100904420FDF739
:1090D0009CFB01200C23F94A082100906220FDF737
:1090E00094FB049848B3059838B30398B0F5885FAB
:1090F00024D10120F24914231A46CDE9001006219B
:109100000A20FDF717FB012010230B222E210090CF
:109110000C20FDF767FA0120E94914231A46CDE92E
:10912000001006212820FDF705FB012010230B224B
:109130002E2100902A20FDF755FA79E00398B0F52A
:109140007F4F24D10120DF4914231A46CDE90010B6
:1091500006210A20FDF7EEFA012010230C222E2111
:1091600000901046FDF73EFA0120D64914231A4616
:10917000CDE9001006212820FDF7DCFA012010239C
:109180000C222E2100902A20FDF72CFA50E00398A3
:10919000B0F5F85F24D10120C94914231A46CDE95E
:1091A000001006210A20FDF7C5FA012010230B222A
:1091B0002E2100900C20FDF715FA0120C14914233F
:1091C0001A46CDE9001006212820FDF7B3FA012048
:1091D00010230C222E2100902A20FDF703FA27E00D
:1091E0000398B0F5714F23D10120B64914231A46D4
:1091F000CDE9001006210A20FDF79CFA012010237A
:109200000C222E2100901046FDF7ECF90120AC490C
:1092100014231A46CDE9001006212820FDF78AFA0A
:10922000012010230B222E2100902A20FDF7DAF9CD
:109230007FE400BF00BF00BF00BF00BF00BF00BF92
:1092400001200C239D4A082100904420FDF7DDFAFF
:109250000498002840D005980028FBD008980028E2
:10926000F8D041F201110398884236D10120944987
:1092700014231A46CDE9001006210A20FDF75AFAF8
:10928000012010230B222E2100900C20FDF7AAF9BB
:1092900001208B4914231A46CDE90010062128200D
:1092A000FDF748FA012010230B222E2100902A20DE
:1092B000FDF798F90120824914231A46CDE90010E0
:1092C00006216420FDF736FA012010230B222E21FF
:1092D00000906620FDF786F9A9E141F20F1103988D
:1092E000884236D10120764914231A46CDE9001070
:1092F00006210A20FDF71EFA012010230B222E2141
:1093000000900C20FDF76EF901206D4914231A46D8
:10931000CDE9001006212820FDF70CFA01201023CA
:109320000B222E2100902A20FDF75CF901206549CF
:1093300014231A46CDE9001006216420FDF7FAF93E
:10934000012010230C222E2100906620FDF74AF9FF
:109350006DE141F601710398884236D101205849E8
:1093600014231A46CDE9001006210A20FDF7E2F980
:10937000012010230B222E2100900C20FDF732F942
:109380000120504914231A46CDE900100621282057
:10939000FDF7D0F9012010230C222E2100902A2065
:1093A000FDF720F90120464914231A46CDE90010A3
:1093B00006216420FDF7BEF9012010230B222E2187
:1093C00000906620FDF70EF931E141F60F71039828
:1093D000884236D101203A4914231A46CDE90010BB
:1093E00006210A20FDF7A6F9012010230B222E21C9
:1093F00000900C20FDF7F6F80120324914231A469C
:10940000CDE9001006212820FDF794F90120102352
:109410000C222E2100902A20FDF7E4F80120294992
:1094200014231A46CDE9001006216420FDF782F9C5
:10943000012010230C222E2100906620FDF7D2F887
:10944000F5E04FF20111039888423DD101201D49FA
:1094500014231A46CDE9001006210A20FDF76AF907
:10946000012010230C222E2100901046FDF7BAF89F
:109470000120134914231A46CDE9001006212820A3
:10948000FDF758F9012010230B222E2100902A20ED
:10949000FDF7A8F801200A4914231A46CDE9001067
:1094A00006216420FDF746F9012010230B222E210E
:1094B00000906620FDF796F8B9E00000F00000206B
:1094C000000000203C0000204FF20F11039888425A
:1094D00036D10120F84914231A46CDE9001006219F
:1094E0000A20FDF727F9012010230C222E210090DD
:1094F0001046FDF777F80120F04914231A46CDE90C
:10950000001006212820FDF715F9012010230B2259
:109510002E2100902A20FDF765F80120E64914234A
:109520001A46CDE9001006216420FDF703F9012059
:1095300010230C222E2100906620FDF753F876E0D0
:109540004FF601710398884236D10120DA4914237D
:109550001A46CDE9001006210A20FDF7EBF801209C
:1095600010230C222E2100901046FDF73BF801201D
:10957000D14914231A46CDE9001006212820FDF711
:10958000D9F8012010230C222E2100902A20FDF76B
:1095900029F80120C94914231A46CDE900100621F3
:1095A0006420FDF7C7F8012010230B222E21009024
:1095B0006620FDF717F83AE04FF60F7103988842DE
:1095C00035D10120BC4914231A46CDE900100621EB
:1095D0000A20FDF7AFF8012010230C222E21009065
:1095E0001046FCF7FFFF0120B34914231A46CDE9CA
:1095F000001006212820FDF79DF8012010230C22E1
:109600002E2100902A20FCF7EDFF0120AA49142307
:109610001A46CDE9001006216420FDF78BF80120E1
:1096200010230C222E2100906620FCF7DBFF3EE584
:1096300000BF00BF00BF00BF00BF00BF00BF0120D0
:109640000C239F4A082100906220FDF7DEF8049861
:10965000002840D005980028FBD006980028F8D0B4
:1096600041F210110398884236D101209349142306
:109670001A46CDE9001006210A20FDF75BF801200B
:1096800010230B222E2100900C20FCF7ABFF0120B1
:109690008A4914231A46CDE9001006214620FDF719
:1096A00049F8012010230B222E2100904820FCF7BE
:1096B00099FF0120814914231A46CDE900100621A3
:1096C0002820FDF737F8012010230B222E210090CF
:1096D0002A20FCF787FFA8E141F2F01103988842A5
:1096E00036D10120754914231A46CDE90010062110
:1096F0000A20FDF71FF8012010230B222E210090D5
:109700000C20FCF76FFF01206C4914231A46CDE9A9
:10971000001006212820FDF70DF8012010230B2250
:109720002E2100902A20FCF75DFF012062491423BE
:109730001A46CDE9001006214620FCF7FBFF012068
:1097400010230C222E2100904820FCF74BFF6CE1E7
:1097500041F610710398884236D1012057491423ED
:109760001A46CDE9001006210A20FCF7E3FF01208C
:1097700010230B222E2100900C20FCF733FF012038
:109780004D4914231A46CDE9001006212820FCF784
:10979000D1FF012010230C222E2100902A20FCF75B
:1097A00021FF0120454914231A46CDE90010062166
:1097B0004620FCF7BFFF012010230B222E21009032
:1097C0004820FCF70FFF30E141F6F0710398884222
:1097D00036D10120394914231A46CDE9001006215B
:1097E0000A20FCF7A7FF012010230B222E21009056
:1097F0000C20FCF7F7FE01202F4914231A46CDE96F
:10980000001006212820FCF795FF012010230C22D0
:109810002E2100902A20FCF7E5FE01202649142382
:109820001A46CDE9001006214620FCF783FF0120EF
:1098300010230C222E2100904820FCF7D3FEF4E0E8
:109840004FF21011039888423CD101201A49142389
:109850001A46CDE9001006210A20FCF76BFF012013
:1098600010230C222E2100901046FCF7BBFE012095
:10987000124914231A46CDE9001006212820FCF7CE
:1098800059FF012010230B222E2100902A20FCF7E3
:10989000A9FE0120094914231A46CDE9001006212A
:1098A0004620FCF747FF012010230B222E210090B9
:1098B0004820FCF797FEB8E03C00002000000020A4
:1098C000F00000204FF2F0110398884236D10120B9
:1098D000FE4914231A46CDE9001006210A20FCF7A0
:1098E00029FF012010230C222E2100901046FCF7A6
:1098F00079FE0120F64914231A46CDE9001006210D
:109900002820FCF717FF012010230B222E210090A6
:109910002A20FCF767FE0120EC4914231A46CDE902
:10992000001006214620FCF705FF012010230C2221
:109930002E2100904820FCF755FE76E04FF610717E
:109940000398884236D10120E04914231A46CDE914
:10995000001006210A20FCF7EDFE012010230C2246
:109960002E2100901046FCF73DFE0120D74914231C
:109970001A46CDE9001006212820FCF7DBFE012065
:1099800010230C222E2100902A20FCF72BFE012010
:10999000CF4914231A46CDE9001006214620FCF7D2
:1099A000C9FE012010230B222E2100904820FCF735
:1099B00019FE3AE04FF6F0710398884235D1012044
:1099C000C24914231A46CDE9001006210A20FCF7EB
:1099D000B1FE012010230C222E2100901046FCF72E
:1099E00001FE0120B94914231A46CDE900100621D1
:1099F0002820FCF79FFE012010230C222E2100902E
:109A00002A20FCF7EFFD0120B04914231A46CDE9C6
:109A1000001006214620FCF78DFE012010230C22A9
:109A20002E2100904820FCF7DDFD00E600BF00BFBE
:109A300000BF00BF00BF00BF00BF00BF00BF00BF2E
:109A400000BF00BF00BF00BF00BF0498002855D072
:109A500005980028FBD006980028F8D00898002820
:109A6000F5D041F211110398884248D1012098495C
:109A700014231A46CDE9001006210A20FCF75AFEED
:109A8000012010230B222E2100900C20FCF7AAFDB0
:109A900001208F4914231A46CDE900100621282001
:109AA000FCF748FE012010230B222E2100902A20D3
:109AB000FCF798FD0120864914231A46CDE90010D1
:109AC00006214620FCF736FE012010230B222E2112
:109AD00000904820FCF786FD01207D4914231A469A
:109AE000CDE9001006216420FCF724FE012010239C
:109AF0000B222E2100906620FCF774FD25E241F236
:109B00001F110398884248D10120714914231A4635
:109B1000CDE9001006210A20FCF70CFE01201023DD
:109B20000B222E2100900C20FCF75CFD01206849DF
:109B300014231A46CDE9001006212820FCF7FAFD6F
:109B4000012010230B222E2100902A20FCF74AFD31
:109B500001205F4914231A46CDE900100621462052
:109B6000FCF7E8FD012010230B222E210090482055
:109B7000FCF738FD0120554914231A46CDE90010A1
:109B800006216420FCF7D6FD012010230C222E2193
:109B900000906620FCF726FDD7E141F2F111039811
:109BA000884248D101204A4914231A46CDE90010C1
:109BB00006210A20FCF7BEFD012010230B222E21D6
:109BC00000900C20FCF70EFD0120414914231A4699
:109BD000CDE9001006212820FCF7ACFD0120102360
:109BE0000B222E2100902A20FCF7FCFC0120374993
:109BF00014231A46CDE9001006214620FCF79AFDF1
:109C0000012010230C222E2100904820FCF7EAFCB2
:109C100001202F4914231A46CDE9001006216420A3
:109C2000FCF788FD012010230B222E2100906620D6
:109C3000FCF7D8FCFEE341F2FF11039888424DD1B6
:109C40000120234914231A46CDE9001006210A20D9
:109C5000FCF770FD012010230B222E2100900C2018
:109C6000FCF7C0FC01201A4914231A46CDE9001064
:109C700006212820FCF75EFD012010230B222E2157
:109C800000902A20FCF7AEFC0120104914231A464C
:109C9000CDE9001006214620FCF74CFD01201023E1
:109CA0000C222E2100904820FCF79CFC0120074943
:109CB00014231A46CDE9001006216420FCF73AFD72
:109CC000012010230C222E21009003E03C000020F4
:109CD000000000206620FCF785FCABE341F6117123
:109CE0000398884248D10120FE4914231A46CDE941
:109CF000001006210A20FCF71DFD012010230B2275
:109D00002E2100900C20FCF76DFC0120F649142355
:109D10001A46CDE9001006212820FCF70BFD012092
:109D200010230C222E2100902A20FCF75BFC01203E
:109D3000EC4914231A46CDE9001006214620FCF711
:109D4000F9FC012010230B222E2100904820FCF763
:109D500049FC0120E34914231A46CDE900100621ED
:109D60006420FCF7E7FC012010230B222E21009039
:109D70006620FCF737FC5DE341F61F7103988842CB
:109D800048D10120D74914231A46CDE900100621F5
:109D90000A20FCF7CFFC012010230B222E2100907B
:109DA0000C20FCF71FFC0120CF4914231A46CDE9F3
:109DB000001006212820FCF7BDFC012010230C22F6
:109DC0002E2100902A20FCF70DFC0120C549142308
:109DD0001A46CDE9001006214620FCF7ABFC012015
:109DE00010230B222E2100904820FCF7FBFB0120C2
:109DF000BD4914231A46CDE9001006216420FCF762
:109E000099FC012010230C222E2100906620FCF7E3
:109E1000E9FB0FE341F6F1710398884248D1012034
:109E2000B04914231A46CDE9001006210A20FCF798
:109E300081FC012010230B222E2100900C20FCF726
:109E4000D1FB0120A84914231A46CDE900100621B0
:109E50002820FCF76FFC012010230C222E210090FB
:109E60002A20FCF7BFFB01209F4914231A46CDE9A5
:109E7000001006214620FCF75DFC012010230C2277
:109E80002E2100904820FCF7ADFB012095491423BA
:109E90001A46CDE9001006216420FCF74BFC012096
:109EA00010230B222E2100906620FCF79BFBC1E2C1
:109EB00041F6FF710398884248D101208949142353
:109EC0001A46CDE9001006210A20FCF733FC0120D8
:109ED00010230B222E2100900C20FCF783FB012085
:109EE000814914231A46CDE9001006212820FCF7E9
:109EF00021FC012010230C222E2100902A20FCF7A7
:109F000071FB0120784914231A46CDE9001006217F
:109F10004620FCF70FFC012010230C222E2100907C
:109F20004820FCF75FFB01206F4914231A46CDE956
:109F3000001006216420FCF7FDFB012010230C22F9
:109F40002E2100906620FCF74DFB73E24FF21111B9
:109F50000398884248D10120634914231A46CDE969
:109F6000001006210A20FCF7E5FB012010230C223B
:109F70002E2100901046FCF735FB0120594914238F
:109F80001A46CDE9001006212820FCF7D3FB01205A
:109F900010230B222E2100902A20FCF723FB012006
:109FA000504914231A46CDE9001006214620FCF73B
:109FB000C1FB012010230B222E2100904820FCF72A
:109FC00011FB0120474914231A46CDE90010062150
:109FD0006420FCF7AFFB012010230B222E21009000
:109FE0006620FCF7FFFA25E24FF21F110398884222
:109FF00048D101203C4914231A46CDE9001006211E
:10A000000A20FCF797FB012010230C222E21009040
:10A010001046FCF7E7FA0120324914231A46CDE92D
:10A02000001006212820FCF785FB012010230B22BD
:10A030002E2100902A20FCF7D5FA0120294914236B
:10A040001A46CDE9001006214620FCF773FB0120DB
:10A0500010230B222E2100904820FCF7C3FA012088
:10A06000214914231A46CDE9001006216420FCF78B
:10A0700061FB012010230C222E2100906620FCF7AA
:10A08000B1FAD7E14FF2F111039888424DD1012086
:10A09000154914231A46CDE9001006210A20FCF7C1
:10A0A00049FB012010230C222E2100901046FCF7C2
:10A0B00099FA01200B4914231A46CDE90010062114
:10A0C0002820FCF737FB012010230B222E210090C3
:10A0D0002A20FCF787FA0120034914231A46CDE908
:10A0E000001003E0000000203C0000200621462074
:10A0F000FCF720FB012010230C222E210090482089
:10A10000FCF770FA0120DE4914231A46CDE900104D
:10A1100006216420FCF70EFB012010230B222E21C8
:10A1200000906620FCF75EFA84E14FF2FF1103987D
:10A13000884248D10120D34914231A46CDE90010A2
:10A1400006210A20FCF7F6FA012010230C222E210A
:10A1500000901046FCF746FA0120C94914231A461C
:10A16000CDE9001006212820FCF7E4FA0120102395
:10A170000B222E2100902A20FCF734FA0120C1493D
:10A1800014231A46CDE9001006214620FCF7D2FA26
:10A19000012010230C222E2100904820FCF722FAE7
:10A1A0000120B84914231A46CDE900100621642085
:10A1B000FCF7C0FA012010230C222E21009066200B
:10A1C000FCF710FA36E14FF611710398884248D136
:10A1D0000120AC4914231A46CDE9001006210A20BB
:10A1E000FCF7A8FA012010230C222E210090104623
:10A1F000FCF7F8F90120A34914231A46CDE9001011
:10A2000006212820FCF796FA012010230C222E218B
:10A2100000902A20FCF7E6F90120994914231A46F8
:10A22000CDE9001006214620FCF784FA0120102316
:10A230000B222E2100904820FCF7D4F901209049F0
:10A2400014231A46CDE9001006216420FCF772FAA7
:10A25000012010230B222E2100906620FCF7C2F96A
:10A26000E8E04FF61F710398884248D101208549E4
:10A2700014231A46CDE9001006210A20FCF75AFAE9
:10A28000012010230C222E2100901046FCF7AAF981
:10A2900001207C4914231A46CDE90010062128200C
:10A2A000FCF748FA012010230C222E2100902A20CE
:10A2B000FCF798F90120724914231A46CDE90010E1
:10A2C00006214620FCF736FA012010230B222E210E
:10A2D00000904820FCF786F901206A4914231A46A9
:10A2E000CDE9001006216420FCF724FA0120102398
:10A2F0000C222E2100906620FCF774F99AE04FF6AC
:10A30000F1710398884248D101205E4914231A460E
:10A31000CDE9001006210A20FCF70CFA01201023D9
:10A320000C222E2100901046FCF75CF901205549C3
:10A3300014231A46CDE9001006212820FCF7FAF96B
:10A34000012010230C222E2100902A20FCF74AF92C
:10A3500001204C4914231A46CDE90010062146205D
:10A36000FCF7E8F9012010230C222E210090482050
:10A37000FCF738F90120424914231A46CDE90010B0
:10A3800006216420FCF7D6F9012010230B222E2190
:10A3900000906620FCF726F94CE04FF6FF71039819
:10A3A000884247D10120374914231A46CDE90010CD
:10A3B00006210A20FCF7BEF9012010230C222E21D1
:10A3C00000901046FCF70EF901202E4914231A467E
:10A3D000CDE9001006212820FCF7ACF9012010235C
:10A3E0000C222E2100902A20FCF7FCF801202549A0
:10A3F00014231A46CDE9001006214620FCF79AF9ED
:10A40000012010230C222E2100904820FCF7EAF8AE
:10A4100001201C4914231A46CDE9001006216420AE
:10A42000FCF788F9012010230C222E2100906620D1
:10A43000FCF7D8F820E001200C23134A08210090F3
:10A440000846FCF7E2F901200C230F4A082100908E
:10A450002620FCF7DAF901200C230B4A0821009092
:10A460004420FCF7D2F901200C23074A0821009070
:10A470006220FCF7CAF900BF00BF07B000BD0000B2
:10A48000000000203C000020F000002090B0F7F712
:10A490000DFAFCF7A5FCFBF745FAFBF7A5F9FBF76E
:10A4A00085FBFBF7C9FBFBF7FDFBFBF76BFCFBF741
:10A4B00085FCFBF79FFCFBF72DFCFBF747FCFBF74C
:10A4C00099FBFBF757F9FBF7B9FA2448F8F714FBA7
:10A4D0002348F8F711FB00BFFBF734FF0020FBF720
:10A4E000D1FE0020FBF7DCFE00BF00BF1D48006866
:10A4F000C06840F010001B490968C8604FF4006252
:10A5000019491848F9F779F800BF18480068C06879
:10A5100040F0200015490968C86000BF14A0FDF78D
:10A52000A1F9BB20184908700320184908703C2283
:10A53000154910316846F5F775FE13480FC8F9F74D
:10A54000EBF8FBF78BFF00BF00F086FDFAF7BAFED1
:10A55000FBF7AAF900F060FA00BFFEE71C1F00201D
:10A56000641F0020AC270020AC1F0020F027002033
:10A570004A4C5F4454555F424C30312D73746172C4
:10A58000742E2E2E0D0A0000F4020020CB010020B4
:10A5900008B50120102314220D2100900A20FCF799
:10A5A00021F80120102315220D2100901B20FCF71B
:10A5B00019F80120102327A20D2100902C20FCF770
:10A5C00024F9012010231C220D2100903F20FCF7CC
:10A5D00009F8012010231D220D2100905020FCF7C6
:10A5E00001F8012010230D22282100900A20FBF7FA
:10A5F000F9FF012010230E22282100902120FBF7D3
:10A60000F1FF012010230F22282100903720FBF7B3
:10A61000E9FF012010231A46282100905020FBF763
:10A62000E1FF0D484078012808D1002010230BA23B
:10A630000D2100906420FCF7E8F80AE00648407815
:10A6400038B90020102305A2282100906420FCF7CF
:10A65000DCF808BD534E0000F40200203C2D2D0014
:10A6600001460020842901D0CA1C10447047000014
:10A6700000B54FF480524FF470410C48008801F04F
:10A68000B7FC4FF480724FF470610948008801F004
:10A69000AFFC1022F0210748008801F0A9FC01223C
:10A6A0000F210548008801F0A3FC00BDF601002041
:10A6B000F8010020FA010020FC0100200EB58F48AF
:10A6C000C078042873D18D48007804280BD08B48BB
:10A6D0000078052807D089480078062803D08748E5
:10A6E00000780728EED185480078042838D18448BE
:10A6F0000068401C824908600846008881B2814891
:10A70000FDF772F87D484078012813D17C4AD2E9E0
:10A7100004109269CDE90102009179480FC8FDF754
:10A72000EBF942F222217848FDF75EF83220F6F785
:10A730000DFE15E07148407890B9714AD2E90410D5
:10A740009269CDE9010200916D480FC800F0F4F85C
:10A7500041F211116C48FDF747F83220F6F7F6FD8B
:10A7600066480078052837D165484068401C644930
:10A7700048600846808881B26448FDF735F85F4834
:10A780004078012814D15E49D1E904028969CDE9F4
:10A79000012100905A480FC8FDF7AEF942F222217C
:10A7A0005B48FDF721F83220F6F7D0FD14E0A4E075
:10A7B0005248407880B9524A103207CA8DE80700E3
:10A7C0004F480FC800F0B8F841F211115048FDF79A
:10A7D0000BF83220F6F7BAFD48480078062836D143
:10A7E00047488068401C464988600846008981B215
:10A7F0004848FCF7F9FF41484078012811D1404A08
:10A80000103207CA8DE807003D480FC8FDF774F9FC
:10A8100042F222214048FCF7E7FF3220F6F796FD8E
:10A8200015E03648407890B9354AD2E9041092696B
:10A83000CDE90102009132480FC800F07DF841F2E5
:10A8400011113548FCF7D0FF3220F6F77FFD2B4879
:10A850000078072834D12A48C068401C2849C860BD
:10A860000846808981B22D48FCF7BEFF2348407816
:10A87000012811D1224A103207CA8DE8070020486A
:10A880000FC8FDF739F942F222212548FCF7ACFF49
:10A890003220F6F75BFD13E01848407880B9184A7B
:10A8A000103207CA8DE8070015480FC800F044F8B9
:10A8B00041F211111A48FCF797FF3220F6F746FDD6
:10A8C000114800F06FFC17490880114800F06AFC3D
:10A8D00015490880104800F065FC144908801048AC
:10A8E00000F060FC124908806420F6F72FFD032079
:10A8F0000249C87001200F4908700EBDF402002003
:10A90000C0070020003807080000070800400708BB
:10A910000010070800480708002007080050070833
:10A9200000300708F6010020F8010020FA0100209D
:10A93000FC010020F50000200FB470B586B02AA0FD
:10A940000068059029A30FCB01AC0FC42B480078F9
:10A95000042800D10A9C29480078052800D10B9CC6
:10A9600026480078062800D10C9C24480078072847
:10A9700000D10D9C200E8DF80600200C8DF80700EC
:10A98000200A8DF80800E0B28DF809000E9E300E06
:10A990008DF80A00300C8DF80B00300A8DF80C0091
:10A9A000F0B28DF80D000F9D280E8DF80E00280CCA
:10A9B0008DF80F00280A8DF81000E8B28DF811000C
:10A9C0009DF840008DF8120001200F2301AA0221FA
:10A9D000009005A801F000FA1420F5F78DFD06B0EF
:10A9E00070BC5DF814FB000066010000020C000062
:10A9F000000000000000000000000000F402002041
:10AA000070B5044625460DB1294600E001210846EF
:10AA100001F014FC002070BD10B501F03DFC0020D9
:10AA200010BD7FB504460D46606998B1A06988B134
:10AA3000B4F90800FFF714FE0646D4E90510CDE985
:10AA4000006102902B462269D4E9001001F06EFEED
:10AA5000039013E0B4F90800FFF702FE064603A8CE
:10AA6000CDE90060238A9AB22B46D4E9001001F0A8
:10AA70002BFE012802D0002004B070BD0398FBE734
:10AA80002DE9F04105460E461C4807681C48006841
:10AA9000001D01F0D7FA50B91948006890F82C1041
:10AAA0000120884017490968814316480160681CE5
:10AAB00038B936B112480168091D134801F00CFB82
:10AAC0001AE07C190E4800684460BC4207D20C486A
:10AAD0000168091D0D48006801F0E4FA0CE008481F
:10AAE0000168091D0A48006801F0DCFA094800689D
:10AAF000844201D207480460BDE8F081A40200202E
:10AB000090020020A8020020243D0020980200208E
:10AB100094020020C002002010B5044601F0E8FABB
:10AB200023480068401C224908602248006840B958
:10AB3000204804600846006801280DD100F03AF969
:10AB40000AE01D48006838B91A480068C06AE16A1E
:10AB5000884201D81748046018480068401C17490B
:10AB6000086094F82C1001208840154909680843B2
:10AB700013490860E16A01EB8101124A02EB81008E
:10AB8000211D01F0A9FA01F0DDFA0B48006868B157
:10AB900008480068C06AE16A884207D24FF08050D6
:10ABA00009490860BFF34F8FBFF36F8F10BD0000DE
:10ABB000A002002090020020AC020020BC02002075
:10ABC000A8020020483C002004ED00E010B516E08B
:10ABD00001F08EFA0C48C068C468201D01F032FAFA
:10ABE0000A480068401E0949086009480068401E7C
:10ABF0000749086001F0A6FA204600F00BF8044867
:10AC000000680028E4D110BD103D0020A002002003
:10AC10009C02002010B5044694F8510030B9206B16
:10AC200001F0AEFA204601F0ABFA1AE094F85100B8
:10AC3000012803D1204601F0A3FA12E094F8510054
:10AC4000022801D1012000E0002050B900BF5020AF
:10AC500080F31188BFF34F8FBFF36F8F00BF00BF2A
:10AC6000FEE710BD30B54FF44063174800F007040D
:10AC70002CB1C01D20F00700134C041B1B1B024607
:10AC8000124C22600024114D6C60D018083820F05E
:10AC900007000F4C206000240D4D2D686C600C4D9A
:10ACA0002D682C601146441A4C60094C24680C60D5
:10ACB000084D4C682C60084D4C682C604FF00044E7
:10ACC000064D2C6030BD0000383D0020CC02002035
:10ACD000D4020020DC020020D8020020E002002084
:10ACE00000BFFFF773FF064800680128F9D94FF04D
:10ACF000805004490860BFF34F8FBFF36F8FF0E7B8
:10AD0000483C002004ED00E02DE9FF5F81460F463E
:10AD10009246DDE90E6B109CAAF10100216B01EB5C
:10AD2000800828F0070808F0070008B9012000E0B3
:10AD3000002050B900BF502080F31188BFF34F8F1F
:10AD4000BFF36F8F00BF00BFFEE7002507E0795D0E
:10AD500004F134004155785D00B902E06D1C102DFE
:10AD6000F5D300BF002143200155072E00D306264E
:10AD7000E66266640020A064201D01F090F904F1F1
:10AD8000180001F08CF92461C6F10700A06164622B
:10AD90000020E06484F8500049464046039A00F0E1
:10ADA00049F92060BBF1000F01D0CBF80040BDE8AD
:10ADB000FF9F000010B5002407E004EB84010F4A58
:10ADC00002EB810001F05EF9641C072CF5D30C48FE
:10ADD00001F058F90B4801F055F90B4801F052F910
:10ADE0000A4801F04FF90A4801F04CF904480949B2
:10ADF000086004480849086010BD0000483C002075
:10AE0000D43C0020E83C0020FC3C0020103D002009
:10AE1000243D0020940200209802002010B5014635
:10AE2000164800E0006803688B42FBD30246436883
:10AE300013448B4204D143684C6823444360014669
:10AE40000A464B6813440468A34211D10C4C0368B2
:10AE50002468A34208D04B680468646823444B60AC
:10AE600003681B680B6005E0054B1B680B6001E085
:10AE700003680B60884200D0016010BDCC02002046
:10AE8000D40200200A490968096809B9012100E0D3
:10AE9000002121B14FF0FF31064A116006E004495C
:10AEA0000968C968C868034A4168116070470000B2
:10AEB00094020020C00200200E480068401C08B91F
:10AEC000012000E0002050B900BF502080F311881D
:10AED000BFF34F8FBFF36F8F00BF00BFFEE700BF10
:10AEE000502080F31188BFF34F8FBFF36F8F00BFE7
:10AEF00000BFFEE7E40200202DE9F04104464FF0D8
:10AF0000000801F021FA4648006808B9FFF7AAFED8
:10AF100044480068204000286BD1D4B1083404F0C4
:10AF20000700B0B104F00700C0F10800044404F0C9
:10AF3000070008B9012000E0002050B900BF5020F0
:10AF400080F31188BFF34F8FBFF36F8F00BF00BF37
:10AF5000FEE7002C4DD034480068844249D8334E77
:10AF60003046056801E02E462D686868A04202D28E
:10AF700028680028F7D12A480068854239D030680F
:10AF800000F10808286830606868001B102819D98B
:10AF90002F1907F0070008B9012000E0002050B980
:10AFA00000BF502080F31188BFF34F8FBFF36F8F26
:10AFB00000BF00BFFEE76868001B78606C60384621
:10AFC000FFF72CFF184968680968081A16490860D5
:10AFD0000846006816490968884203D2124800688A
:10AFE000134908600F4968680968084368600020D1
:10AFF000286001F09BFC08F0070008B9012000E080
:10B00000002050B900BF502080F31188BFF34F8F4C
:10B01000BFF36F8F00BF00BFFEE74046BDE8F08181
:10B02000D4020020E0020020D8020020CC02002040
:10B03000DC020020001F4FF080730360001F21F02E
:10B0400001030360001F034B0360143802602038C3
:10B0500070470000B9AE00082DE9F05F00F0A8F8D5
:10B060003A4800F09FF88046394800F09BF8814646
:10B07000384800F097F88246374800F093F8834646
:10B08000364800F092F80446354800F08EF8054640
:10B09000344800F08AF80646334800F086F8074640
:10B0A0004FF6FF70804502D00120304908704FF6FE
:10B0B000FF70814502D001202D4908704FF6FF70C6
:10B0C000824502D001202B4908704FF6FF7083455E
:10B0D00002D0012028490870601C18B901202749B6
:10B0E000086001E025480460681C18B90120234964
:10B0F000486001E021484560701C18B901201F49D3
:10B10000886001E01D488660781C18B901201B4941
:10B11000C86001E01948C760194800F043F81949B0
:10B120000880194800F03EF818490880184800F0D7
:10B1300039F818490880184800F034F81749088091
:10B14000012017490870BDE8F09F00000060070863
:10B150000068070800770708007807080038070824
:10B16000004007080048070800500708F6000020C4
:10B17000F7000020F8000020F9000020C0070020A0
:10B1800000000708F601002000100708F801002061
:10B1900000200708FA01002000300708FC01002009
:10B1A000F50000200146088870470146086870478E
:10B1B0002DE9F0417448FFF7F5FF04467348FFF7A7
:10B1C000F1FF05467248FFF7EDFF06467148FFF7AD
:10B1D000E9FF0746012C09D16FA07149486171A0B0
:10B1E000886076A0C86001207B490870022C09D1D4
:10B1F0007AA06B4948617BA0886080A0C86001206C
:10B2000075490870032C09D183A06549486184A061
:10B21000886089A0C86001206F490870042C09D19A
:10B220008CA05F4948618DA0886092A0C860012011
:10B2300069490870052C09D195A05949486196A023
:10B2400088609BA0C860012063490870062C09D162
:10B250009EA0534948619FA08860A4A0C8600120B7
:10B260005D490870072C09D1A7A04D494861A8A0E5
:10B270008860ADA0C860012057490870082C09D12A
:10B28000B0A047494861B1A08860B6A0C86001205D
:10B2900051490870092C09D1B9A041494861BAA0A7
:10B2A0008860BFA0C86001204B4908700A2C09D1F2
:10B2B000C2A03B494861C3A08860C8A0C860012003
:10B2C000454908700B2C09D1CBA035494861CCA069
:10B2D0008860D1A0C86001203F4908700C2C09D1BA
:10B2E000D4A02F494861D5A08860DAA0C8600120A9
:10B2F000394908700D2C09D1DDA029494861DEA02B
:10B300008860E3A0C8600120334908700E2C09D181
:10B31000E6A023494861E7A08860ECA0C86001204E
:10B320002D4908700F2C09D1EFA01D494861F0A0EC
:10B330008860F5A0C860012027490870102C09D149
:10B34000F8A017494861F9A08860FEA0C8600120F4
:10B3500021490870012D09D10FA01149486211A09F
:10B36000886116A0C8610120FD490870022D09D12D
:10B370001AA00B4948621BA0886120A0C861012067
:10B38000F749EFE1EFE100000060070800680708F7
:10B3900000770708007807083030303100000000DF
:10B3A000F402002041542B434F4E4E3D313031309A
:10B3B00030303030303030310D0A00002B434F4EEA
:10B3C0004E45435445443A302C31303130303030E2
:10B3D0003030303031000000F600002030303032A4
:10B3E0000000000041542B434F4E4E3D3130313070
:10B3F00030303030303030320D0A00002B434F4EA9
:10B400004E45435445443A302C31303130303030A1
:10B410003030303032000000303030330000000077
:10B4200041542B434F4E4E3D31303130303030306F
:10B43000303030330D0A00002B434F4E4E454354FD
:10B4400045443A302C3130313030303030303030CB
:10B4500033000000303030340000000041542B43F2
:10B460004F4E4E3D3130313030303030303030346E
:10B470000D0A00002B434F4E4E45435445443A308D
:10B480002C3130313030303030303030340000004A
:10B49000303030350000000041542B434F4E4E3DBC
:10B4A0003130313030303030303030350D0A00003E
:10B4B0002B434F4E4E45435445443A302C313031A6
:10B4C0003030303030303030350000003030303601
:10B4D0000000000041542B434F4E4E3D313031307F
:10B4E00030303030303030360D0A00002B434F4EB4
:10B4F0004E45435445443A302C31303130303030B1
:10B50000303030303600000030303037000000007E
:10B5100041542B434F4E4E3D31303130303030307E
:10B52000303030370D0A00002B434F4E4E45435408
:10B5300045443A302C3130313030303030303030DA
:10B5400037000000303030380000000041542B43F9
:10B550004F4E4E3D31303130303030303030303879
:10B560000D0A00002B434F4E4E45435445443A309C
:10B570002C31303130303030303030303800000055
:10B58000303030390000000041542B434F4E4E3DC7
:10B590003130313030303030303030390D0A000049
:10B5A0002B434F4E4E45435445443A302C313031B5
:10B5B0003030303030303030390000003030304101
:10B5C0000000000041542B434F4E4E3D313031308E
:10B5D00030303030303030410D0A00002B434F4EB8
:10B5E0004E45435445443A302C31303130303030C0
:10B5F0003030303041000000303030420000000078
:10B6000041542B434F4E4E3D31303130303030308D
:10B61000303030420D0A00002B434F4E4E4543540C
:10B6200045443A302C3130313030303030303030E9
:10B6300042000000303030430000000041542B43F2
:10B640004F4E4E3D3130313030303030303030437D
:10B650000D0A00002B434F4E4E45435445443A30AB
:10B660002C31303130303030303030304300000059
:10B67000303030440000000041542B434F4E4E3DCB
:10B680003130313030303030303030440D0A00004D
:10B690002B434F4E4E45435445443A302C313031C4
:10B6A0003030303030303030440000003030304501
:10B6B0000000000041542B434F4E4E3D313031309D
:10B6C00030303030303030450D0A00002B434F4EC3
:10B6D0004E45435445443A302C31303130303030CF
:10B6E000303030304500000030303046000000007F
:10B6F00041542B434F4E4E3D31303130303030309D
:10B70000303030460D0A00002B434F4E4E45435417
:10B7100045443A302C3130313030303030303030F8
:10B7200046000000303031300000000041542B430F
:10B730004F4E4E3D3130313030303030303031309E
:10B740000D0A00002B434F4E4E45435445443A30BA
:10B750002C3130313030303030303031300000007A
:10B76000F70000200870032D0CD1AFF25430FE49D1
:10B770004862AFF254308861AFF24430C8610120B2
:10B78000FA490870042D0CD1AFF23830F6494862FE
:10B79000AFF238308861AFF22430C8610120F3493C
:10B7A0000870052D0CD1AFF21830EF494862AFF2A6
:10B7B00018308861AFF20830C8610120EB49087089
:10B7C000062D0CD1AFF2FC20E7494862AFF2FC2015
:10B7D0008861AFF2E820C8610120E4490870072DB4
:10B7E0000CD1AFF2DC20E0494862AFF2DC20886186
:10B7F000AFF2CC20C8610120DC490870082D0CD1C3
:10B80000AFF2C020D8494862AFF2C0208861AFF2E1
:10B81000AC20C8610120D5490870092D0CD1AFF2C8
:10B82000A020D1494862AFF2A0208861AFF29020F9
:10B83000C8610120CD4908700A2D0CD1AFF28420D7
:10B84000C9494862AFF284208861AFF27020C861B4
:10B850000120C64908700B2D0CD1AFF26420C249FB
:10B860004862AFF264208861AFF25420C8610120C1
:10B87000BE4908700C2D0CD1AFF24820BA4948627D
:10B88000AFF248208861AFF23420C8610120B74987
:10B8900008700D2D0CD1AFF22820B3494862AFF2E9
:10B8A00028208861AFF21820C8610120AF490870D4
:10B8B0000E2D0CD1AFF20C20AB494862AFF20C2038
:10B8C0008861AFF2F810C8610120A84908700F2DF7
:10B8D0000CD1AFF2EC10A4494862AFF2EC108861D1
:10B8E000AFF2DC10C8610120A0490870102D0CD106
:10B8F000AFF2D0109C494862AFF2D0108861AFF22D
:10B90000BC10C861012099490870012E0CD1AFF21A
:10B91000785095494863AFF274508862AFF2645032
:10B92000C862012092490870022E0CD1AFF2545027
:10B930008D494863AFF254508862AFF24050C862FC
:10B9400001208B490870032E0CD1AFF23450864988
:10B950004863AFF234508862AFF22450C8620120CD
:10B9600083490870042E0CD1AFF218507E49486309
:10B97000AFF218508862AFF20450C86201207C49CF
:10B980000870052E0CD1AFF2F84077494863AFF24A
:10B99000F8408862AFF2E840C8620120744908703C
:10B9A000062E0CD1AFF2DC406F494863AFF2DC40A9
:10B9B0008862AFF2C840C86201206D490870072E46
:10B9C0000CD1AFF2BC4068494863AFF2BC4088621A
:10B9D000AFF2AC40C862012065490870082E0CD156
:10B9E000AFF2A04060494863AFF2A0408862AFF276
:10B9F0008C40C86201205E490870092E0CD1AFF25C
:10BA0000804059494863AFF280408862AFF270408D
:10BA1000C8620120564908700A2E0CD1AFF264406A
:10BA200051494863AFF264408862AFF25040C86247
:10BA300001204F4908700B2E0CD1AFF244404A4907
:10BA40004863AFF244408862AFF23440C8620120DC
:10BA5000474908700C2E0CD1AFF228404249486388
:10BA6000AFF228408862AFF21440C862012040491A
:10BA700008700D2E0CD1AFF208403B494863AFF27D
:10BA800008408862AFF2F830C86201203849087077
:10BA90000E2E0CD1AFF2EC3033494863AFF2EC30EC
:10BAA0008862AFF2D830C8620120314908700F2E89
:10BAB0000CD1AFF2CC302C494863AFF2CC30886265
:10BAC000AFF2BC30C862012029490870102E0CD199
:10BAD000AFF2B03024494863AFF2B0308862AFF2C1
:10BAE0009C30C862012022490870012F0CD1AFF2AE
:10BAF00058701D494864AFF254708863AFF24470C7
:10BB0000C86301201B490870022F0CD1AFF23470BA
:10BB100015494864AFF234708863AFF22070C8638F
:10BB2000012014490870032F0CD1AFF214700E4994
:10BB30004864AFF214708863AFF20470C8630120E8
:10BB40000C490870042F0CD1AFF2F8600649486424
:10BB5000AFF2F8608863AFF2E460C8630120054982
:10BB60000870052F15D107E0F4020020F70000202F
:10BB7000F8000020F9000020AFF2EC60584948645A
:10BB8000AFF2EC608863AFF2D860C863012055491A
:10BB90000870062F0CD1AFF2CC6051494864AFF267
:10BBA000CC608863AFF2BC60C86301204D49087067
:10BBB000072F0CD1AFF2B06049494864AFF2B060D2
:10BBC0008863AFF29C60C863012046490870082F63
:10BBD0000CD1AFF2906042494864AFF29060886344
:10BBE000AFF28060C86301203E490870092F0CD174
:10BBF000AFF274603A494864AFF274608863AFF2A0
:10BC00006060C8630120374908700A2F0CD1AFF279
:10BC1000546033494864AFF254608863AFF24460C3
:10BC2000C86301202F4908700B2F0CD1AFF2386088
:10BC30002B494864AFF238608863AFF22460C86370
:10BC40000120284908700C2F0CD1AFF2186024494C
:10BC50004864AFF218608863AFF20860C8630120DF
:10BC6000204908700D2F0CD1AFF2FC501C494864DC
:10BC7000AFF2FC508863AFF2E850C8630120194965
:10BC800008700E2F0CD1AFF2DC5015494864AFF2AA
:10BC9000DC508863AFF2CC50C863012011490870B2
:10BCA0000F2F0CD1AFF2C0500D494864AFF2C05015
:10BCB0008863AFF2AC50C86301200A490870102FA6
:10BCC0000CD1AFF2A05006494864AFF2A05088638F
:10BCD000AFF29050C863012002490870BDE8F081BE
:10BCE000F4020020F90000202DE9F04704468946BF
:10BCF00015461E46002700BF21E005EB85004FEAF0
:10BD0000400821461048FBF763FC3220F5F71EFB84
:10BD10000E490FA0FBF7A6FD0AE049460B48F4F7D1
:10BD2000A5FA10B10120BDE8F0876420F5F70EFBFD
:10BD3000B8F10000A8F10108EFD1781CC7B2B742F2
:10BD4000DBDB0020EFE70000AC27002028340020D8
:10BD50002D2D2D2D2D2D2D3E257300002DE9F04785
:10BD60000446894615461E46002700BF25E005EB20
:10BD700085004FEA400821461248FBF729FC1E20A7
:10BD8000F5F7E4FA104911A0FBF76CFD0EE0494607
:10BD90000D48F4F76BFA30B132210B48F4F75BFA37
:10BDA0000120BDE8F0876420F5F7D0FAB8F1000073
:10BDB000A8F10108EBD1781CC7B2B742D7DB00204D
:10BDC000EFE70000F0270020DC0F00202D2D2D2DA7
:10BDD0002D2D2D3E257300002DE9F0478AB0054634
:10BDE000884616461C46DDF84890142105A8F4F74D
:10BDF00032FA28788DF8140068788DF815002146FD
:10BE0000304600F015FE824600200190029003901B
:10BE1000049000BF03E0315C01AA1154401CA04211
:10BE2000F9D301A800F804A0B9F1000F09D0144A11
:10BE300014491548F4F7A5FA102201A91248F4F79D
:10BE400082FA002006E001A9095C00EB080205ABBC
:10BE50009954401C1028F6DB122105A8FBF7ACFE14
:10BE60000746F8B28DF82600380A8DF8270014220C
:10BE700005A90648FBF796FB0AB0BDE8F08700006D
:10BE80005002002040020020202B0020F02700203C
:10BE900008B50120102350A2022100901420FAF7C7
:10BEA000B4FC01200E231422022100903220FAF764
:10BEB00099FB01200E231522022100904620FAF75B
:10BEC00091FB0120102345A2112100901420FAF7C4
:10BED0009CFC01200E231422112100903220FAF73D
:10BEE00081FB01200E231522112100904620FAF734
:10BEF00079FB012010233AA2202100901420FAF7A8
:10BF000084FC01200E231422202100903220FAF715
:10BF100069FB01200E231522202100904620FAF70C
:10BF200061FB012010232FA22F2100901420FAF78B
:10BF30006CFC01200E2314222F2100903220FAF7EE
:10BF400051FB01200E2315222F2100904620FAF7E5
:10BF500049FB2548407803280BD12348807840B915
:10BF60000020102321A2022100906420FAF74DFC4A
:10BF700030E01D48407802280CD11B488078012809
:10BF800008D10020102319A2112100906420FAF793
:10BF90003CFC1FE01448407801280CD112488078FE
:10BFA000022808D10020102310A220210090642034
:10BFB000FAF72BFC0EE00C48407858B90A48807814
:10BFC000032807D10020102308A22F21009064200D
:10BFD000FAF71BFC08BD00004C2031004C20320059
:10BFE0004C2033004C203400F40200203C2D2D0066
:10BFF00010B541F2111398420DD10C4B5B680B4008
:10C000008B4202D1094B5A600EE0084B5B68134328
:10C01000064C636008E042F22223984204D1034BAD
:10C020005B680B43014C636010BD0000F40200200C
:10C0300010B5F7F72DFCF7F721FDF7F70FFEF8F72E
:10C04000DDFE10BD01460A69D1E901309860D1E9F1
:10C05000010358605068884201D188685060002010
:10C0600008611068401E106010687047034B036041
:10C07000034B0B608023136070470000DC17002027
:10C080003018002000F1080141604FF0FF3181605D
:10C0900000F10801C16001610021016070470021C9
:10C0A0000161704710B502460B685C1C0CB9106941
:10C0B00007E002F1080000E04068446824689C4200
:10C0C000FAD944684C604C68A160886041600A619C
:10C0D0001468641C146010BD42684A6093688B60E9
:10C0E000936859609160086103685B1C0360704746
:10C0F00000BF502080F31188BFF34F8FBFF36F8FC5
:10C1000000BF0E480068401C0C49086008460068E3
:10C11000012812D10A480068C0B208B9012000E025
:10C12000002050B900BF502080F31188BFF34F8F1B
:10C13000BFF36F8F00BF00BFFEE77047E40200202F
:10C1400004ED00E00D48006850B900BF502080F3B6
:10C150001188BFF34F8FBFF36F8F00BF00BFFEE7A3
:10C1600006480068401E054908600846006820B976
:10C17000002080F3118800BF00BF7047E402002058
:10C1800070B506463546002E3FD0083D2C461F4967
:10C1900060680968084008B1012000E0002050B93B
:10C1A00000BF502080F31188BFF34F8FBFF36F8F14
:10C1B00000BF00BFFEE7206808B9012000E00020B2
:10C1C00050B900BF502080F31188BFF34F8FBFF3E9
:10C1D0006F8F00BF00BFFEE70C4960680968084028
:10C1E00098B1206888B90949606809688843606027
:10C1F00000F0AAF806496068096808440449086024
:10C200002046FEF70BFE00F091FB70BDE00200201F
:10C21000D802002000204FF0E02108618861064824
:10C2200000684FF47A71B0FBF1F0401E4FF0E0214E
:10C2300048610720086170478C02002070B50446F1
:10C240000025D4B11248006808B9012000E00020A0
:10C2500050B900BF502080F31188BFF34F8FBFF358
:10C260006F8F00BF00BFFEE700F06EF80021204690
:10C27000FEF706FC00F05AFB05463DB94FF0805032
:10C2800004490860BFF34F8FBFF36F8F70BD00008C
:10C29000C802002004ED00E010B586B00020059033
:10C2A000049003AA04A905A8FFF7E0FE0022DDE937
:10C2B00004101346CDE9002102901CA11D48039AE9
:10C2C00000F034FA1C4908600846006808B10124EF
:10C2D00000E00024012C15D100BF502080F311880C
:10C2E000BFF34F8FBFF36F8F00BF4FF0FF30134985
:10C2F000086001201249086000201249086000F01F
:10C3000067F910E0601C08B1012000E0002050B97E
:10C3100000BF502080F31188BFF34F8FBFF36F8FA2
:10C3200000BF00BFFEE706B010BD000049444C4509
:10C3300000000000E1AC0008C4020020C0020020A0
:10C34000AC020020A402002002480068401C014901
:10C3500008607047C80200201D48006818B101201D
:10C360001C49086032E000201A4908601A48006839
:10C37000B0FA80F0C0F11F0101EB8100174A52F8BA
:10C38000200008B1012000E0002050B900BF50207B
:10C3900080F31188BFF34F8FBFF36F8F00BF00BFD3
:10C3A000FEE701EB81020D4B03EB8200426852680D
:10C3B000426000F108024368934202D14268526829
:10C3C00042604268D268064B1A6000BF70470000A6
:10C3D000C8020020B4020020A8020020483C00202F
:10C3E000900200200FB408B50120102338A20821C4
:10C3F00000900420FAF709FA01200C2335A2082145
:10C4000000900020FAF701FA0120122300220C21EB
:10C4100000903720FAF7E6F80120122302460C219B
:10C4200000904B20FAF7DEF8012012230222282187
:10C4300000903720FAF7D6F8012012230322282192
:10C4400000904B20FAF7CEF89DF80800042806D19A
:10C450000020009010231E21079AFAF7D6F99DF8C4
:10C460000800052806D10020009010231E210B9AF9
:10C47000FAF7CBF99DF80800062806D100200090B5
:10C4800010231E210F9AFAF7C0F99DF8080007281B
:10C4900006D10020009010231E21139AFAF7B5F957
:10C4A0009DF80900012808D1002010230CA20C21BE
:10C4B00000905D20FAF7A9F907E00020102308A2F8
:10C4C000282100905D20FAF7A0F901B05DF814FB77
:10C4D000534E3A004C4F434B4E414D453A000000FD
:10C4E0003C2D2D003048007800B970472E48007868
:10C4F000662857D12C484078012853D12A488078A3
:10C5000001284FD12848C07828490880264800795A
:10C5100027490870244840792649096841EA0060A3
:10C520002449086020488079096841EA004021498F
:10C5300008601D48C079096841EA00201D4908606B
:10C540001948007A096808431A4908601648407A71
:10C55000194908701448807A184908701248C07A3E
:10C56000174908701048007B164908700E48407B38
:10C570001549098841EA0020134908800A48807B50
:10C5800009880843104908800748C07B0F4909887B
:10C5900041EA00200D4908800348007C09880843CF
:10C5A0000A49088000BFA0E7DC0F0020300200200D
:10C5B000320200203402002038020020390200201C
:10C5C0003A0200203B0200203C0200203E020020F4
:10C5D0001CB53849084600780190FF200A461070C3
:10C5E0000846007800909DF8000000F0F0009DF8EB
:10C5F0000020904201D1012000E0002050B900BF8E
:10C60000502080F31188BFF34F8FBFF36F8F00BFAF
:10C6100000BFFEE79DF8000000F05000264A1070B1
:10C620000720264A106009E024480068401E234A7B
:10C6300010609DF800004006000E00909DF800007C
:10C6400000F080008028EFD01C480068C0F107008F
:10C65000042801D1012000E0002050B900BF502083
:10C6600080F31188BFF34F8FBFF36F8F00BF00BF00
:10C67000FEE7124800680002104A10601046008869
:10C6800000F4E06010600B4A019810700C480068DC
:10C6900040F470000A4908600846006840F07040A5
:10C6A0000860FFF7B7FD002006490860F3F75EFD5C
:10C6B00000201CBD00E400E0E8020020EC020020A5
:10C6C00020ED00E0E40200202DE9FF4F85B0804618
:10C6D00089461746DDE912ABB800FEF70DFC0646A9
:10C6E00056B15420FEF708FC04460CB1266304E062
:10C6F0003046FFF745FD00E000248CB1002084F8AF
:10C700005100CDE900ABCDE902403A4649464046EA
:10C71000089BFEF7F9FA2046FEF7FEF9012501E035
:10C720004FF0FF35284609B0BDE8F08F2DE9F04FF6
:10C7300085B00746884691469A46DDE90EB6109CBC
:10C740000EB1012000E0002050B900BF502080F35E
:10C750001188BFF34F8FBFF36F8F00BF00BFFEE79D
:10C760000CB1012000E0002050B900BF502080F340
:10C770001188BFF34F8FBFF36F8F00BF00BFFEE77D
:10C78000542003900398542801D1012000E0002098
:10C7900050B900BF502080F31188BFF34F8FBFF313
:10C7A0006F8F00BF00BFFEE7B4B1AEB125462C4687
:10C7B0002E63022085F85100002004A953464A4602
:10C7C000CDE900B1CDE9025041463846FEF79CFA6A
:10C7D0002846FEF7A1F901E000200490049805B076
:10C7E000BDE8F08F2DE9F0414FF0000844480068A3
:10C7F000002877D143480068451C4248056015BBB6
:10C8000041480068006808B9012000E0002050B9E4
:10C8100000BF502080F31188BFF34F8FBFF36F8F9D
:10C8200000BF00BFFEE7384807683848006836494F
:10C8300008603648076036480068401C3449086084
:10C84000FEF720FB00BF3348006885423CD300BFA1
:10C850002D480068006808B9012000E0002020B1E0
:10C860004FF0FF302B4908602DE027480068C06872
:10C87000C4686668B54202D22648066023E0201DDF
:10C88000FFF7E0FBA06A18B104F11800FFF7DAFB2C
:10C8900094F82C10012088401F49096808431E495C
:10C8A0000860E16A01EB81011C4A02EB8100211D55
:10C8B000FFF712FC1A49E06A0968C96A8842C7D3BF
:10C8C0004FF00108C4E700BF15480068C06A00EBDC
:10C8D0008000124951F82000012801D94FF00108C9
:10C8E00005E0FFE70F480068401C0E4908600E484D
:10C8F000006808B14FF001084046BDE8F081000033
:10C90000C8020020A4020020940200209802002007
:10C91000B8020020C0020020A8020020483C0020ED
:10C9200090020020B0020020B402002070B5002464
:10C9300000263648006850B900BF502080F31188A7
:10C94000BFF34F8FBFF36F8F00BF00BFFEE7FFF74E
:10C95000CFFB2E480068401E2C490860084600683E
:10C9600000284FD12A48006800284BD024E02948ED
:10C97000C068C46804F11800FFF764FB201DFFF7CE
:10C9800061FB94F82C100120884023490968084372
:10C9900021490860E16A01EB8101204A02EB810034
:10C9A000211DFFF799FB1E49E06A0968C96A8842A0
:10C9B00002D301201B4908601648006808B901200D
:10C9C00000E000200028D2D00CB1FEF75BFA164838
:10C9D000056865B100BFFFF705FF10B101201149DF
:10C9E00008606D1E002DF6D100200F4908600D482B
:10C9F000006838B1012630070C490860BFF34F8F3B
:10CA0000BFF36F8FFFF79EFB304670BDC80200205A
:10CA1000A0020020FC3C0020A8020020483C00208E
:10CA200090020020B4020020B002002004ED00E0DB
:10CA300010B502461378012002E0145C6340401CEC
:10CA40008842FADB184610BD0146C80900EBC00059
:10CA500000EB400080EA4100C0B2704700000000D7
:10CA600000000000002F0000000007000700001475
:10CA70007F147F1400242A7F2A1200626408132383
:10CA800000364955225000000503000000001C221A
:10CA90004100000041221C000014083E0814000858
:10CAA000083E0808000000A0600000080808080808
:10CAB000000060600000002010080402003E5149A0
:10CAC000453E0000427F400000426151494600213E
:10CAD00041454B31001814127F1000274545453958
:10CAE000003C4A49493000017109050300364949B3
:10CAF000493600064949291E00003636000000006C
:10CB000056360000000814224100001414141414B6
:10CB1000000041221408000201510906003249595F
:10CB2000513E007C1211127C007F49494936003E7B
:10CB300041414122007F4141221C007F4949494136
:10CB4000007F09090901003E4149497A007F080830
:10CB5000087F0000417F4100002040413F01007FED
:10CB600008142241007F40404040007F020C027FB9
:10CB7000007F0408107F003E4141413E007F0909CB
:10CB80000906003E4151215E007F091929460046F1
:10CB9000494949310001017F0101003F4040403FC8
:10CBA000001F2040201F003F4038403F0063140812
:10CBB00014630007087008070061514945430000ED
:10CBC0007F41410000552A552A55000041417F0010
:10CBD0000004020102040040404040400000010205
:10CBE0000400002054545478007F484444380038EE
:10CBF0004444442000384444487F00385454541876
:10CC000000087E0901020018A4A4A47C007F080487
:10CC100004780000447D4000004080847D00007F57
:10CC2000102844000000417F4000007C0418047874
:10CC3000007C0804047800384444443800FC242470
:10CC400024180018242418FC007C08040408004858
:10CC50005454542000043F444020003C4040207C79
:10CC6000001C2040201C003C4030403C0044281068
:10CC70002844001CA0A0A07C004464544C4414141C
:10CC80001414141400000000000000000000000054
:10CC90000000FC000000000002000000000C020C7C
:10CCA000020000000000000090D0BCD0BC90000347
:10CCB000000300001824FE448C0003020702010058
:10CCC0001824D8B04C80000300010201C038E438B9
:10CCD000E00001020201020208060000000000005C
:10CCE00000000000000000F804020000000102043F
:10CCF000000204F800000004020100009060F860E7
:10CD000090000000010000002020FC202000000016
:10CD10000100000000000000000008060000000004
:10CD20002020202020000000000000000000000063
:10CD300000000002000000000080601C02000403EC
:10CD400000000000F8040404F800010202020100DF
:10CD50000008FC00000000020302000018844424C4
:10CD6000180003020202020008042424D800010271
:10CD70000202010040B088FC8000000000030200B5
:10CD80003C242424C400010202020100F824242CC3
:10CD9000C0000102020201000C04E41C04000000B7
:10CDA00003000000D8242424D8000102020201005C
:10CDB00038444444F800000302020100000010005F
:10CDC0000000000002000000000020000000000041
:10CDD000060000000020508804020000000001024C
:10CDE00090909090900000000000000000020488E5
:10CDF00050200002010000001804C42418000000A4
:10CE000002000000F804E494F800010202020200AB
:10CE100000E09CF0800002030000030204FC2424D4
:10CE2000D800020302020100F80404040C0001020D
:10CE30000202010004FC0404F800020302020100E3
:10CE400004FC24740C0002030202030004FC24749A
:10CE50000C00020302000000F0080444CC40000172
:10CE60000202010004FC2020FC0402030000030273
:10CE70000404FC040400020203020200000404FC97
:10CE8000040406040403000004FC24D00C04020380
:10CE90000200030204FC0400000002030202020379
:10CEA000FC3CC03CFC0003000300030004FC30C455
:10CEB000FC04020302000300F8040404F800010269
:10CEC0000202010004FC24241800020302000000F6
:10CED000F8848404F80001020207050004FC2464BD
:10CEE0009800020302000302182424448C00030269
:10CEF000020201000C04FC040C000002030200000A
:10CF000004FC0000FC04000102020100047C80E03B
:10CF10001C040000030000001CE03CE01C000003B7
:10CF200000030000049C609C040002030003020054
:10CF3000041CE01C04000002030200000C84641CBA
:10CF400004000203020203000000FE0202000000CF
:10CF500007040400000E30C00000000000010200C1
:10CF6000000202FE000000040407000000040204A6
:10CF700000000000000000000000000000000808A1
:10CF8000080808080000020000000000000000007F
:10CF90000040A0A0C00000010202030204FC202007
:10CFA000C00000030202010000C020206000000158
:10CFB0000202020000C02024FC0000010202030261
:10CFC00000C0A0A0C0000001020202000020F8245E
:10CFD00024040002030202000040A0A06020000719
:10CFE0000A0A0A0404FC2020C00002030200030213
:10CFF0000020E4000000000203020000000020E422
:10D00000000008080807000004FC80E0202002035C
:10D01000020003020404FC000000020203020200FA
:10D02000E020E020C00003000300030020E02020F7
:10D03000C00002030200030200C02020C000000163
:10D040000202010020E02020C000080F0A020100B7
:10D0500000C02020E0000001020A0F0820E040206C
:10D0600020000203020000000060A0A020000002D7
:10D07000020203000020F82000000000010202006C
:10D0800020E00020E00000010202030220E02080F6
:10D0900060200000030100006080E0806000000369
:10D0A00000030000206080602000020300030200F3
:10D0B00020E0208060200808070100000020A06018
:10D0C0002000000203020200000020DE0200000037
:10D0D00000070400000000FF00000000000F000037
:10D0E0000002DE200000000407000000020102042C
:10D0F000040200000000000000000000000000002A
:10D100000000000000000000000000F80000000027
:10D11000000000333000000000100C06100C060068
:10D12000000000000000000040C07840C0784000CF
:10D13000043F04043F040400007088FC0830000031
:10D14000001820FF211E0000F008F000E018000089
:10D1500000211C031E211E0000F008887000000042
:10D160001E2123241927211010160E000000000094
:10D170000000000000000000000000E018040200B1
:10D18000000000071820400000020418E000000022
:10D190000040201807000000404080F08040400020
:10D1A0000202010F01020200000000F00000000076
:10D1B0000101011F0101010000000000000000004A
:10D1C00080B07000000000000000000000000000BF
:10D1D0000001010101010101000000000000000048
:10D1E00000303000000000000000000080601804E3
:10D1F000006018060100000000E010080810E000C0
:10D20000000F102020100F00001010F80000000088
:10D210000020203F202000000070080808887000CF
:10D22000003028242221300000300888884830004F
:10D230000018202020110E000000C02010F800006F
:10D2400000070424243F240000F808888808080008
:10D250000019212020110E0000E01088881800001D
:10D26000000F112020110E0000380808C8380800EF
:10D270000000003F0000000000708808088870006F
:10D28000001C222121221C0000E010080810E000F0
:10D290000000312222110F00000000C0C000000079
:10D2A000000000303000000000000080000000009E
:10D2B0000000806000000000000080402010080096
:10D2C000000102040810200040404040404040005F
:10D2D000040404040404040000081020408000003A
:10D2E0000020100804020100007048080808F0003F
:10D2F0000000003036010000C030C828E810E0000F
:10D300000718272423140B000000C038E000000099
:10D31000203C23020227382008F888888870000003
:10D32000203F202020110E00C030080808083800D7
:10D33000071820202010080008F808080810E0004E
:10D34000203F202020100F0008F88888E8081000EF
:10D35000203F20202320180008F88888E8081000C3
:10D36000203F200003000000C030080808380000FB
:10D3700007182020221E020008F808000008F808FC
:10D38000203F210101213F20000808F80808000083
:10D390000020203F2020000000000808F8080800B6
:10D3A000C08080807F00000008F888C0281808002E
:10D3B000203F20012638200008F808000000000067
:10D3C000203F20202020300008F8F800F8F808005E
:10D3D000203F003F003F200008F830C00008F80858
:10D3E000203F200007183F00E01008080810E00068
:10D3F0000F10202020100F0008F808080808F0007F
:10D40000203F210101010000E01008080810E000A1
:10D410000F18242438504F0008F888888888700036
:10D42000203F2000030C30200070880808083800D6
:10D430000038202121221C00180808F808081800CC
:10D440000000203F2000000008F808000008F8084D
:10D45000001F202020201F000878880000C83808FE
:10D46000000007380E010000F80800F80008F80076
:10D47000033C0700073C0300081868808068180810
:10D4800020302C03032C30200838C800C83808008E
:10D490000000203F2000000010080808C8380800DD
:10D4A0002038262120201800000000FE0202020081
:10D4B0000000007F40404000000C30C00000000031
:10D4C000000000010638C00000020202FE00000059
:10D4D000004040407F0000000000040202020400FF
:10D4E000000000000000000000000000000000003C
:10D4F0008080808080808080000202040000000024
:10D50000000000000000000000008080808000001B
:10D510000019242222223F2008F800808000000009
:10D52000003F112020110E000000008080800000CC
:10D53000000E112020201100000000808088F800DB
:10D54000000E112020103F2000008080808000000D
:10D55000001F222222221300008080F08888881871
:10D560000020203F2020000000008080808080007C
:10D57000006B94949493600008F800808080000011
:10D58000203F210000203F200080989800000000EC
:10D590000020203F2020000000000080989800001C
:10D5A00000C08080807F000008F80000808080003C
:10D5B000203F24022D302000000808F80000000061
:10D5C0000020203F2020000080808080808080001C
:10D5D000203F20003F20003F8080008080800000AE
:10D5E000203F210000203F2000008080808000003C
:10D5F000001F202020201F0080800080800000006D
:10D6000080FFA12020110E0000000080808080009B
:10D61000000E112020A0FF8080808000808080008C
:10D6200020203F21200001000000808080808000B9
:10D630000033242424241900008080E0808000002E
:10D640000000001F2020000080800000008080007B
:10D65000001F202020103F208080800000808080DC
:10D6600000010E300806010080800080008080806C
:10D670000F300C030C300F00008080008080800091
:10D680000020312E0E3120008080800000808080BC
:10D6900080818E701806010000808080808080006C
:10D6A0000021302C2221300000000000807C02028A
:10D6B00000000000003F404000000000FF000000AC
:10D6C00000000000FF0000000002027C800000005B
:10D6D0000040403F00000000000601010202040477
:10D6E000000000000000000000000000000000003A
:10D6F000000000000000000000000000000000002A
:10D700000000000000000000000000000000000019
:10D7100000F0F0F0000000000000000000017F01B8
:10D720000000000000000000001C1C1C00000000A5
:10D7300000008060301C8C60301C0C000000000079
:10D7400000000000000000000000000000000000D9
:10D7500000000000000000E00000000000E0000009
:10D760000086E69F86868686E69F860000011F016A
:10D77000010101011F010100000080C06020F820AC
:10D78000E0C00000000003070C18FF70E1810000FA
:10D790000000070F10107F100F070000806020604E
:10D7A00080000000E02000000F3020309F70DC3748
:10D7B0001030C0000000100E0300071810180700FA
:10D7C0000000C02020E0C0000000000080E01F3802
:10D7D000E88703C43C040000070F1810100B070D66
:10D7E0001010080000808C4C380000000000000081
:10D7F0000000000000000000000000000000000029
:10D80000000000000000000000000000000080E0B8
:10D81000300804000000000000FEFF0100000000CE
:10D82000000000000000030F182040000004083032
:10D83000E0800000000000000000000001FFFE008A
:10D8400000000000004020180F030000000000004E
:10D85000000000000000C0000000000000426666FA
:10D860003C18FF183C666642000000000000030000
:10D870000000000000000000000080000000000028
:10D88000001010101010FF101010101000000000F9
:10D890000000030000000000000000000000000085
:10D8A0000000000000000000000000000000000078
:10D8B00000808C4C380000000000000000000000D8
:10D8C00000000000000000000010101010101010E8
:10D8D0001010100000000000000000000000000018
:10D8E0000000000000000000000000000000000038
:10D8F000000000000000000000001C1C1C000000D4
:10D90000000000000000000000000000E0380C00F3
:10D910000000000080701C03000000000060380E52
:10D920000100000000000000000080C060202060B6
:10D93000C080000000FEFF010000000001FFFE00AB
:10D940000001070E181010180E070100000080805B
:10D9500080C0E000000000000000000000FFFF00A9
:10D960000000000000001010101F1F101010000019
:10D970000080402020202060C080000000030300C1
:10D98000804020381F070000001C1A1918181818AA
:10D99000181F00000080C020202060C08000000010
:10D9A000000303001010182FE780000000070F107D
:10D9B000101010180F070000000000000000C0E069
:10D9C000F000000000C0B088868180FFFF808000EA
:10D9D000000000000010101F1F1010000000E06089
:10D9E000606060606060000000003F100808081878
:10D9F000F0E0000000070B101010101C0F030000D7
:10DA0000000080C040202020E0C0000000FCFF217A
:10DA10001008080818F0E0000001070C181010109A
:10DA2000080F03000000C0E06060606060E060001C
:10DA3000000003000000E0180700000000000000E4
:10DA4000001F1F00000000000080C0602020202078
:10DA500060C080000087EF2C1818303068CF83003A
:10DA600000070F0810101010180F07000000C0C0AA
:10DA700020202020C0800000001F3F604040402048
:10DA800010FFFE0000000C1C101010080F03000017
:10DA90000000000000000000000000000000000086
:10DAA000000E0E0E0000000000000000001C1C1CF8
:10DAB0000000000000000000000000000000000066
:10DAC00000000000000C0C0000000000000000003E
:10DAD0000058380000000000000000000000008036
:10DAE00040201000000010284482010000000000C7
:10DAF0000000000000000102040810000000000007
:10DB00000000000000000000008484848484848479
:10DB10008484840000000000000000000000000079
:10DB20000000102040800000000000000000000005
:10DB300000000182442810000000100804020100C7
:10DB40000000000000C020201010101030E0C000C5
:10DB50000003030000F010080C07030000000000A1
:10DB60001C1C1C0000000000000000C040602020C1
:10DB70002040C00000FCFF01F00E03C1FE03807FC7
:10DB80000001070E08111110110904020000000025
:10DB900080E0E000000000000000807C4340477F00
:10DBA000F880000010181F1000000000131F1C1048
:10DBB00020E0E02020202060C080000000FFFF1057
:10DBC000101010182FE78000101F1F1010101010D9
:10DBD000180F0700000080C0402020202060E000D7
:10DBE00000FCFF0100000000000001000001070E22
:10DBF000181010100804030020E0E020202020402E
:10DC0000C080000000FFFF000000000001FFFE00D8
:10DC1000101F1F10101018080E07010020E0E02050
:10DC2000202020202060800000FFFF101010107CBA
:10DC300000000000101F1F10101010101018060018
:10DC400020E0E020202020206060800000FFFF1006
:10DC50001010107C00000100101F1F1000000000B9
:10DC600000000000000080C06020202040E0000094
:10DC700000FCFF0100004040C0C140400001070E11
:10DC8000181010100F0F000020E0E020000000002E
:10DC900020E0E02000FFFF101010101010FFFF0028
:10DCA000101F1F1000000000101F1F100000202078
:10DCB00020E0E020202000000000000000FFFF0026
:10DCC0000000000000001010101F1F1010100000B6
:10DCD00000000000202020E0E020202000000000C4
:10DCE000000000FFFF0000000060E0808080C07F37
:10DCF0003F00000020E0E020000020A06020200085
:10DD000000FFFF30187CE3C000000000101F1F1050
:10DD1000000001131F1C181020E0E020000000008C
:10DD20000000000000FFFF000000000000000000F5
:10DD3000101F1F10101010101018060020E0E0E057
:10DD400000000000E0E0E02000FF013FFEC0E01E18
:10DD500001FFFF00101F1000031F0300101F1F1002
:10DD600020E0E0C0000000000020E02000FF0003F1
:10DD7000071C78E08000FF00101F1000000000006A
:10DD8000030F1F00000080C060202060C0800000E2
:10DD900000FEFF010000000000FFFE000001070E72
:10DDA000181010180C07010020E0E020202020208F
:10DDB00060C0800000FFFF2020202020301F0F00C7
:10DDC000101F1F100000000000000000000080C0B5
:10DDD00060202060C080000000FEFF010000000005
:10DDE00000FFFE000001070E1111133C7C672100AB
:10DDF00020E0E0202020202060C0800000FFFF10F5
:10DE00001030F0D0080F0700101F1F100000000393
:10DE10000F1C10100080C060202020204040E00037
:10DE200000070F0C1818303060E08100001F0C084C
:10DE300010101010180F07008060202020E0E02054
:10DE4000202060800100000000FFFF0000000001B2
:10DE500000000000101F1F100000000020E0E02064
:10DE6000000000000020E02000FFFF000000000094
:10DE70000000FF0000070F18101010101008070016
:10DE80002060E0E02000000020E060200000077F2C
:10DE9000F88000807C03000000000000071F1C07C2
:10DEA0000000000020E0E02000E0E0200020E02072
:10DEB0000007FFF8E01FFFFCE01F00000000031F49
:10DEC0000300011F03000000002060E0A00000200C
:10DED000E0602000000000038F7CF8C60100000015
:10DEE0000010181E130001171F1810002060E0E03A
:10DEF0002000000020E06020000001073EF8E0184C
:10DF00000700000000000010101F1F10100000008C
:10DF100000806020202020A0E0E020000000000021
:10DF2000C0F03E0F0300000000101C1F171010105F
:10DF3000101806000000000000FC040404040400A3
:10DF40000000000000FF00000000000000000000D2
:10DF5000007F404040404000000010E00000000012
:10DF60000000000000000000031C608000000000B2
:10DF700000000000000000030C708000000004049A
:10DF8000040404FC0000000000000000000000FF8A
:10DF900000000000000040404040407F00000000C2
:10DFA00000000010080C040C081000000000000025
:10DFB0000000000000000000000000000000000061
:10DFC0000000000000000000000000000000000051
:10DFD0000000000000000000000000008080808041
:10DFE0008080808080808080000000040408080019
:10DFF0000000000000000000000000000000000021
:10E000000000000000000000000000000000000010
:10E010000000000000000000000098D844642424A0
:10E02000FCF80000000F1F18101010081F1F101818
:10E030000020E0F000000000000000000000FFFFF2
:10E04000180804040CF8F00000001F0F181010103E
:10E05000180F030000000000000000000000000096
:10E0600000E0F8180404043C3800000000030F0C22
:10E070001010101008060000000000000000002032
:10E08000E0F0000000E0F81C04040408FFFF0000BA
:10E0900000030F18101010081F0F080000000000E8
:10E0A00000000000000000000000E0F84844444484
:10E0B0004C7870000000030F0C18101010080400BA
:10E0C0000000000080C0602020E0C00000040404C4
:10E0D000FFFF040404040000000010101F1F1010B4
:10E0E0001000000000000000000000000000000020
:10E0F000000070F88C04048CF874040C007076CF67
:10E100008D8D8D89C87870000020E0F0000000003F
:10E11000000000000000FFFF08040404FCF80000F9
:10E1200000101F1F100000101F1F10000000000033
:10E1300000606000000000000000040404FCFC001B
:10E140000000000000001010101F1F101010000031
:10E1500000000000000000606000000000000000FF
:10E16000040404FCFC0000000000C0C08080C07FEC
:10E170003F0000000020E0F0000000000000000070
:10E180000000FFFF80C0F41C0404000000101F1FEB
:10E190001100031F1C1010000000202020E0F000E0
:10E1A000000000000000000000FFFF000000000071
:10E1B00000001010101F1F101010000000000000C1
:10E1C000000000000000000004FCFC0804FCFC0847
:10E1D00004FCFC00101F1F10001F1F10001F1F1049
:10E1E0000000000000000000000000000004FCFC33
:10E1F00008080404FCF8000000101F1F10000010A5
:10E200001F1F1000000000000000000000000000C0
:10E2100000E0F0180C04040C18F0E00000030F0CF0
:10E22000101010100C0F0300000000000000000090
:10E23000000000000004FCFC080404040CF8F000DA
:10E240000080FFFF889010101C0F030000000000EA
:10E25000000000000000000000E0F81C04040408B6
:10E26000F8FC000000030F1810109088FFFF8000DA
:10E27000000000000000000000000000040404FC96
:10E28000FC100804040C0C001010101F1F101010BC
:10E29000000000000000000000000000000000007E
:10E2A00000003078CCC48484840C1C0000001E184C
:10E2B00010101011190F06000000000000C000002F
:10E2C0000000000000040404FFFF04040400000038
:10E2D000000000000F1F1010100C000000000000D4
:10E2E00000000000000000000004FCFE000000042C
:10E2F000FCFE000000000F1F181010081F0F080080
:10E3000000000000000000000000000000040C3CC1
:10E31000FCC40000C43C0C0400000000010F1E0EF1
:10E3200001000000000000000000000000000000EC
:10E33000043CFCC400E47CFC84807C040000071FD7
:10E34000070000071F070000000000000000000099
:10E35000000000000004041C7CE4C0341C04040021
:10E360000010101C1601131F1C18100000000000E4
:10E37000000000000000000000040C3CFCC400C4CD
:10E380003C0404000000C080C1370E010000000002
:10E3900000000000000000000000000000001C045D
:10E3A00004C4F47C1C0400000000101C1F17111092
:10E3B00010180E0000000000000000F80C0400001F
:10E3C00000000000001028EF000000000000000026
:10E3D0000000003F60400000000000000000FF005F
:10E3E00000000000000000000000FF00000000002E
:10E3F000000000000000FF00000000000000040C0E
:10E40000F80000000000000000000000EF281000ED
:10E4100000000000000040603F000000000000001D
:10E420000018060202040810202030080000000036
:10E4300000000000000000000000000000000000DC
:10E44000000000000000F010101010FF101010105D
:10E45000F000000000000F04040404FF040404049E
:10E460000F0000004040405F555555755555555FAC
:10E47000404040000040200F094989790909090FEF
:10E480002040000000FE02424ACA4A4ACA4A4A42A2
:10E4900002FE000000FF40504C4340404F50505C93
:10E4A00040FF00000000F888888888FF88888888F6
:10E4B000F800000000001F080808087F8888888886
:10E4C0009F80F00080828282828282E2A2928A868B
:10E4D00082808000000000000040807F000000007B
:10E4E00000000000101010FF109008888888FF8836
:10E4F000888808000444827F01808040432C1028D3
:10E50000468180000010101010D030FF30D0121C57
:10E510001010000010080402010000FF00000102BA
:10E520000408100004040484E43C2724242424E484
:10E530000404040004020100FF0909090949897F54
:10E540000000000000FE225A8600FE9292929292F3
:10E55000FE00000000FF04080700FF4020030C1429
:10E56000224140000080402018068000071820400B
:10E57000800000000100207028262120202438601F
:10E5800000010100001012929292929292121202D5
:10E59000FE0000000000003F101010103F004080FF
:10E5A0007F00000080828282FE8282828282FE82DE
:10E5B00082828000008040300F0000000000FF00D9
:10E5C0000000000000001011161010F010101413BD
:10E5D000100000008181414121110D030D112141E5
:10E5E000418181000008488808C83800901010FF59
:10E5F000101010000020100C030418000043807F4E
:10E600000000000020102CE7242400E22C20BF2072
:10E6100028E600000101017F2111804F20100F101A
:10E62000204F8000008060F80740300FF88888880D
:10E6300088080800010000FF00000000FF0808082B
:10E64000080800000010608000FF000000FF0000CC
:10E65000C030000040404043407F4040407F424146
:10E66000404040001010F196909010E80784FC8420
:10E6700044C4040080601F40807F013F41405F44EC
:10E68000484778002010EC27F42CE00022920ED2AC
:10E69000221E000080601F093F89FF000A0909FF50
:10E6A00009090800404848487F4848480090101031
:10E6B000FF10100040C444443F2424240000438041
:10E6C0007F000000404042CC0040A09E8282829E9B
:10E6D000A02020000000003F908840432C102846D6
:10E6E00041808000809090484C57242424544C440E
:10E6F00080808000000000FF4949497F494949FF67
:10E70000000000001010FF1090E02F29E909E9290E
:10E710002FE0000042827F414425150D05FE0D15B6
:10E7200025454400008060F80740300FF88888884D
:10E7300088080800010000FF00000000FF0808082A
:10E7400008080000404424A4948C84FF848C94A482
:10E75000244440004040405F4A4A4A4A4A4A4A5F8D
:10E760004040400020222A2AAA6A3A2E2929292933
:10E770002920200008040201FF555555555555FF25
:10E780000000000000083000FF20202020FF202093
:10E79000222C200004040201FF8040300E010618E4
:10E7A00020408000000484844424548F1424448432
:10E7B00084040000413900003C4040424C4040701D
:10E7C000040931002038E730004848FF484800FE7F
:10E7D00042B20E00222712120082621F020200FFC4
:10E7E00008100F00100C4444444445C644444444BB
:10E7F00044140C008040201E2040407F4444444488
:10E8000044404000000000FC444444454644444425
:10E81000447C00004020180700FC44444444444425
:10E8200044FC00004044C4444444401010FF101015
:10E8300010F00000103C131014B840300E0140805E
:10E84000403F000080808888888888FF8888888882
:10E850008880800020201008040201FF01020408C3
:10E86000102020002038E730004848FF484800FECC
:10E8700042B20E00222712120082621F020200FF23
:10E8800008100F00100C4444444445C6444444441A
:10E8900044140C008040201E2040407F44444444E7
:10E8A000444040001060028C00445454547F54543F
:10E8B0005444400004047E010000FF1515155595D1
:10E8C0007F000000100C44241404050604041424E2
:10E8D00044140C00004040414141417F41414141CD
:10E8E000404000002038E730004848FF484800FE1C
:10E8F00042B20E00222712120082621F020200FFA3
:10E9000008100F00100C4444444445C64444444499
:10E9100044140C008040201E2040407F4444444466
:10E9200044404000008060F8070004242425262489
:10E9300024240400010000FF000000F9494949496E
:10E9400049F90000000000FC54545655545454FC3E
:10E9500000000000403000033941414559414173F6
:10E9600000083000000000C080808080808080FC33
:10E9700084808080808080C0C0000000000000FF94
:10E980007F404040404040FF40404040404040FFCA
:10E990007F00000000000000000000000000007F79
:10E9A00070000000000000000000000000000000F7
:10E9B0000000000000000000000000FCF800000063
:10E9C0000000000000000000000000000000000047
:10E9D000FFFE020202020202020202FFFF02020224
:10E9E000020202020202FF03000000000000000019
:10E9F0001F1F040404040404040404FFFF040404AB
:10EA00000404040404041F000000000000000000CF
:10EA100000000000000000000000007F3F00000038
:10EA200000000000000000000000000000000000E6
:10EA300000000000000000000000000000000000D6
:10EA4000000000000000000000F8F8F0F070200066
:10EA500000000000000000000000000000000000B6
:10EA600000000000000000000000000000000000A6
:10EA70000000000080000000000000000000000016
:10EA8000000000000000000000FFFFFFFF0000008A
:10EA90000000000000000000000000000000000076
:10EAA0008080000000000000000000000000000066
:10EAB0000000000000FFFFFE06060606060606062A
:10EAC000060606060606060606FFFFFFFF06060602
:10EAD000060606060606060606060606060606FFDD
:10EAE000FFFFFF0702000000000000000000000020
:10EAF0000000000000FFFFFF000000000000000019
:10EB0000000000000000000000FFFFFFFF00000009
:10EB1000000000000000000000000000000000FFF6
:10EB2000FFFFFF00000000000000000000000000E8
:10EB30000000000000FFFFFF181818181818181818
:10EB4000181818181818181818FFFFFFFF181818A9
:10EB5000181818181818181818181818181818FF4E
:10EB6000FFFFFF00000000000000000000000000A8
:10EB70000000000002010100000000000000000091
:10EB8000000000000000000000FFFFFFFF00000089
:10EB90000000000000000000000000000000000174
:10EBA0000100000000000000000000000000000064
:10EBB0000000000000000000000000000000000055
:10EBC000000000000000000000FFFFFFFF00000049
:10EBD0000000000000000000000000000000000035
:10EBE0000000000000000000000000000000000025
:10EBF0000000000000000000000000000000000015
:10EC00000000000000000000001F1F0F0F000000A8
:10EC100000000000000000000000000000000000F4
:10EC200000000000000000000000000042F22EE2A0
:10EC300000F453F25A56F0000007020708070107D4
:10EC400001090F001011F2000000C03FC0000000D9
:10EC50000000070209060100010608001011F20079
:10EC6000FE0A2A4A894939000804030609080A09E4
:10EC700008090A0000FE0202F29292F20202FE006D
:10EC8000000F04040404040404040F0094F392002D
:10EC9000F21410DF1014F200000F0408090402013E
:10ECA0000204090000001010F800000000004040BD
:10ECB0007F40000000000000000000000070080815
:10ECC0000810E0000060584442417000000000005D
:10ECD000000000000030080808F0600000304041EB
:10ECE00041221C00000000000000000000008040E5
:10ECF00030F8000000060948487F4000000000008E
:10ED00000000000004FD26E444F342FE2212F2005B
:10ED10000807080F0007080B08090D00202424BF6E
:10ED20002424488808FF0800080909070505000988
:10ED3000080F000008F453FA56F0896741E94F00C4
:10ED400008070107090F0002020F02000202020277
:10ED5000FE02122242820200000000000F000000AA
:10ED600000010000404040404040404040404000E2
:10ED700000000000000000000000000010FC03087C
:10ED80006888090A08E80800000F0008080B080C4A
:10ED90000B080800DCB30880FE2AEA2BEA2AEE0002
:10EDA000040402000F01070107090F00645CF74427
:10EDB00010F7555555F7100002020F01040705051D
:10EDC000050F0200FC242424FF242424FC0000005E
:10EDD000030101010709090909080E008868FF28D5
:10EDE00040FE0202FE00000000000F0804030000C5
:10EDF00007080E00001F25E525252525E5273000FD
:10EE000001090503010101010F0101000C04755600
:10EE100054D7545675040C0000070101010F01017D
:10EE20000507000021E20004342C27F42424040008
:10EE3000080708090909090F090909008888FF4816
:10EE4000A4ACB5E6B4ACA40000080F00080A0B049B
:10EE5000040B080000FC2424E404FF04856604007D
:10EE6000080700020B04020102040F000404FC0462
:10EE70000408FF080808F800020201090503000061
:10EE80000808070000244484641C00488808FF0820
:10EE9000080010080601030C000021203F000000BC
:10EEA0001028E7242400F21410DF1014F2000101EE
:10EEB0003F11092027100807081027004020F807F5
:10EEC000201807FC44444444040000003F000000B4
:10EED000003F0404040404000830C000FF000000E8
:10EEE000FF00C0380000202021203F2020203F21AB
:10EEF000202020002021E60040A09E8282829EA049
:10EF0000200000001F0824201314081412212000E0
:10EF1000002FA9A9AFA9F9A9AFA9A92F0000202006
:10EF20003F2020203C2020203F2020004444A49467
:10EF30008C84BF848C94A444440020202F2A2A2A45
:10EF40002A2A2A2A2F20200020222AAAEABAAEAA98
:10EF5000A9A9A92120000402013F2A2A2A2A2A2A33
:10EF60003F000000041880FF001010907F901214E2
:10EF700010000201003F20100C0300030C102000C1
:10EF80008484444424548F142444448484002018EA
:10EF9000001C2020222C2030000418004042CC000D
:10EFA0008888FF888888FF88880020100F10202814
:10EFB000272020202F2020008844E2190020222230
:10EFC00022E22222200000003F0000000020203F1B
:10EFD0000000000008F8494AC81008E784FC44E42F
:10EFE0000400201F00203F00011F202F242738008D
:10EFF00008F493FA96F000D28EE2929E0000201F51
:10F00000041F243F0504043F04040400202424BFFB
:10F01000242400488808FF0808001011110F09096E
:10F02000000021203F0000004048C4A6AB9292920D
:10F03000AAA6C240400000003F2424243F242424E8
:10F040003F00000090DCB3980424FF2400FE02621D
:10F050009E000808040421110F01003F0808070062
:10F060000C0424242425E624242424040C00201049
:10F070000F1020203F22222222202000404141FF69
:10F080004141414141FF4141400020100C0300003B
:10F090000000003F00000000808888898E88F88882
:10F0A0008C8B88888000202010080403000304084B
:10F0B000102020000808FF880070577505755770EC
:10F0C000000021213F0012120A063F060A12120018
:10F0D0004020F807201807FC444444440400000082
:10F0E0003F000000003F040404040400000008F195
:10F0F0008E88884828D80FF02888888808000080E3
:10F10000704F80807F0202FF81BF81889C83E00076
:10F1100000000000000000000000000000000000EF
:10F1200000000000888888FF888880A0202020FFB9
:10F130002020200000C04444447F44242420018E29
:10F1400080FF000000000000000000000000000040
:10F1500000000001000000000040F02C27F42CE02B
:10F160006040E29CC262223E000000807F05057F75
:10F1700005FF080A0909FF09090908000000000045
:10F18000000000010000000001000000000000007D
:10F19000888888FF888880A0202020FF20202000E9
:10F1A00000C04444447F44242420018E80FF00009A
:10F1B000000000000000000000000000000000014E
:10F1C00000000000000010FF1090E0203EEA0A0A54
:10F1D000F22E20E00000008282FF01804745351BAF
:10F1E000FE0A172545C74400000000010100000089
:10F1F0000000010000000000000000008060FC032F
:10F2000040201C0FF08888888888000000010000DA
:10F21000FF0000000000FF080808080800000000C8
:10F2200000000100000000000100000000000000DC
:10F23000000000F010101010101EFA10121CD090D8
:10F2400000000080601F2121413F8080433C3866E0
:10F25000C180E0000001000000000001000000008B
:10F260000000000001000000080808F0080808205D
:10F2700020FF202020E0000000003010100F088840
:10F2800040201C038080807F0000000000000001FF
:10F29000010000000000000101000000000000F873
:10F2A00088888888FF88888888F80800000000001F
:10F2B000000F04040404FF848484848F80E08000B1
:10F2C000000000000000000000000000000000003E
:10F2D0000000000010D0FF90100000FC020202FEAF
:10F2E0000000000000180601FF0081631C030000FD
:10F2F00000FF8080E000000000000101000000002D
:10F30000000000000000000000000000FE92929249
:10F3100092929292929EE080000000000888886895
:10F320001E08080808FE0A0808080000000001007E
:10F3300000000000000000010000000000000020AC
:10F34000300809EA2C282F29282CEA082818000060
:10F350000000000078070505FE050505457C040052
:10F36000000000000000000000000100000000009C
:10F370000000000000000000F888888C8B888888D6
:10F3800088F80800000000000000FF48484848488E
:10F39000484848FF00000000000000000100000095
:10F3A00000000000000100000000000010E0FF90DD
:10F3B0009050209887868890206000000008060101
:10F3C000FF000384B8808698C0B986808000000062
:10F3D000000001000000000000000000000000002C
:10F3E00098F60008056B000803000000000000000C
:10F3F00080000000000000000000000074F600081B
:10F40000FB6A00080300000000000000800000000C
:10F4100000000000000000008CF600083D6B0008B2
:10F420000300000000000000800000000000000059
:10F430000000000080F600086D6D00080300000069
:10F44000000000008000000000000000000000003C
:10F45000637C777BF26B6FC53001672BFED7AB7691
:10F46000CA82C97DFA5947F0ADD4A2AF9CA472C03C
:10F47000B7FD9326363FF7CC34A5E5F171D83115A9
:10F4800004C723C31896059A071280E2EB27B275CA
:10F4900009832C1A1B6E5AA0523BD6B329E32F8442
:10F4A00053D100ED20FCB15B6ACBBE394A4C58CF3A
:10F4B000D0EFAAFB434D338545F9027F503C9FA80E
:10F4C00051A3408F929D38F5BCB6DA2110FFF3D2DC
:10F4D000CD0C13EC5F974417C4A77E3D645D197390
:10F4E00060814FDC222A908846EEB814DE5E0BDB8A
:10F4F000E0323A0A4906245CC2D3AC629195E479C1
:10F50000E7C8376D8DD54EA96C56F4EA657AAE081A
:10F51000BA78252E1CA6B4C6E8DD741F4BBD8B8AB5
:10F52000703EB5664803F60E613557B986C11D9E1B
:10F53000E1F8981169D98E949B1E87E9CE5528DF92
:10F540008CA1890DBFE6426841992D0FB054BB16BE
:10F5500052096AD53036A538BF40A39E81F3D7FB48
:10F560007CE339829B2FFF87348E4344C4DEE9CB92
:10F57000547B9432A6C2233DEE4C950B42FAC34E07
:10F58000082EA16628D924B2765BA2496D8BD125BD
:10F5900072F8F66486689816D4A45CCC5D65B69261
:10F5A0006C704850FDEDB9DA5E154657A78D9D8405
:10F5B00090D8AB008CBCD30AF7E45805B8B3450625
:10F5C000D02C1E8FCA3F0F02C1AFBD0301138A6B3F
:10F5D0003A9111414F67DCEA97F2CFCEF0B4E6736F
:10F5E00096AC7422E7AD3585E2F937E81C75DF6E1D
:10F5F00047F11A711D29C5896FB7620EAA18BE1B83
:10F60000FC563E4BC6D279209ADBC0FE78CD5AF428
:10F610001FDDA8338807C731B11210592780EC5F6E
:10F6200060517FA919B54A0D2DE57A9F93C99CEFCA
:10F63000A0E03B4DAE2AF5B0C8EBBB3C83539961CB
:10F64000172B047EBA77D626E169146355210C7D09
:10F650008D01020408102040801B360000000000CD
:10F660000000000102030406070809000000000171
:10F6700002030400425434475461736B00000000DD
:10F680006C6F67696E666F5461736B007465737439
:10F690005461736B000000005363616E4B657954D5
:10F6A00061736B00C4F6000800000020F402000043
:10F6B000F0020008B0F70008F4020020444A0000FD
:10F6C000CC7800084A80012DFCFEFF870147070720
:10F6D0001F1E1CFF3718E42222F408390E113B07C5
:10F6E00008013B090907620F39384939580887FF73
:10F6F000FFFEFC80802E116738E44040E43C5AFF56
:10F700003C193D593F0C1908080778E8080222F413
:10F71000C8E0E0E0782A0F0189784CFEFF8F78AAD4
:10F72000FE782A3C783B38C001C978393F770F070B
:10F730006E756C6C5D3130313001AA310DAA320D1D
:10F74000AA330DAA340DAA350DAA360DAA370DAA73
:10F75000380DAA390DAA410DAA420DAA430DAA449B
:10F760000DAA450D9A460D233130100A20574152FB
:10F770004E494E4720133C3CA33E3E00114B2B43C9
:10F780004F4E4E4543542054494D454F5554D81281
:10F790004A49414C4F4E475F324038213523393278
:10F7A0003101012432104201035524F41AAA01C187
:0400000508000131BD
:00000001FF
